:100000000C94C3370C94F4370C94F4370C94F437F5
:100010000C94F4370C94F4370C94F4370C94F437B4
:100020000C94F4370C94F4370C94F4370C94F437A4
:100030000C94F4370D94E7AA0C94F4370C94F4372D
:100040000C94F4370C9414E90C94F4370C94F437B2
:100050000C94F4370C94F4370C94DBE50D949DAAC2
:100060000C94F4370D94D3810D94C9810C94F4371A
:100070000C94F4370C94F4370C94F4370C94F43754
:100080000D941A4A0C94F4370C94F4370C94F4370A
:100090000C94F4370C94F4370C94F4370C94F43734
:1000A0000C94F4370C94F4370D94EC490C94F43719
:1000B0000C94F4370C94F4370C94F4370C94F43714
:1000C0000C94F4370C94F4370C94F4370C94F43704
:1000D0000C94F4370C94F4370C94F4370C94F437F4
:1000E0000C94F437084AD73B3BCE016E84BCBFFD6D
:1000F000C12F3D6C74319ABD56833DDA3D00C77FF8
:1001000011BED9E4BB4C3E916BAAAABE0000008090
:100110003F05A84CCDB2D44EB93836A9020C50B91F
:10012000918688083CA6AAAA2ABE000000803F0744
:10013000634236B79BD8A71A39685618AEBAAB5582
:100140008C1D3CB7CC5763BD6DEDFD753EF6177247
:1001500031BF000000803F08000000BE9224491219
:100160003EABAAAA2ABECDCCCC4C3E00000080BE3D
:10017000ABAAAAAA3E00000000BF000000803F001A
:1001800000000000084178D3BB4387D1133D190E0E
:100190003CC3BD4282AD2B3E68EC8276BED98FE176
:1001A000A93E4C80EFFFBE01C4FF7F3F000000006E
:1001B00000000C9416520D9498B50C94923A0C943D
:1001C0003A6E0D94BCA40C94E1560C94553B0C94DF
:1001D00053470D9469820C94E8560C94FB3A0C94A6
:1001E00078D80D9477840C942B540C9469740D94E6
:1001F0001C800C945C430C94B5520C94529F0C944C
:10020000187F0C94AB830D94E3350C94604C0D94E3
:1002100070A40D9440820C94124D0D9421830C9483
:10022000C2400D9475820D94B4A40C9455D90C94CD
:10023000F6370C94B6400D945E820C94815F0C945A
:10024000A6830C9427500C947F4F0C9474440C9408
:10025000845F0C9494D90C94873B0C94CB8F0C94B2
:100260005EDA0C9457D50D94954B0D94E6310C94B1
:1002700019380C94FA850D949CA40C94755F0C9419
:1002800049470C94668A0C94D53B0C94795F0D9485
:1002900089A50C94F67C0C94EC3A0D94A6A40C94CD
:1002A000BB850C949F8E0C94AA440C949D830C9453
:1002B0002B410C94566F0C947A400C94DFD70D941C
:1002C000EE7E0D947D820C94D1560C9498400C9443
:1002D000415B0C94715F0C94EB830D94EBB50C9423
:1002E000DD680C94ABD60C948D860D9480830C94B1
:1002F000A3830C9486830D94C2A40C94CD560C94C5
:10030000568E0C94AA400C9480400C94423B0D9461
:1003100052A50C94EE480D94AAA40C9443D70C94C7
:10032000314D0C9458D50C94C43A0D947FA50D947E
:10033000A47D0D94B6490C94B24C0C943D8A0D9456
:1003400048A50C949A830D9471820C94C2D70C9496
:100350006E3B0C94BC4F0D9445370C9463380C9451
:100360003E9A0C944C900C944E530D941AA50C94F8
:10037000833C0C9467D90C940E670C949C3C0C94B1
:100380005F580C94C8400C94E9850C94844F0C94ED
:10039000363C0C946F590D949B490D944C450C942C
:1003A0002F4B0C94C5560C9447580C946C380C94F5
:1003B000CB4F0C9497830D9424A50D94AB7D0D9495
:1003C0002EA50D94AEA40C94BC3B0D9479820C9494
:1003D00071490C94D09A0D94D1490C94D3760D9414
:1003E0004E830C940F3C0C948C400C942E3C0C943B
:1003F0007A4F0C94BCD80C94254B0C94BC400D94B3
:100400008FA40C946A3C0C9457510D945CA50C94E9
:1004100061870D9480490C94B46A0C9469410C94E2
:100420007D5F0D9497820C94EC3B0D94C6A40C94C4
:10043000C9560D940BA50C94775F0C94B79C0C9443
:100440004C510C94DD560C94EE560C94718D0C941A
:10045000CE450C9491830C94CE3C0C9457D80C94BC
:1004600085380C94735F0C9406460C94DB580D94FD
:1004700075A50C94A3480C948E640C94D7D80C9456
:1004800027840C94D2850D9475A40D9409B60D940F
:1004900087A40D946D820C94876C0C94B53C0C94DD
:1004A000D25F0C9457590D9403A50C94FD650C94E0
:1004B0002F3B0C946D8D0C948D430C94344B0C9409
:1004C00015590C94744C0D946BA50C94AD830C943D
:1004D00009570C94B0400C9466590C94BC3E0C9493
:1004E0006A4C0C94D5560D9423800C941E500C9499
:1004F0009E400D94F67D0C9484490C9443790D94A0
:1005000013800C94773F0C94934C0C9458600C948B
:100510003D580D9436A50D9493A50C94D9790D945E
:10052000A0A40C94FD850D94B83A0C9424380C9436
:100530004E470C94EB560C943F4C0D9484820C94D3
:100540009D480C94C1560C94C88A0C94654C0D942B
:1005500096A40C9419710C94033C0D946E4B0C945E
:1005600036840C9492400C946F4C0D949DA50C9481
:10057000B0830C94163B0D948BA40C9486400C9481
:1005800007900C94963B0D9493A40C947F5F0C946D
:10059000274B0C94097F0D943EA50D944F820C942B
:1005A000E1690C94DE5F0C94D9560D9410A50C945F
:1005B000BD560C94F34C0C94A0830C94D33A0D9438
:1005C00065820C9449750C9494830C944E620D943E
:1005D00011820C94A93B0D94B8A40C947B5F0C94ED
:1005E000AB3A0C94294B0C94405E0C94D5D40C94EB
:1005F000D93C0C94698D0C94A03D0C944F600C94E4
:10060000A4400D948F820C94E5564E414E494E49BC
:100610005459494E46CDCCCC3D0AD7233C17B7D1CF
:100620003877CC2B329595E6241FB14F0A00002075
:10063000410000C84200401C4620BCBE4CCA1B0EF4
:100640005AAEC59D7400407A10F35A00A0724E183D
:10065000090010A5D4E80000E87648170000E40B74
:1006600054020000CA9A3B000000E1F5050000803A
:10067000969800000040420F000000A08601000094
:1006800000102700000000E80300000000640000E4
:100690000000000A00000000000100000000002C23
:1006A00076D888DC674F0823DFC1DFAE59E1B1B7E8
:1006B00096E5E3E453C63AE651997696E8E6C284B5
:1006C00026EB898C9B62ED407C6FFCEFBC9C9F40CD
:1006D000F2BAA56FA5F490055A2AF75C936B6CF9F2
:1006E000676DC11BFCE0E40D47FEF520E6B500D0C8
:1006F000ED902E0300943577050080841E080000DD
:10070000204E0A000000C80C333333330F986E12AA
:10071000831141EF8D2114893BE65516CFFEE6DBB0
:1007200018D1844B381BF77C1D901DA4BBE42420FA
:100730003284725E228100C9F124ECA1E53D275587
:100740004E4C4F41442046494C414D454E54004C7F
:100750004F41442046494C414D454E540046494C7A
:10076000414D454E54204348414E47450050494471
:10077000204175746F74756E65202A005049442DB0
:1007800044202A005049442D49202A005049442D34
:1007900050202A0020082046616374002008204D64
:1007A0006178002008204D696E004F6666004F6E2C
:1007B000004175746F74656D7000565472617620D7
:1007C0004D696E00566D696E00566D61782045006A
:1007D000566D6178205A00566D6178205900566D2B
:1007E0006178205800416D6178204500416D617845
:1007F000205A00416D6178205900416D6178205880
:1008000000412D54726176656C00412D5265747201
:1008100061637400416363656C0056652D4A6572BF
:100820006B00565A2D4A65726B0056592D4A6572F7
:100830006B0056582D4A65726B0050726F626520CE
:100840005A204F66667365740050726F6265205956
:10085000204F66667365740050726F626520582081
:100860004F666673657400452073746570732F6DF1
:100870006D005A2053746570732F6D6D00592053AD
:10088000746570732F6D6D00582053746570732FED
:100890006D6D00416476616E6365642053657474A8
:1008A000696E6773003F0043616E63656C00496E5B
:1008B0006974004D34323800496E697469616C693D
:1008C0007A6520454550524F4D0046696C616D6513
:1008D0006E740054656D7065726174757265005355
:1008E000746570732F6D6D0050726F6265204F6676
:1008F0006673657473004A65726B00416363656C6F
:1009000065726174696F6E0056656C6F63697479A6
:100910000053657420486F6D65204F66667365747B
:100920007300436F6E66696775726174696F6E00FC
:100930003F004E65787420506F696E7400446F6E8E
:1009400065004E657874003F0043616E63656C20FE
:100950004F626A656374004E4F005945530043610E
:100960006E63656C204F626A656374203D004D6163
:10097000696E0053746F770053572D4D6F64650097
:100980004465706C6F790053656C662D54657374A3
:1009900000526573657400426564004E6F7A7A6C2C
:1009A000650046616E20537065656400436F6E6636
:1009B000696775726174696F6E00526573746F72E6
:1009C000652044656661756C7473004C6F616420CA
:1009D00053657474696E67730053746F7265205346
:1009E000657474696E677300507265686561742020
:1009F0002420436F6E6600506F776572204F7574C8
:100A0000616765004F6666004F6E0052756E6F75C8
:100A1000742053656E736F7200424C546F75636837
:100A20000050726F6265205A204F666673657400CD
:100A3000416476616E6365642053657474696E67A2
:100A400073004D61696E004D3730322054256400CB
:100A50004D36303020423020542564004D3730323E
:100A6000203B2564004D37303120542564004D373C
:100A70003032004D373031004D36303020423000BA
:100A80004D61696E00436F6E74696E7565004F66E7
:100A900066004F6E0052756E6F75742053656E73ED
:100AA0006F72005075726765206D6F7265005245F8
:100AB00053554D45204F5054494F4E533A005052D4
:100AC000494E54205041555345440020204E6F7AE2
:100AD0007A6C653A20005061726B696E672E2E2E1B
:100AE0000000005761697420666F720066696C616E
:100AF0006D656E74206368616E676500746F207346
:100B000074617274005761697420666F720066695F
:100B10006C616D656E7420756E6C6F616400004E63
:100B20006F7A7A6C652068656174696E6700506CD5
:100B30006561736520776169742E2E2E00005072F6
:100B400065737320627574746F6E00746F206865CE
:100B50006174206E6F7A7A6C650000496E736572FD
:100B6000742066696C616D656E7400616E642070DE
:100B70007265737320627574746F6E00746F206396
:100B80006F6E74696E7565005761697420666F7267
:100B90000066696C616D656E74206C6F6164000045
:100BA000507265737320427574746F6E00746F2099
:100BB000726573756D65207072696E74000057619F
:100BC000697420666F72207072696E7400746F2091
:100BD000726573756D652E2E2E0000576169742045
:100BE000666F720066696C616D656E7420707572F7
:100BF000676500003E2000256C642E25696D004568
:100C00007874727564656420546F74616C003E2062
:100C1000004C6F6E67657374204A6F622054696D73
:100C200065003E2000546F74616C205072696E74D0
:100C30002054696D6500436F6D706C657465640068
:100C40003A20005072696E7420436F756E74003ADA
:100C500020003135300035004245443A20415443AC
:100C60002031303447542D320052756E61776179EE
:100C70002057617463683A204F4E004D61782054CC
:100C8000656D7000333135004D696E2054656D70AF
:100C900000350045313A204550434F532031303024
:100CA0004B005053550047656E6572696300507282
:100CB0006F746F636F6C00312E3000426175640099
:100CC00032353030303000437265616C697479338D
:100CD000442052414D505300556E69666965642049
:100CE000426564204C6576656C696E670045787472
:100CF00072756465727300310074696E796D616339
:100D000068696E657333642E636F6D003530302013
:100D1000537550655200323032312D30342D313818
:100D200000322E302E375F4457372E33004D61721C
:100D30006C696E005072696E7465722053746174D0
:100D40007300546865726D6973746F727300426FDB
:100D500061726420496E666F005072696E746572CC
:100D600020496E666F004D61696E004D3130303044
:100D70000053746F70205072696E74005265737501
:100D80006D65205072696E7400506F776572204FE8
:100D90007574616765004D3139305335350A473216
:100DA000380A47323950310A47323950330A47320C
:100DB0003953310A47323953300A47323946302ED7
:100DC000300A473239410A4D313034533231350A15
:100DD0004732380A4D313039533231350A473158AC
:100DE0003135305931353046353030300A47315A97
:100DF000300A4D3530300A4D3430300A4D313137FC
:100E000020536574205A204F6666736574004D3117
:100E10003036533132380A4D333033433853323160
:100E2000354530550A4D3530300A4D313137205077
:100E300049442054756E6520446F6E65004D31390C
:100E4000305335350A4D313034533231350A47325B
:100E5000380A4732394C310A47312058313030593D
:100E600031303046353030300A47315A30004D3558
:100E700030300A4D3131372053657474696E6773B1
:100E80002053746F726564005072657020666F72D3
:100E9000205A2041646A7573740050494420547587
:100EA0006E650053746F72652053657474696E6764
:100EB00073005365747570004D61696E003F0042A8
:100EC00061636B0053746F70005072696E742066BA
:100ED000726F6D204D65646961004368616E67657E
:100EE000204D65646961004D32310041626F757457
:100EF000205072696E746572004368616E67652088
:100F000046696C616D656E74004C6576656C696EE2
:100F10006720546F6F6C7300436F6E6669677572FC
:100F20006174696F6E0054656D706572617475727D
:100F300065004D6F74696F6E00486F737420537451
:100F4000617274004E6F204D656469610052657373
:100F5000756D65205072696E740043616E63656CD7
:100F6000204F626A6563740054756E650053746F38
:100F700070205072696E74005061757365205072F4
:100F8000696E7400496E666F2053637265656E000A
:100F90003F005374617274205072696E7400436133
:100FA0006E63656C005072696E740043616E6E6FA3
:100FB0007420656E746572207375626469723A207C
:100FC00000022E2E004D61696E002100486F74658D
:100FD0006E6420746F6F20636F6C64004261636B9A
:100FE0000050726F63656564004F6666004F6E0067
:100FF000536F667420456E6473746F7073004D6F29
:1010000074696F6E0044697361626C652053746526
:101010007070657273004D3834004D343820507252
:101020006F62652054657374004732384F0A4D343F
:101030003820503130004C6576656C20436F726EFD
:1010400065727300556E6966696564204265642047
:101050004C6576656C696E6700486F6D65205A0057
:101060004732385A00486F6D652059004732385969
:1010700000486F6D6520580047323858004175743C
:101080006F20486F6D65004D61696E005072656834
:10109000656174202420456E640050726568656146
:1010A000742024204265640054656D70657261741B
:1010B00075726500436F6F6C646F776E0050726578
:1010C0006865617420240046616E20537065656414
:1010D000207E00426564004E6F7A7A6C65004D6137
:1010E000696E0050726F6265205A204F66667365A4
:1010F0007400416476616E6365204B00466C6F77C7
:101100000046616E205370656564207E0042656410
:10111000004E6F7A7A6C65005370656564004D61AE
:10112000696E005A2056616C7565004732380A4D69
:10113000313930205325690A4D3130392053256922
:101140000A473239205031004265642054656D7081
:1011500000486F74656E642054656D70002E2569BB
:10116000004732395036432D00486569676874205E
:10117000416D6F756E740041646A757374204D65BE
:101180007368204865696768740046696E65205415
:10119000756E6520436C6F73657374004732395008
:1011A00034540046696E652054756E6520416C6C40
:1011B0000047323950345239393954004732380AED
:1011C00047323643504825694225690056616C69AB
:1011D0006461746520437573746F6D204D65736829
:1011E000004732380A473236435049310056616C65
:1011F0006964617465204D6573682028242900475F
:1012000032380A47323643504930004732394A258E
:1012100069004C6576656C204D65736800536964A0
:101220006520506F696E74730047726964204D6564
:101230007368204C6576656C696E6700332D506F5E
:10124000696E74204C6576656C696E67004732394B
:101250004A3000473239503352432E2569004D61E0
:101260006E75616C2046696C6C2D696E0047323971
:10127000503242543000536D6172742046696C6C78
:101280002D696E00473239503354300046696C6C1A
:101290002D696E20416D6F756E74004D6573682009
:1012A000696E76616C6964617465642E0A00496ECA
:1012B000666F2053637265656E00496E76616C6976
:1012C0006461746520436C6F7365737400473239D1
:1012D0004900496E76616C696461746520416C6C8B
:1012E00000436F6E74696E756520426564204D65BC
:1012F0007368004732395031430046696C6C2D6980
:101300006E204D657368004275696C6420436F6C94
:1013100064204D657368004732394E503100427584
:10132000696C6420437573746F6D204D657368003C
:101330004732380A4D31393049310A4D3130394957
:10134000310A47323950310A4D31303453300A4D69
:101350003134305330004275696C64204D657368D8
:1013600020282429004732380A4D31393049300AC3
:101370004D31303949300A47323950310A4D313018
:101380003453300A4D3134305330004732392563FD
:1013900025690A4D31313720004D65736820256974
:1013A000204C6F61646564004D6573682025692079
:1013B0005361766564005361766520426564204D13
:1013C000657368004C6F616420426564204D6573ED
:1013D00068004D656D6F727920536C6F74004E6FAD
:1013E0002053746F72616765004732395034582555
:1013F0007359257352256900202D2D2D2D2D005A4E
:101400003A00593A00486F6D696E672058595A0082
:10141000473238004F6666205072696E74657220DC
:101420004261636B757000473239532D31004F753F
:101430007470757420666F722043535600473239BA
:101440005431004F757470757420666F7220486F48
:101450007374004732395430004D657368204C6511
:1014600076656C696E670045646974204D657368C4
:101470000056616C6964617465204D657368004D48
:10148000616E75616C6C79204275696C64204D6584
:10149000736800473239493939390A47323950328D
:1014A000425430004275696C64204D6573680037A2
:1014B0002E205361766520426564204D6573680077
:1014C000362E2046696E652054756E6520416C6C21
:1014D000004732395034523939395400352E2056AC
:1014E000616C6964617465204D65736800342E20F9
:1014F00046696E652054756E6520416C6C004732FC
:10150000395034523939395400332E2056616C69C0
:1015100064617465204D65736800322E20536D61DF
:1015200072742046696C6C2D696E004732395033F5
:10153000543000312E204275696C6420436F6C6416
:10154000204D657368004732394E503100556E6941
:101550006669656420426564204C6576656C696ED9
:1015600067004661646520486569676874004F7567
:10157000747075742055424C20496E666F00473276
:1015800039570055424C20546F6F6C73004F75747F
:10159000707574204D657368204D6170004D6573E2
:1015A000682053746F72616765004D6573682045EC
:1015B00064697400537465702D42792D537465709D
:1015C0002055424C00416374697661746520554230
:1015D0004C00473239410044656163746976617437
:1015E000652055424C0047323944004D6F74696F95
:1015F0006E00434F4D4D554E49434154494F4E00A7
:1016000044525952554E004552524F525300494E82
:10161000464F004543484F004F46460A0046616426
:1016200065204865696768742000426564204C65E0
:1016300076656C696E6720004661696C656420742C
:101640006F20656E61626C6520426564204C657632
:10165000656C696E670A00496E76616C6964206D1D
:101660006573682E0A0076616C69640A53746F7240
:1016700061676520736C6F743A2000696E004D6578
:10168000736820697320003F557365203020746FA4
:1016900020003F496E76616C69642073746F7261DB
:1016A000676520736C6F742E0A003F454550524F9A
:1016B0004D2073746F72616765206E6F7420617660
:1016C00061696C61626C652E0A004D6573682070FB
:1016D0006F696E74206F7574206F662072616E671B
:1016E000650A004D34323120696E636F7272656332
:1016F0007420706172616D657465722075736167C5
:10170000650A00446576696174696F6E0025533A15
:101710002025730046696E6973686564210A003A82
:10172000207A3A2000206F662000476F696E67209C
:10173000746F3A20580043570A00206469723A00D7
:1017400020616E676C653A00537461727420726137
:10175000646975733A004D343820506F696E7400B7
:1017600025533A2025642F256400506F73697469EE
:101770006F6E696E67207468652070726F62652E87
:101780002E2E0A003F4C656773206F66206D6F76C2
:10179000656D656E7420696D706C61757369626CDE
:1017A000652028302D3135292E0A003F2028582C5D
:1017B0005929206F7574206F6620626F756E64738F
:1017C0002E0A0050726F6265206F7574206F66205C
:1017D000626F756E6473003F53616D706C6520734A
:1017E000697A65206E6F7420706C61757369626CC4
:1017F000652028342D3530292E0A004D3438205AE2
:101800002D50726F62652052657065617461626906
:101810006C69747920546573740A003F28562965F1
:1018200072626F7365206C6576656C20696D706C93
:1018300061757369626C652028302D34292E0A0089
:101840005374616E64617264204465766961746981
:101850006F6E3A20002052616E67653A2000204D7D
:1018600061783A2000204D696E3A20002053696764
:101870006D613A20004D65616E3A20005741524E2D
:10188000494E4721204C6F77205A204A65726B20C1
:101890006D6179206C65616420746F20756E77616D
:1018A0006E746564207061757365732E0A004F460F
:1018B00046004F4E0020204D61783A200020002045
:1018C000204D696E3A2000536F667420656E647314
:1018D000746F70733A20004D32342053256C6420AD
:1018E00054256C64004739322E3920452573004752
:1018F0003120462564004739322E39205A2573009D
:101900004731205A302046323030004731205825A8
:101910007320592573204633303030004D34323037
:1019200020532569205A2573004D3130362050252B
:101930006920532569004D3230302044257300471B
:10194000323852305859004739322E39204530202C
:101950005A300A47315A2573004D3130392053250A
:1019600069004D31393020532569004D3432302023
:101970005330205A300020496E76616C69642065CE
:1019800078747275646572200047322F4733206285
:10199000616420706172616D65746572730A0053D1
:1019A0006C6565702E2E2E005A2050726F62652075
:1019B00050617374204265640A005A2050726F624D
:1019C0006520506173742042656400205A3A2000FB
:1019D00020593A200042656420583A20004D657332
:1019E0006820706F696E74206F7574206F66207246
:1019F000616E67650A004D302053746F70004D3181
:101A00002053746F7000436C69636B20746F2052B5
:101A10006573756D652E2E2E004E6F204D6F7665A9
:101A20002E00456E642066696C65206C6973740ACB
:101A300000426567696E2066696C65206C69737425
:101A40000A004E6F206D656469610A005265737506
:101A50006D696E6720534400286E6F2066696C655F
:101A6000290043757272656E742066696C653A2050
:101A7000005072696E742074696D653A20000A53D3
:101A8000746174733A2046696C616D656E7420757B
:101A90007365643A20002C204C6F6E676573742068
:101AA0006A6F623A2000546F74616C2074696D65CE
:101AB0003A200053746174733A20002C2046616907
:101AC0006C65643A20002C2046696E697368656411
:101AD0003A20005072696E74733A20005374617436
:101AE000733A2000436F6F6C696E672E2E2E00488C
:101AF000656174696E672E2E2E0045202553006F98
:101B00006B006F66660013160E1607160016F215A8
:101B100044454255473A004D313133205300426528
:101B20006420436F6F6C696E672E2E2E00426564D1
:101B30002048656174696E672E2E2E003530302086
:101B40005375506552204F46462E002F2F004D31C1
:101B5000343520533C696E6465783E206F7574207F
:101B60006F662072616E67652028302D31290A006A
:101B7000205200416363656C65726174696F6E3AEF
:101B80002050004D32303620580046523A00204650
:101B90006C6F773A20003A200020536572766F20F0
:101BA00000206F7574206F662072616E67650A0091
:101BB000536572766F200020643A0020693A002055
:101BC000703A00496E76616C69642065787472754C
:101BD0006465720A0020643A0020693A0020703A75
:101BE0000064697300656E0043290A0061626C65D8
:101BF0006420286D696E2074656D702000436F6CE1
:101C00006420657874727564657320617265200064
:101C100046696C616D656E742072756E6F757420A7
:101C200064697374616E636520286D6D293A2000C4
:101C300046696C616D656E742072756E6F75742087
:101C4000004F666673657473204170706C696564DB
:101C5000004572723A20546F6F2066617221005401
:101C60006F6F206661722066726F6D2072656665A7
:101C700072656E636520706F696E740A0045455029
:101C8000524F4D204F4B0A002E0A002028302D3194
:101C90003029002076616C7565206F7574206F6641
:101CA0002072616E676500416476616E6365204BEA
:101CB0003D00506F7765722D6C6F73732072656392
:101CC0006F7665727920004D383400446F6E652060
:101CD0007072696E74696E672066696C650A004D82
:101CE0003737004D3331004361703A004D45415460
:101CF0005041434B00434F4F4C45525F54454D506C
:101D000045524154555245004348414D4245525F6A
:101D100054454D5045524154555245004241425957
:101D20005354455050494E470041524353004D4F84
:101D300054494F4E5F4D4F44455300544845524D12
:101D4000414C5F50524F54454354494F4E004C4F05
:101D50004E475F46494C454E414D45004155544F15
:101D60005245504F52545F53445F5354415455535E
:101D70000053445F57524954450052455045415421
:101D8000005344434152440050524F4D50545F530E
:101D90005550504F525400454D455247454E4359BA
:101DA0005F50415253455200434153455F4C4947B0
:101DB00048545F4252494748544E45535300544F8C
:101DC00047474C455F4C494748545300534F46548E
:101DD000574152455F504F574552004255494C4478
:101DE0005F50455243454E54004C4556454C494E74
:101DF000475F44415441005A5F50524F42450052A0
:101E0000554E4F5554004155544F4C4556454C0086
:101E10005052494E545F4A4F420050524F4752452C
:101E20005353004155544F5245504F52545F5445FF
:101E30004D5000564F4C554D455452494300454571
:101E400050524F4D0042494E4152595F46494C4510
:101E50005F5452414E534645520053455249414CFE
:101E60005F584F4E5F584F4646004649524D5741C6
:101E700052455F4E414D453A4D61726C696E20325C
:101E80002E302E375F4457372E3320544D334420A5
:101E900035534D444255202841707220323520324E
:101EA0003032312030303A30303A34302920534FFC
:101EB000555243455F434F44455F55524C3A687411
:101EC0007470733A2F2F6769746875622E636F6D33
:101ED0002F496E73616E6974794175746F6D6174A9
:101EE000696F6E2F4D61726C696E2F747265652F0C
:101EF000437265616C6974794477696E5F322E3024
:101F00002050524F544F434F4C5F56455253494F08
:101F10004E3A312E30204D414348494E455F545989
:101F200050453A353030205375506552204558544D
:101F300052554445525F434F554E543A3120555502
:101F400049443A63656465326132662D34316132E9
:101F50002D343734382D396231322D6335356336BF
:101F6000326633363766660A0050726F6265204FFC
:101F70006666736574205A0050726F6265204F6602
:101F800066736574205A00290A0020746F20003F90
:101F90005A206F7574206F662072616E6765202805
:101FA00000290A0020746F20003F59206F757420AB
:101FB0006F662072616E676520282D00290A002057
:101FC000746F20003F58206F7574206F6620726117
:101FD0006E676520282D0050726F6265204F66661F
:101FE00073657420580043616E6E6F74206F706566
:101FF0006E2073756264697220002569730025691B
:102000006D20256973002569682025696D20256983
:102010007300256964202569682025696D2025697C
:102020007300256979202569642025696820256960
:102030006D202569730023646566696E65204445DB
:102040004641554C545F00626564004B6420004B70
:102050006920004B702000504944204175746F7412
:10206000756E652066696E697368656421205075B8
:102070007420746865206C617374204B702C204B45
:102080006920616E64204B6420636F6E7374616EAF
:1020900074732066726F6D2062656C6F7720696E55
:1020A000746F20436F6E66696775726174696F6ED5
:1020B0002E680A00504944204175746F74756E652E
:1020C000206661696C6564212074696D656F757443
:1020D0000A00504944204175746F74756E6520661E
:1020E00061696C6564212054656D706572617475F9
:1020F000726520746F6F20686967680A00204B64FE
:102100003A2000204B693A2000204B703A200020F2
:10211000436C617373696320504944200A00204E68
:102120006F206F76657273686F6F740A0020547544
:102130003A2000204B753A2000206D61783A20004B
:10214000206D696E3A200020643A200020626961A7
:10215000733A2000504944204175746F74756E6560
:102160002073746172740A00504944204175746F81
:1021700074756E65206661696C6564212054656DB7
:10218000706572617475726520746F6F206869671D
:10219000680A00504944204175746F74756E65007B
:1021A000504944204175746F74756E65206661698D
:1021B0006C656421204261642068656174657220E9
:1021C00069640A004572723A207574663820666F39
:1021D0006E74206E6F7420696E697469616C697ABF
:1021E00065642E004572723A207574663820666FF9
:1021F0006E74206E6F7420696E697469616C697A9F
:1022000065642E004572723A207574663820666FD8
:102210006E74206E6F7420696E697469616C697A7E
:1022200065642E0000FE0003FF8007C7C00701E0C1
:102230000000E00000F00000700400700E00701F4D
:1022400000703F80F00E00E00F01E007C7C003FF01
:102250008000FE0000FE0003FF8007C7C00F01E002
:102260000E00E03F80F01F00700E00700400700050
:1022700000700000F00000E00701E007C7C003FFA6
:102280008000FE000E000E000E000E000E000E007C
:102290000E000E007FC03F801F000E0004000400EF
:1022A0000E001F003F807FC00E000E000E000E00CB
:1022B0000E000E000E000E00FFFFFF7F80FFC0FF2C
:1022C000C0FFC07F807F80FFC0FFC0FFC03F001EF7
:1022D000000C0042656400456E636C6F7375726537
:1022E000002568753A2530326875002530326875EA
:1022F0003A25303268750020202020202020002040
:10230000202020001FE0201020102010102010207E
:102310002010201030300840048003001FE03FF000
:102320003FF03FF01FE01FE03FF03FF03FF00FC0F5
:10233000078003003FFFF038007030FC3020FC10B5
:102340002078102030102C00D02E31D02F7BD02FB1
:102350007BD02E31D02C00D020301020781020FCE3
:102360001030FC303800703FFFF03FFFF038007055
:102370003186302387102787902F87D02F03D020D6
:1023800030102078102078102030102F03D02F87A5
:10239000D02787902387103186303800703FFFF0B8
:1023A0001FFFF81FFFF80410400208200208200455
:1023B00010400820801041001041000820800410C7
:1023C000400000001FFFF81FFFF8FFFFFF80000123
:1023D0008E00E19F01F19381399F81F99F81F99FDF
:1023E000B9F98F28F18038018000019FFFF99174BD
:1023F000999B06A99B54A99B56A99B54999FFFF9A9
:10240000FFFFFF3530302053755065522052656113
:1024100064792E005072696E74696E672E2E2E00DC
:102420006E6F74696669636174696F6E20006361C1
:102430006E63656C005072696E742041626F7274D5
:102440006564004469736D69737300554920416286
:102450006F72746564004D323520500A4D3234007D
:102460005072696E742050617573656400526573B3
:10247000756D650055492050617573650050617533
:1024800073696E672E2E2E00726573756D65004D33
:1024900032340050726F6265205A204F6666736551
:1024A000740052756E6F75742044697374206D6D7D
:1024B000004C6F6164206D6D00556E6C6F6164201F
:1024C0006D6D0046696C2E204469612E00452069BF
:1024D0006E206D6D5E3300416476616E6365204BE6
:1024E000004D33303320553120452569205325696F
:1024F00000000C0F00FE07022503BB017FFE08FE53
:1025000008FE05080806000040F0C8888898781082
:10251000050808060000C0F88888888888F805053E
:10252000050600012030F8302005080806000020CC
:1025300070F820202020E00509090600FF2070A87F
:10254000A8B888887020070505070001D86C366C8C
:10255000D80509090600FFF8A88888888888A8F89F
:10256000050A0A0600FE205050505088A8A888701E
:1025700003030306000340A040FFFFFFFFFFFFFF30
:10258000FFFFFFFFFFFFFFFFFFFFFFFFFFFFFF005A
:1025900000000605FF01070706020080808080809A
:1025A0000080030303060105A0A0A005060606009F
:1025B0000050F85050F8500509090600FF2070A897
:1025C000A07028A87020050707060000C8C81020C2
:1025D00040989805070706000040A0A040A8906812
:1025E0000103030602058080800309090601FF201C
:1025F00040408080804040200309090601FF804060
:102600004020202040408005070706000020A870D9
:102610002070A8200505050600012020F8202002D2
:1026200003030601FFC04080050101060003F80214
:102630000202060100C0C0050707060000081010CE
:1026400020404080050707060000708898A8C888C9
:102650007003070706010040C040404040E0050706
:1026600007060000708808102040F80507070600DC
:1026700000F80810300888700507070600001030C1
:102680005090F81010050707060000F880F00808C1
:102690008870050707060000304080F088887005C4
:1026A0000707060000F8081010202020050707067D
:1026B0000000708888708888700507070600007021
:1026C000888878081060020505060100C0C000C0B7
:1026D000C00206060601FFC0C000C0408003050519
:1026E0000601012040804020050303060002F80097
:1026F000F803050506010180402040800507070614
:1027000000007088102020002005070706000070D8
:1027100088B8A8B88070050707060000708888F898
:10272000888888050707060000F04848704848F088
:1027300005070706000070888080808870050707FD
:10274000060000F04848484848F005070706000022
:10275000F88080F08080F8050707060000F8808088
:10276000F0808080050707060000708880809888C8
:1027700070050707060000888888F888888803079E
:1027800007060100E04040404040E0050707060022
:1027900000381010101090600507070600008890A0
:1027A000A0C0A09088050707060000808080808078
:1027B00080F805070706000088D8A888888888055B
:1027C00007070600008888C8A898888805070706B4
:1027D000000070888888888870050707060000F068
:1027E0008888F08080800507070600007088888848
:1027F000A89068050707060000F08888F0A0908878
:1028000005070706000070888070088870050707B4
:10281000060000F8202020202020050707060000E1
:102820008888888888887005070706000088888857
:102830008850502005070706000088888888A8A8C7
:102840005005070706000088885020508888050733
:102850000706000088885020202020050707060072
:1028600000F80810204080F80309090601FFE08005
:10287000808080808080E00507070600008040405F
:10288000201010080309090601FFE0202020202065
:102890002020E005030306000520508805010106FD
:1028A00000FEF80303030601058040200505050628
:1028B000000070087888780507070600008080F01F
:1028C000888888F0050505060000708080887005FE
:1028D0000707060000080878888888780505050637
:1028E00000007088F080700507070600003048403F
:1028F000E04040400507070600FE70888888780899
:10290000700507070600008080F088888888030724
:10291000070601004000C0404040E00409090601EC
:10292000FE10003010101010906005070706000020
:1029300080808890E09088030707060100C040402F
:10294000404040E0050505060000D0A8A8A8A8055D
:102950000505060000B0C888888805050506000042
:1029600070888888700507070600FEF0888888F060
:1029700080800507070600FE7888888878080805A3
:102980000505060000B0C88080800505050600002A
:1029900078807008F00507070600002020F8202046
:1029A0002018050505060000888888986805050533
:1029B00006000088888850200505050600008888E4
:1029C000A8A8500505050600008850205088050776
:1029D000070600FE8888885020408005050506000F
:1029E00000F8102040F80309090601FF204040408C
:1029F00080404040200109090602FF8080808080DD
:102A0000808080800309090601FF8040404020400B
:102A100040408005030306000248A890FF486F6D00
:102A2000696E67204661696C6564006F70656E0051
:102A3000545249474745524544003A200066696C64
:102A4000616D656E74007A5F6D696E00795F6D69A6
:102A50006E00785F6D696E005265706F7274696E9A
:102A60006720656E6473746F70207374617475731E
:102A70000A0020746F6F206C6F6E67206578747227
:102A80007573696F6E2070726576656E7465640A21
:102A90000020636F6C6420657874727573696F6E63
:102AA0002070726576656E7465640A00486F6D65A6
:102AB000202573257325732046697273740057614E
:102AC000726E696E673A20486F6D696E6720427555
:102AD0006D702044697669736F72203C20310A0062
:102AE00002020400000000000000000000000000DE
:102AF00000FF430000FA430000FA430000004100D9
:102B000000004100000040FFFFFF00000001000046
:102B1000000100008000555555000000400033338F
:102B20003300AAAA2A004992240000002000C7719D
:102B30001C0099991900D1451700555515003BB156
:102B400013002449120011111100000010000F0F92
:102B50000F00E3380E0043790D00CCCC0C00C330DD
:102B60000C00E8A20B0064210B00AAAA0A00703D29
:102B70000A009DD80900427B090092240900DCD399
:102B80000800888808001042080000000800F0C112
:102B900007008787070075500700711C07003EEB90
:102BA0000600A1BC06006990060066660600703E3D
:102BB00006006118060017F4050074D105005BB02B
:102BC0000500B29005006272050055550500783980
:102BD0000500B81E0500050505004EEC040087D46D
:102BE0000400A1BD040090A7040049920400C17D27
:102BF0000400EE690400C7560400444404005C323B
:102C000004000821040041100400000004003FF00B
:102C10000300F8E0030026D20300C3C30300CCB5D1
:102C200003003AA803000A9B0300388E0300C0810A
:102C300003009F750300D0690300505E03001D531D
:102C4000030034480300913D030033330300162989
:102C50000300381F030097150300300C0300030323
:102C600003000BFA020049F10200BAE802005CE03E
:102C700002002DD802002DD0020059C80200B0C0B9
:102C8000020031B90200DAB10200AAAA0200A0A330
:102C90000200BC9C0200FA9502005C8F0200DF88F3
:102CA000020082820200457C020027760200277023
:102CB0000200436A02007C640200D05E02003F59B9
:102CC0000200C8530200FFFDFCFAF8F6F4F2F0EE41
:102CD000ECEAE9E7E5E3E1E0DEDCDAD9D7D5D4D206
:102CE000D0CFCDCBCAC8C7C5C3C2C0BFBDBCBAB99F
:102CF000B7B6B4B3B2B0AFADACAAA9A8A6A5A4A20A
:102D0000A1A09E9D9C9A99989795949392908F8E4E
:102D10008D8B8A8988878684838281807F7E7D7B74
:102D20007A797877767574737271706F6E6D6C6B7B
:102D30006A696867666564636261605F5E5D5C5B6B
:102D40005A5958585756555453525150504F4E4D4A
:102D50004C4B4A4A49484746464544434242414013
:102D60003F3E3E3D3C3B3B3A3938383736353534CB
:102D70003332323130302F2E2E2D2C2B2B2A292975
:102D800028272726252524232322212120201F1E12
:102D90001E1D1C1C1B1B1A191918181716161515A1
:102DA00014131312121111100F0F0E0E0D0D0C0C27
:102DB0000B0A0A09090808070706060505040403A3
:102DC0000302020100000000FF430000FA4300007C
:102DD000FA430000000000000000000000005365FE
:102DE0007474696E67732053746F7265640045452F
:102DF00050524F4D20496E697469616C697A6564FF
:102E00000A003F556E61626C6520746F20736176B5
:102E100065206D65736820646174612E0A003F55FA
:102E20006E61626C6520746F206C6F6164206D65EB
:102E3000736820646174612E0A00556E6966696565
:102E40006420426564204C6576656C696E67003B62
:102E500020003A0A0020204D363033200020440064
:102E600020204D34313220530046696C616D656E0F
:102E7000742072756E6F75742073656E736F723A1D
:102E8000002055004C0046696C616D656E74206CC5
:102E90006F61642F756E6C6F6164206C656E677412
:102EA00068733A0020204D393030204B004C696E59
:102EB00065617220416476616E63653A0020204D41
:102EC0003835312058005A2D50726F6265204F6698
:102ED000667365740020204D343133205300506FE9
:102EE0007765722D4C6F7373205265636F766572D0
:102EF000793A0020440020490020204D333034200E
:102F0000500020440020490020204D333031205013
:102F1000005049442073657474696E67733A0020E9
:102F2000460020480020204D3134352053004D61AB
:102F300074657269616C2068656174757020706178
:102F400072616D65746572733A00206D65736865B2
:102F5000732E0A0A00454550524F4D2063616E2082
:102F6000686F6C642000416374697665204D6573F9
:102F70006820536C6F743A200020204D343230208A
:102F8000530020204D323036205800486F6D6520A8
:102F90006F66667365743A00205800205300202045
:102FA0004D323035204200416476616E6365643A8B
:102FB00020423C6D696E5F7365676D656E745F740A
:102FC000696D655F75733E20533C6D696E5F666524
:102FD0006564726174653E20543C6D696E5F747205
:102FE0006176656C5F66656564726174653E2058E4
:102FF0003C6D61785F785F6A65726B3E20593C6D0D
:1030000061785F795F6A65726B3E205A3C6D6178CA
:103010005F7A5F6A65726B3E20453C6D61785F65E3
:103020005F6A65726B3E0020540020520020204DE4
:10303000323034205000416363656C65726174699D
:103040006F6E2028756E6974732F7332293A205081
:103050003C7072696E745F616363656C3E20523CC4
:10306000726574726163745F616363656C3E205462
:103070003C74726176656C5F616363656C3E0020D1
:10308000204D3230312058004D6178696D756D20CA
:10309000416363656C65726174696F6E2028756E3B
:1030A0006974732F7332293A0020204D3230332057
:1030B00058004D6178696D756D2066656564726153
:1030C0007465732028756E6974732F73293A0053E1
:1030D000746570732070657220756E69743A002093
:1030E000440020204D323030205300204469736169
:1030F000626C65640A0046696C616D656E7420736C
:10310000657474696E67733A0020204D313439203C
:1031100043203B20556E69747320696E2043656CB3
:10312000736975730A0020286D6D290020204732CD
:1031300031202020203B20556E69747320696E2059
:103140006D6D003F4D65736820746F6F2062696715
:1031500020666F7220454550524F4D2E0A000000E8
:10316000FA430000C843000070410000964200008E
:10317000A0420000A0420000C8430000BE42E80395
:103180000000BC020000640000004B00000024F4BA
:10319000D43050C38E20C2A24017828B7011127A95
:1031A000910D816CD90AA861E108C7586607615181
:1031B00043061E4B5D05C145A7041A411104093D94
:1031C0009803713931034036DB0265339102D43004
:1031D0005402802E1D02632CEE01752AC501B02811
:1031E000A001102781018F2564012B244B01E022CF
:1031F0003401AC211F018D200D01801FFC00841EB5
:10320000ED00971DDF00B81CD200E61BC600201B96
:10321000BC00641AB200B219A8000A19A0006A180A
:103220009900D117910040178B00B5168400311614
:103230007E00B31579003A157300C7146F00581457
:103240006A00EE1366008813630025135E00C71240
:103250005B006C12570015125400C111510070111F
:103260004F0021114B00D61049008D104700461029
:10327000440002104200C00F4000800F3E00420F89
:103280003C00060F3B00CB0E3800930E37005C0E5F
:103290003500270E3400F30D3200C10D3100900DC2
:1032A0003000600D2E00320D2D00050D2C00D90CC4
:1032B0002B00AE0C2900850C29005C0C2700350C76
:1032C00027000E0C2600E80B2400C40B2400A00BE2
:1032D00023007D0B23005A0B2100390B2100180B12
:1032E0002000F80A1F00D90A1E00BB0A1E009D0A12
:1032F0001D00800A1D00630A1C00470A1B002C0ADF
:103300001B00110A1A00F7091A00DD091900C40987
:103310001900AB091900920917007B09180063090D
:1033200017004C09160036091600200916000A0974
:103330001500F5081500E0081400CC081400B808C2
:103340001400A4081400900813007D0812006B08F4
:103350001300580812004608120034081100230810
:1033600011001208110001081100F0071000E00719
:103370001000D0071000C0071000B0070F00A10711
:10338000100091070E0083070F0074070F006507F8
:103390000E0057070E0049070E003B070D002E07D1
:1033A0000E0020070D0013070D0006070D00F9069B
:1033B0000C00ED060D00E0060C00D4060C00C8065B
:1033C0000C00BC060C00B0060C00A4060B0099060D
:1033D0000C008D060B0082060B0077060B006C06B6
:1033E0000B0061060A0057060B004C060A00420655
:1033F0000A0038060A002E060A0024060A001A06E9
:103400000A001006090007060A00FD050900F40578
:103410000900EB050900E2050900D9050900D005FE
:103420000900C7050900BE050900B5050800AD057E
:103430000800A50509009C050800940508008C05F6
:103440000800840508007C050800740508006C0568
:103450000700650508005D050700560508004E05D4
:10346000070047050700400508003805070031053B
:1034700007002A050700230507001C05060016059E
:1034800007000F0507000805060002050700FB04FA
:103490000600F5040700EE040600E8040600E20456
:1034A0000700DB040600D5040600CF040600C904AB
:1034B0000600C3040600BD040600B7040600B104FC
:1034C0000500AC040600A6040600A00405009B0449
:1034D000060095040500900406008A040500850492
:1034E0000500800406007A040500750405007004D8
:1034F00005006B04050066040500610405005C041A
:10350000050057040500520405004D040500480459
:103510000500430405003E0404003A040500350498
:103520000500300404002C040500270404002304D3
:1035300005001E0404001A0404001604050011040A
:1035400004000D0404000904050004040400000440
:103550000400FC030400F8030400F4030400F00377
:103560000400EC030400E8030400E4030400E003A7
:103570000400DC030400D8030400D4030400D003D7
:103580000400CC030400C8030300C503030024F4B3
:1035900004D9201BC40C5C0E9804C4095F026507A3
:1035A0007101F405F900FB04B30048048700C1036E
:1035B00069005803550003034500BE023A00840227
:1035C000310053022A002902250004022000E401F0
:1035D0001C00C8011900AF011700980114008401F4
:1035E0001300710110006101100051010E00430130
:1035F0000D0036010B002B010B0020010B00150103
:1036000009000C01090003010800FB000800F30099
:103610000800EB000700E4000600DE000600D8000A
:103620000600D2000600CC000500C7000500C2005D
:103630000500BD000400B9000400B5000400B1009D
:103640000400AD000400A9000400A5000300A200CE
:1036500003009F0004009B000300980003009500F6
:10366000020093000300900003008D0002008B0015
:10367000030088000200860002008400030081002D
:1036800002007F0002007D0002007B000200790042
:103690000200770001007600020074000200720050
:1036A0000100710002006F0002006D0001006C005B
:1036B00002006A0001006900020067000100660064
:1036C0000100650001006400020062000100610069
:1036D0000100600001005F0002005D0001005C006D
:1036E00001005B0001005A00010059000100580070
:1036F0000100570001005600010055000100540070
:10370000010053000000530001005200010051006D
:103710000100500001004F0001004E0000004E006B
:1037200001004D0001004C0001004B0000004B0067
:1037300001004A0001004900010048000000480063
:10374000010047000100460000004600010045005E
:103750000000450001004400010043000000430058
:103760000100420000004200010041000000410051
:103770000100400001003F0000003F0001003E004A
:1037800000003E0001003D0000003D0001003C0043
:1037900000003C0000003C0001003B0000003B003A
:1037A00001003A0000003A00010039000000390031
:1037B0000100380000003800000038000100370028
:1037C000000037000100360000003600000036001F
:1037D0000100350000003500000035000100340014
:1037E000000034000000340001003300000033000A
:1037F00000003300010032000000320000003200FF
:1038000001003100000031000000310001003000F3
:10381000000030000000300001002F0000002F00E9
:1038200000002F0000002F0001002E0000002E00DD
:1038300000002E0001002D0000002D0000002D00D2
:1038400000002D0001002C0000002C0000002C00C6
:1038500000002C0001002B0000002B0000002B00BA
:1038600000002B0001002A0000002A0000002A00AE
:1038700000002A00010029000000290000002900A2
:103880000000290000002900010028000000280095
:103890000000280000002800000028000100270088
:1038A000000027000000270000002700000027007C
:1038B000010026000000260000002600000026006F
:1038C0000000260001002500000025000000250062
:1038D0000000250000002500000025000100240054
:1038E0000000240000002400000024000000240048
:1038F000010023000000230000002300000023003B
:10390000000023000000230000002300010022002B
:10391000000022000000220000002200000022001F
:103920000000220001002100000021000000210011
:103930000000210000002100000021000000210003
:1039400001002000000020000000200000002000F6
:1039500000002000000020000000200000002000E7
:1039600001001F0000001F0000001F0000001F00DA
:1039700000001F0000001F0000001F0001001E00CB
:1039800000001E0000001E0000001E000000232C8E
:103990000000B8220000561800003A0F0000B808D6
:1039A0000000B1040000710200003E01000020434D
:1039B0006F756E7420583A004265640045310062AC
:1039C0006564002C2073797374656D2073746F7057
:1039D00070656421204865617465725F49443A20CE
:1039E0000048656174696E67204661696C656400B2
:1039F00048656174696E67206661696C6564004D35
:103A00003131322053687574646F776E001000C9CD
:103A10000210012C014001220170011801B0010EB9
:103A200001F00104015002FA00B002F0003003E698
:103A300000D003DC009004D2007005C800A006BED0
:103A4000000008B400B009AA00D00BA000600E96D8
:103A50000060118C000015820020197800C01D6ED6
:103A600000A0226400B0275A00902C50000031467C
:103A700000E0343C0010383200903A2800603C1ED0
:103A800000A03D1400803E0A00203F00005448453D
:103A9000524D414C2052554E415741590054686592
:103AA000726D616C2052756E61776179004572723A
:103AB0003A204D415854454D50004D415854454DC4
:103AC0005020747269676765726564004572723A66
:103AD000204D494E54454D50004D494E54454D5092
:103AE0002074726967676572656400202F00204248
:103AF000403A0020403A0020573A0020573A004907
:103B00006E76616C69642065787472756465720A9A
:103B1000007C3C3E5E2B3D3F2F5B5D3B2C2A225CB4
:103B20000043616E6E6F74206F70656E20737562F6
:103B30006469722000534420496E697420466169AB
:103B40006C0053442063617264206F6B0A006F70D5
:103B5000656E526F6F74206661696C65640A0076E9
:103B60006F6C756D652E696E6974206661696C6530
:103B7000640A004E6F20534420636172640A000A95
:103B80004D3234004D323320257300363726033C46
:103B90003D380E2E303E121A1C180AFF4309070842
:103BA00044000124F404D9201BC40C5C0E9804C406
:103BB000095F0265077101F405F900FB04B30048D1
:103BC000048700C10369005803550003034500BE84
:103BD000023A008402310053022A0029022500041F
:103BE000022000E4011C00C8011900AF0117009871
:103BF00001140084011300710110006101100051D3
:103C0000010E0043010D0036010B002B010B0020BB
:103C1000010B00150109000C01090003010800FB5C
:103C2000000800F3000800EB000700E4000600DED7
:103C3000000600D8000600D2000600CC000500C730
:103C4000000500C2000500BD000400B9000400B575
:103C5000000400B1000400AD000400A9000400A5A8
:103C6000000300A20003009F0004009B00030098D3
:103C70000003009500020093000300900003008DF4
:103C80000002008B0003008800020086000200840E
:103C9000000300810002007F0002007D0002007B23
:103CA0000002007900020077000100760002007433
:103CB00000020072000100710002006F0002006D3E
:103CC0000001006C0002006A000100690002006748
:103CD000000100660001006500010064000200624E
:103CE00000010061000100600001005F0002005D52
:103CF0000001005C0001005B0001005A0001005956
:103D00000001005800010057000100560001005555
:103D10000001005400010053000000530001005254
:103D200000010051000100500001004F0001004E51
:103D30000000004E0001004D0001004C0001004B4E
:103D40000000004B0001004A00010049000100484A
:103D50000000004800010047000100460000004646
:103D6000000100450000004500010044000100433F
:103D70000000004300010042000000420001004139
:103D800000000041000100400001003F0000003F32
:103D90000001003E0000003E0001003D0000003D2B
:103DA0000001003C0000003C0000003C0001003B22
:103DB0000000003B0001003A0000003A0001003919
:103DC0000000003900010038000000380000003811
:103DD0000001003700000037000100360000003607
:103DE00000000036000100350000003500000035FD
:103DF00000010034000000340000003400010033F2
:103E000000000033000000330001003200000032E7
:103E100000000032000100310000003100000031DC
:103E20000001003000000030000000300001002FD1
:103E30000000002F0000002F0000002F0001002EC6
:103E40000000002E0000002E0001002D0000002DBB
:103E50000000002D0000002D0001002C0000002CAF
:103E60000000002C0000002C0001002B0000002BA3
:103E70000000002B0000002B0001002A0000002A97
:103E80000000002A0000002A00010029000000298B
:103E9000000000290000002900000029000100287E
:103EA0000000002800000028000000280000002872
:103EB0000001002700000027000000270000002765
:103EC0000000002700010026000000260000002658
:103ED000000000260000002600010025000000254B
:103EE000000000250000002500000025000000253E
:103EF0000001002400000024000000240000002431
:103F00000000002400010023000000230000002323
:103F10000000002300000023000000230000002315
:103F20000001002200000022000000220000002208
:103F300000000022000000220001002100000021FA
:103F400000000021000000210000002100000021ED
:103F500000000021000100200000002000000020DF
:103F600000000020000000200000002000000020D1
:103F7000000000200001001F0000001F0000001FC3
:103F80000000001F0000001F0000001F0000001FB5
:103F90000001001E0000001E0000001E0000001EA8
:103FA00000000024F4D43050C38E20C2A2401782F7
:103FB0008B7011127A910D816CD90AA861E108C742
:103FC000586607615143061E4B5D05C145A7041A9B
:103FD000411104093D9803713931034036DB026514
:103FE000339102D4305402802E1D02632CEE0175F1
:103FF0002AC501B028A001102781018F2564012B5B
:10400000244B01E0223401AC211F018D200D0180E1
:104010001FFC00841EED00971DDF00B81CD200E6D7
:104020001BC600201BBC00641AB200B219A8000A0B
:1040300019A0006A189900D117910040178B00B59C
:1040400016840031167E00B31579003A157300C747
:10405000146F0058146A00EE13660088136300257D
:10406000135E00C7125B006C12570015125400C19A
:1040700011510070114F0021114B00D61049008DD5
:104080001047004610440002104200C00F4000805C
:104090000F3E00420F3C00060F3B00CB0E38009352
:1040A0000E37005C0E3500270E3400F30D3200C1D0
:1040B0000D3100900D3000600D2E00320D2D0005E9
:1040C0000D2C00D90C2B00AE0C2900850C29005CAE
:1040D0000C2700350C27000E0C2600E80B2400C42A
:1040E0000B2400A00B23007D0B23005A0B21003969
:1040F0000B2100180B2000F80A1F00D90A1E00BB74
:104100000A1E009D0A1D00800A1D00630A1C00474C
:104110000A1B002C0A1B00110A1A00F7091A00DDFD
:10412000091900C4091900AB091900920917007B8D
:10413000091800630917004C0916003609160020FB
:104140000916000A091500F5081500E0081400CC4E
:10415000081400B8081400A4081400900813007D87
:104160000812006B081300580812004608120034A9
:10417000081100230811001208110001081100F0B5
:10418000071000E0071000D0071000C0071000B0B3
:10419000070F00A107100091070E0083070F00749E
:1041A000070F0065070E0057070E0049070E003B7A
:1041B000070D002E070E0020070D0013070D000647
:1041C000070D00F9060C00ED060D00E0060C00D40A
:1041D000060C00C8060C00BC060C00B0060C00A4BF
:1041E000060B0099060C008D060B0082060B00776B
:1041F000060B006C060B0061060A0057060B004C0C
:10420000060A0042060A0038060A002E060A0024A2
:10421000060A001A060A001006090007060A00FD31
:10422000050900F4050900EB050900E2050900D9BC
:10423000050900D0050900C7050900BE050900B53C
:10424000050800AD050800A50509009C05080094B7
:104250000508008C050800840508007C050800742A
:104260000508006C050700650508005D0507005698
:104270000508004E050700470507004005080038FF
:10428000050700310507002A050700230507001C64
:10429000050600160507000F0507000805060002C1
:1042A000050700FB040600F5040700EE040600E81D
:1042B000040600E2040700DB040600D5040600CF74
:1042C000040600C9040600C3040600BD040600B7C6
:1042D000040600B1040500AC040600A6040600A014
:1042E0000405009B04060095040500900406008A5E
:1042F00004050085040500800406007A04050075A5
:10430000040500700405006B0405006604050061E7
:104310000405005C04050057040500520405004D27
:1043200004050048040500430405003E0404003A67
:1043300004050035040500300404002C04050027A2
:10434000040400230405001E0404001A04040016DB
:10435000040500110404000D040400090405000410
:1043600004040000040400FC030400F8030400F447
:10437000030400F0030400EC030400E8030400E479
:10438000030400E0030400DC030400D8030400D4A9
:10439000030400D0030400CC030400C8030300C5D9
:1043A000030300726F746174696F6E206D617472C3
:1043B00069783A0A0024F404D9201BC40C5C0E98D6
:1043C00004C4095F0265077101F405F900FB04B339
:1043D0000048048700C103690058035500030345E2
:1043E00000BE023A008402310053022A002902254D
:1043F0000004022000E4011C00C8011900AF0117ED
:104400000098011400840113007101100061011073
:104410000051010E0043010D0036010B002B010B72
:104420000020010B00150109000C0109000301081F
:1044300000FB000800F3000800EB000700E40006A2
:1044400000DE000600D8000600D2000600CC000501
:1044500000C7000500C2000500BD000400B900044B
:1044600000B5000400B1000400AD000400A9000480
:1044700000A5000300A20003009F0004009B0003AE
:1044800000980003009500020093000300900003D1
:10449000008D0002008B00030088000200860002ED
:1044A0000084000300810002007F0002007D000202
:1044B000007B000200790002007700010076000214
:1044C000007400020072000100710002006F00021F
:1044D000006D0001006C0002006A0001006900022A
:1044E0000067000100660001006500010064000231
:1044F000006200010061000100600001005F000235
:10450000005D0001005C0001005B0001005A000139
:104510000059000100580001005700010056000139
:104520000055000100540001005300000053000139
:10453000005200010051000100500001004F000135
:10454000004E0000004E0001004D0001004C000133
:10455000004B0000004B0001004A0001004900012F
:10456000004800000048000100470001004600002C
:104570000046000100450000004500010044000124
:10458000004300000043000100420000004200011F
:10459000004100000041000100400001003F000018
:1045A000003F0001003E0000003E0001003D000011
:1045B000003D0001003C0000003C0000003C000108
:1045C000003B0000003B0001003A0000003A0001FF
:1045D00000390000003900010038000000380000F8
:1045E00000380001003700000037000100360000ED
:1045F00000360000003600010035000000350000E4
:1046000000350001003400000034000000340001D7
:1046100000330000003300000033000100320000CE
:1046200000320000003200010031000000310000C3
:1046300000310001003000000030000000300001B7
:10464000002F0000002F0000002F0000002F0001AD
:10465000002E0000002E0000002E0001002D0000A2
:10466000002D0000002D0000002D0001002C000096
:10467000002C0000002C0000002C0001002B00008A
:10468000002B0000002B0000002B0001002A00007E
:10469000002A0000002A0000002A00010029000072
:1046A0000029000000290000002900000029000165
:1046B000002800000028000000280000002800005A
:1046C000002800010027000000270000002700004C
:1046D000002700000027000100260000002600003F
:1046E0000026000000260000002600010025000032
:1046F0000025000000250000002500000025000026
:104700000025000100240000002400000024000017
:10471000002400000024000100230000002300000A
:1047200000230000002300000023000000230000FD
:1047300000230001002200000022000000220000EF
:1047400000220000002200000022000100210000E1
:1047500000210000002100000021000000210000D5
:1047600000210000002100010020000000200000C6
:1047700000200000002000000020000000200000B9
:104780000020000000200001001F0000001F0000AA
:10479000001F0000001F0000001F0000001F00009D
:1047A000001F0001001E0000001E0000001E00008F
:1047B000001E00000024F4D43050C38E20C2A2405A
:1047C00017828B7011127A910D816CD90AA861E160
:1047D00008C7586607615143061E4B5D05C145A7D2
:1047E000041A411104093D9803713931034036DB45
:1047F0000265339102D4305402802E1D02632CEEE8
:1048000001752AC501B028A001102781018F2564F8
:10481000012B244B01E0223401AC211F018D200D1E
:1048200001801FFC00841EED00971DDF00B81CD224
:1048300000E61BC600201BBC00641AB200B219A817
:10484000000A19A0006A189900D117910040178B2F
:1048500000B516840031167E00B31579003A157341
:1048600000C7146F0058146A00EE136600881363C3
:104870000025135E00C7125B006C1257001512541E
:1048800000C111510070114F0021114B00D6104989
:10489000008D1047004610440002104200C00F4037
:1048A00000800F3E00420F3C00060F3B00CB0E384D
:1048B00000930E37005C0E3500270E3400F30D32E6
:1048C00000C10D3100900D3000600D2E00320D2D15
:1048D00000050D2C00D90C2B00AE0C2900850C29ED
:1048E000005C0C2700350C27000E0C2600E80B247A
:1048F00000C40B2400A00B23007D0B23005A0B21C6
:1049000000390B2100180B2000F80A1F00D90A1EDD
:1049100000BB0A1E009D0A1D00800A1D00630A1CC0
:1049200000470A1B002C0A1B00110A1A00F7091A7B
:1049300000DD091900C4091900AB09190092091713
:10494000007B091800630917004C09160036091688
:1049500000200916000A091500F5081500E00814E2
:1049600000CC081400B8081400A408140090081320
:10497000007D0812006B0813005808120046081248
:104980000034081100230811001208110001081159
:1049900000F0071000E0071000D0071000C007105B
:1049A00000B0070F00A107100091070E0083070F4A
:1049B0000074070F0065070E0057070E0049070E29
:1049C000003B070D002E070E0020070D0013070DFA
:1049D0000006070D00F9060C00ED060D00E0060CC0
:1049E00000D4060C00C8060C00BC060C00B0060C77
:1049F00000A4060B0099060C008D060B0082060B26
:104A00000077060B006C060B0061060A0057060BC8
:104A1000004C060A0042060A0038060A002E060A62
:104A20000024060A001A060A001006090007060AF2
:104A300000FD050900F4050900EB050900E2050980
:104A400000D9050900D0050900C7050900BE050900
:104A500000B5050800AD050800A50509009C05087E
:104A600000940508008C050800840508007C0508F2
:104A700000740508006C050700650508005D050762
:104A800000560508004E05070047050700400508C9
:104A90000038050700310507002A05070023050730
:104AA000001C050600160507000F0507000805068F
:104AB0000002050700FB040600F5040700EE0406EB
:104AC00000E8040600E2040700DB040600D5040643
:104AD00000CF040600C9040600C3040600BD040696
:104AE00000B7040600B1040500AC040600A60406E5
:104AF00000A00405009B0406009504050090040630
:104B0000008A04050085040500800406007A040577
:104B10000075040500700405006B040500660405BB
:104B200000610405005C04050057040500520405FB
:104B3000004D04050048040500430405003E04043C
:104B4000003A04050035040500300404002C040577
:104B50000027040400230405001E0404001A0404B2
:104B60000016040500110404000D040400090405E6
:104B7000000404040000040400FC030400F803041F
:104B800000F4030400F0030400EC030400E8030451
:104B900000E4030400E0030400DC030400D8030481
:104BA00000D4030400D0030400CC030400C80303B2
:104BB00000C503030024F404D9201BC40C5C0E9828
:104BC00004C4095F0265077101F405F900FB04B331
:104BD0000048048700C103690058035500030345DA
:104BE00000BE023A008402310053022A0029022545
:104BF0000004022000E4011C00C8011900AF0117E5
:104C0000009801140084011300710110006101106B
:104C10000051010E0043010D0036010B002B010B6A
:104C20000020010B00150109000C01090003010817
:104C300000FB000800F3000800EB000700E400069A
:104C400000DE000600D8000600D2000600CC0005F9
:104C500000C7000500C2000500BD000400B9000443
:104C600000B5000400B1000400AD000400A9000478
:104C700000A5000300A20003009F0004009B0003A6
:104C800000980003009500020093000300900003C9
:104C9000008D0002008B00030088000200860002E5
:104CA0000084000300810002007F0002007D0002FA
:104CB000007B00020079000200770001007600020C
:104CC000007400020072000100710002006F000217
:104CD000006D0001006C0002006A00010069000222
:104CE0000067000100660001006500010064000229
:104CF000006200010061000100600001005F00022D
:104D0000005D0001005C0001005B0001005A000131
:104D10000059000100580001005700010056000131
:104D20000055000100540001005300000053000131
:104D3000005200010051000100500001004F00012D
:104D4000004E0000004E0001004D0001004C00012B
:104D5000004B0000004B0001004A00010049000127
:104D60000048000000480001004700010046000024
:104D7000004600010045000000450001004400011C
:104D80000043000000430001004200000042000117
:104D9000004100000041000100400001003F000010
:104DA000003F0001003E0000003E0001003D000009
:104DB000003D0001003C0000003C0000003C000100
:104DC000003B0000003B0001003A0000003A0001F7
:104DD00000390000003900010038000000380000F0
:104DE00000380001003700000037000100360000E5
:104DF00000360000003600010035000000350000DC
:104E000000350001003400000034000000340001CF
:104E100000330000003300000033000100320000C6
:104E200000320000003200010031000000310000BB
:104E300000310001003000000030000000300001AF
:104E4000002F0000002F0000002F0000002F0001A5
:104E5000002E0000002E0000002E0001002D00009A
:104E6000002D0000002D0000002D0001002C00008E
:104E7000002C0000002C0000002C0001002B000082
:104E8000002B0000002B0000002B0001002A000076
:104E9000002A0000002A0000002A0001002900006A
:104EA000002900000029000000290000002900015D
:104EB0000028000000280000002800000028000052
:104EC0000028000100270000002700000027000044
:104ED0000027000000270001002600000026000037
:104EE000002600000026000000260001002500002A
:104EF000002500000025000000250000002500001E
:104F0000002500010024000000240000002400000F
:104F10000024000000240001002300000023000002
:104F200000230000002300000023000000230000F5
:104F300000230001002200000022000000220000E7
:104F400000220000002200000022000100210000D9
:104F500000210000002100000021000000210000CD
:104F600000210000002100010020000000200000BE
:104F700000200000002000000020000000200000B1
:104F80000020000000200001001F0000001F0000A2
:104F9000001F0000001F0000001F0000001F000095
:104FA000001F0001001E0000001E0000001E000087
:104FB000001E00000024F4D43050C38E20C2A24052
:104FC00017828B7011127A910D816CD90AA861E158
:104FD00008C7586607615143061E4B5D05C145A7CA
:104FE000041A411104093D9803713931034036DB3D
:104FF0000265339102D4305402802E1D02632CEEE0
:1050000001752AC501B028A001102781018F2564F0
:10501000012B244B01E0223401AC211F018D200D16
:1050200001801FFC00841EED00971DDF00B81CD21C
:1050300000E61BC600201BBC00641AB200B219A80F
:10504000000A19A0006A189900D117910040178B27
:1050500000B516840031167E00B31579003A157339
:1050600000C7146F0058146A00EE136600881363BB
:105070000025135E00C7125B006C12570015125416
:1050800000C111510070114F0021114B00D6104981
:10509000008D1047004610440002104200C00F402F
:1050A00000800F3E00420F3C00060F3B00CB0E3845
:1050B00000930E37005C0E3500270E3400F30D32DE
:1050C00000C10D3100900D3000600D2E00320D2D0D
:1050D00000050D2C00D90C2B00AE0C2900850C29E5
:1050E000005C0C2700350C27000E0C2600E80B2472
:1050F00000C40B2400A00B23007D0B23005A0B21BE
:1051000000390B2100180B2000F80A1F00D90A1ED5
:1051100000BB0A1E009D0A1D00800A1D00630A1CB8
:1051200000470A1B002C0A1B00110A1A00F7091A73
:1051300000DD091900C4091900AB0919009209170B
:10514000007B091800630917004C09160036091680
:1051500000200916000A091500F5081500E00814DA
:1051600000CC081400B8081400A408140090081318
:10517000007D0812006B0813005808120046081240
:105180000034081100230811001208110001081151
:1051900000F0071000E0071000D0071000C0071053
:1051A00000B0070F00A107100091070E0083070F42
:1051B0000074070F0065070E0057070E0049070E21
:1051C000003B070D002E070E0020070D0013070DF2
:1051D0000006070D00F9060C00ED060D00E0060CB8
:1051E00000D4060C00C8060C00BC060C00B0060C6F
:1051F00000A4060B0099060C008D060B0082060B1E
:105200000077060B006C060B0061060A0057060BC0
:10521000004C060A0042060A0038060A002E060A5A
:105220000024060A001A060A001006090007060AEA
:1052300000FD050900F4050900EB050900E2050978
:1052400000D9050900D0050900C7050900BE0509F8
:1052500000B5050800AD050800A50509009C050876
:1052600000940508008C050800840508007C0508EA
:1052700000740508006C050700650508005D05075A
:1052800000560508004E05070047050700400508C1
:105290000038050700310507002A05070023050728
:1052A000001C050600160507000F05070008050687
:1052B0000002050700FB040600F5040700EE0406E3
:1052C00000E8040600E2040700DB040600D504063B
:1052D00000CF040600C9040600C3040600BD04068E
:1052E00000B7040600B1040500AC040600A60406DD
:1052F00000A00405009B0406009504050090040628
:10530000008A04050085040500800406007A04056F
:105310000075040500700405006B040500660405B3
:1053200000610405005C04050057040500520405F3
:10533000004D04050048040500430405003E040434
:10534000003A04050035040500300404002C04056F
:105350000027040400230405001E0404001A0404AA
:105360000016040500110404000D040400090405DE
:10537000000404040000040400FC030400F8030417
:1053800000F4030400F0030400EC030400E8030449
:1053900000E4030400E0030400DC030400D8030479
:1053A00000D4030400D0030400CC030400C80303AA
:1053B00000C503030070012C0190012701B00122F8
:1053C00001C0011D01F00118011002130130020E8D
:1053D000016002090190020401C002FF000003FA0B
:1053E000004003F5008003F000D003EB002004E64A
:1053F000007004E100E004DC004005D700C005D2E5
:10540000004006CD00D006C8008007C3003008BEAB
:1054100000F008B900C009B400B00AAF00B00BAA90
:1054200000D00CA500000EA000500F9B00C01096ED
:10543000005012910000148C00C0158700B0178234
:1054400000B0197D00D01B7800001E730040206E54
:105450000090226900F024640040275F0090295AE0
:1054600000E02B5500102E500020304B001032462B
:1054700000E033410090353C00103737007038327F
:1054800000A0392D00B03A2800A03B2300603C1E4C
:1054900000103D1900903D1400103E0F00703E0AB0
:1054A00000C03E0500003F0000403FFBFF803FF68C
:1054B000FFC03FF1FF1000C90210012C0140012282
:1054C0000170011801B0010E01F00104015002FA4F
:1054D00000B002F0003003E600D003DC009004D2FC
:1054E000007005C800A006BE000008B400B009AAFC
:1054F00000D00BA000600E960060118C0000158299
:105500000020197800C01D6E00A0226400B0275A48
:1055100000902C500000314600E0343C001038323E
:1055200000903A2800603C1E00A03D1400803E0A16
:1055300000203F00005A5F6D6F76655F636F6D708E
:105540000A00473238580047323859004732385A33
:10555000004732384F0A4D343820503130004D3832
:1055600034004732395034523939395400473239CE
:10557000503454004732380A4732364350493000DD
:105580004732380A47323643504931004732394AA8
:1055900030004732395033543000473239503242AC
:1055A0005430004732380A4D31393049300A4D31D4
:1055B000303949300A47323950310A4D313034538D
:1055C000300A4D3134305330004732380A4D3139CA
:1055D0003049310A4D31303949310A473239503179
:1055E0000A4D31303453300A4D3134305330004796
:1055F00032394E5031004732395031430047323949
:10560000490047323954300047323954310047326B
:1056100039532D3100473239493939390A4732393E
:105620005032425430004732394E503100473239FF
:1056300050335430004732395034523939395400DC
:1056400047323950345239393954004732394400DD
:105650004732394100473239570041786973200099
:10566000206D696E3A00206D61783A004163636590
:105670006C65726174696F6E206C696D69746564C4
:105680002E0A004641535400534C4F57000E000061
:105690000F01000D000F01000F0E0000000F000DA4
:1056A000004572726F722077726974696E67207438
:1056B0006F20454550524F4D210A0053544F5050D2
:1056C00045442E20005072696E7465722073746FA9
:1056D000707065642064756520746F206572726FE8
:1056E00072732E2046697820746865206572726F27
:1056F0007220616E6420757365204D3939392074CC
:105700006F20726573746172742E202854656D70F9
:105710006572617475726520697320726573657452
:105720002E2053657420697420616674657220723E
:10573000657374617274696E67290A004E6F204345
:105740006865636B73756D2077697468206C696E2A
:1057500065206E756D6265722C204C617374204CEF
:10576000696E653A20004E6F20436865636B737500
:105770006D2077697468206C696E65206E756D6246
:1057800065722C204C617374204C696E653A200060
:10579000636865636B73756D206D69736D617463A8
:1057A000682C204C617374204C696E653A20004C63
:1057B000696E65204E756D626572206973206E6F2B
:1057C00074204C617374204C696E65204E756D6257
:1057D00065722B312C204C617374204C696E653AD4
:1057E00020004D3131300053657269616C20737453
:1057F00061747573206D69736D617463680A0077F5
:105800006169740A00534420726561642065727294
:105810006F720A00486F74656E642049646C65207D
:1058200054696D656F757400486F74656E642049C6
:10583000646C652054696D656F75740A00212120C0
:105840004B494C4C20636175736564206279204B31
:10585000494C4C20627574746F6E2F70696E0A002B
:105860002121204B494C4C20636175736564206293
:105870007920746F6F206D75636820696E61637441
:105880006976652074696D65202D20637572726577
:105890006E7420636F6D6D616E643A200070617587
:1058A0007365004D363030002066696C616D656E41
:1058B000745F72756E6F7574200066696C616D65DA
:1058C0006E745F72756E6F757420540046696C61FA
:1058D0006D656E7452756E6F75742054004D6564FD
:1058E00069612052656D6F766564004D656469611C
:1058F00020496E736572746564004D3130303053E9
:1059000000627573793A2070617573656420666F03
:105910007220696E7075740A00627573793A20702E
:10592000617573656420666F7220757365720A0015
:10593000627573793A2070726F63657373696E670D
:105940000A00506C65617365205265736574005080
:1059500052494E5445522048414C54454400255329
:105960003A20255300706F7765726F6666004B4969
:105970004C4C45442E20005072696E74657220684C
:10598000616C7465642E206B696C6C2829206361DE
:105990006C6C6564210A0053544F505045442E20CE
:1059A000005072696E7465722073746F70706564F4
:1059B0002064756520746F206572726F72732E207B
:1059C00046697820746865206572726F7220616E16
:1059D0006420757365204D39393920746F207265E4
:1059E00073746172742E202854656D7065726174D1
:1059F0007572652069732072657365742E20536516
:105A000074206974206166746572207265737461B4
:105A10007274696E67290A006563686F3A0045729F
:105A2000726F723A00204A0020204D3432312049F2
:105A300000202047323920493939390A006163741E
:105A40006976650A00696E00002053797374656D8C
:105A50002076312E303120002020207C0A004E415B
:105A60004E0020202E20202000207C004C43443A71
:105A70000A004353563A0A0020666F7220003A0A21
:105A80000A000A42656420546F706F677261706823
:105A900079205265706F72740050726F62696E6720
:105AA000204661696C65640A0050726F62696E67B6
:105AB000204661696C656400205A3A200020593AFA
:105AC000200042656420583A20004732384C3000AC
:105AD000446F6E652E0A003F496E76616C696420E2
:105AE00073746F7261676520736C6F742E0A3F5513
:105AF0007365203020746F20003F454550524F4D54
:105B00002073746F72616765206E6F7420617661B7
:105B1000696C61626C652E0A00446F6E652E0A0026
:105B20003F496E76616C69642073746F726167655A
:105B300020736C6F742E0A3F557365203020746F8C
:105B400020003F454550524F4D2073746F7261677E
:105B500065206E6F7420617661696C61626C652E80
:105B60000A004732392050322066696E69736865D1
:105B7000642E0A005859206F75747369646520702B
:105B800072696E7461626C65207261646975732EEE
:105B90000A003F4572726F7220696E204275736908
:105BA0006E6573732043617264206D6561737572F5
:105BB000656D656E742E0A004D616E75616C6C7951
:105BC0002070726F62696E6720756E7265616368BE
:105BD00061626C6520706F696E74732E0A00292EE5
:105BE0000A0A0050726F62696E672061726F756E8B
:105BF000642028004D65736820696E76616C696465
:105C0000617465642E2050726F62696E67206D65E5
:105C100073682E0A004D657368207A65726F65643B
:105C20002E0A0044656661756C742073746F72612E
:105C3000676520736C6F7420302073656C656374C6
:105C400065642E0A004C6F6164696E672074657329
:105C5000745F7061747465726E2076616C756573C3
:105C60002E0A0A00496E76616C696420746573744B
:105C70005F7061747465726E2076616C75652E203C
:105C8000282D3120746F2032290A0A0020696E768F
:105C9000616C6964617465642E0A0A004C6F63610B
:105CA00074696F6E7300456E74697265204D65731B
:105CB00068005374616E6461726420446576696142
:105CC00074696F6E3A20004D65616E204D65736892
:105CD000204865696768743A200023206F66207346
:105CE000616D706C65733A20000A4D657368206FB2
:105CF0006E6C79207061727469616C6C7920706F60
:105D000070756C617465642E0A0A0050726F626966
:105D10006E6720506F696E740025532025692F250A
:105D200069002E0A002F0050726F62696E67206D45
:105D300065736820706F696E74200020616E642046
:105D400074616B652061206D6561737572656D6549
:105D50006E742E0A006D6D20746869636B2E0A00E4
:105D6000427573696E657373204361726420697351
:105D7000200052656D6F76652026204D6561737534
:105D80007265204265640052656D6F7665207368A8
:105D9000696D00506C616365207368696D20756E74
:105DA000646572206E6F7A7A6C65000A4D6573685F
:105DB000206F6E6C79207061727469616C6C7920EF
:105DC000706F70756C617465642E0A004D65736840
:105DD00020506F696E74204D656173757265642023
:105DE00061743A20004D65617375726500506C6195
:105DF0006365205368696D2026204D656173757257
:105E000065004D6F76696E6720746F206E657874DB
:105E1000004D6573682045646974696E672053742A
:105E20006F7070656400446F6E65204564697469C5
:105E30006E67204D6573680A00446F6E6520456487
:105E40006974696E67204D6573680046696E6520E8
:105E500054756E696E67204D6573680028582C591B
:105E600029206F757473696465207072696E74613E
:105E7000626C65207261646975732E0A004F6666F4
:105E8000736574206F7574206F6620626F756E6421
:105E9000732E20283020746F2031306D6D290A0A4E
:105EA00000496E76616C6964206D61702074797050
:105EB000652E0A0A003F28462961646520686569E5
:105EC00067687420666F7220426564204C65766551
:105ED0006C20436F7272656374696F6E206E6F74AD
:105EE00020706C61757369626C652E0A0A003F430D
:105EF000616E277420616374697661746520616ED8
:105F000064206465616374697661746520617420DE
:105F10007468652073616D652074696D652E0A0A69
:105F200000426F7468205820262059206C6F6361EE
:105F300074696F6E73206D75737420626520737061
:105F4000656369666965642E0A0A003F496E766179
:105F50006C696420677269642073697A6520284AD5
:105F600029207370656369666965642028322D395C
:105F7000292E0A0A003F285029686173652076613E
:105F80006C756520696E76616C69642028302D36E9
:105F9000292E0A0A003F2856296572626F73652010
:105FA0006C6576656C20696D706C61757369626C87
:105FB000652028302D34292E0A0A003F28522965F1
:105FC0007065746974696F6E20636F756E74206993
:105FD0006E76616C69642028312B292E0A0A0044F0
:105FE0006F696E6720473239009C56975692568DDE
:105FF000565D0A0062656420706C616E65206E6F8C
:10600000726D616C203D205B00436F756C64206E87
:106010006F7420636F6D706C657465204C534621FE
:1060200000436F727265637465645F5A3D00255367
:106030002025692F2569000A0A002F0054696C7415
:10604000696E67206D65736820706F696E742000DB
:106050003F4572726F722070726F62696E67207056
:106060006F696E742E2041626F7274696E67206F63
:106070007065726174696F6E2E0A00436F7272658B
:10608000637465645F5A3D00255320332F330054F9
:10609000696C74696E67206D6573682028332F33CF
:1060A000290A00436F727265637465645F5A3D002C
:1060B000255320322F330054696C74696E67206D4C
:1060C0006573682028322F33290A00436F72726586
:1060D000637465645F5A3D0054696C74696E67202F
:1060E000506F696E7400255320312F330054696C52
:1060F00074696E67206D6573682028312F33290A13
:1061000000646F6E650A00496E737566666963693F
:10611000656E7420646174610A000000803F254947
:10612000124225499042B86DD74225490F436EDB94
:106130003243B86D564301007A4325C98E434A92D3
:10614000A0436E5BB2439324C443B8EDD543DCB6A1
:10615000E7430180F9430000803F25491242254969
:106160009042B86DD74225490F436EDB3243B86D7C
:10617000564301007A4325C98E434A92A0436E5B81
:10618000B2439324C443B8EDD543DCB6E743018062
:10619000F9434578747261706F6C6174696E672041
:1061A0006D6573682E2E2E0021212053544F5020F0
:1061B00063616C6C65642062656361757365206FF3
:1061C0006620424C546F756368206572726F72204E
:1061D0002D20726573746172742077697468204D24
:1061E0003939390A0021212053544F502063616C02
:1061F0006C65642062656361757365206F6620421B
:106200004C546F756368206572726F72202D207216
:106210006573746172742077697468204D393939F7
:106220000A005072696E74696E67204F626A656316
:1062300074002553202569002F2F616374696F6EE8
:106240003A0073746172740070726F6D70745F00E5
:10625000656E6400486F74656E6420746F6F2063B0
:106260006F6C640A0053656E64204D3130382074C1
:106270006F20726573756D650A00496E736572747F
:106280002066696C616D656E7420616E6420736553
:106290006E64204D3130380A0052656865617420A3
:1062A000446F6E6500526568656174696E672E2E75
:1062B0002E005265686561740048656174657220DE
:1062C00054696D656F75740053656E64204D31308F
:1062D0003820746F2068656174206E6F7A7A6C65FF
:1062E0000A004E6F7A7A6C65205061726B656400AB
:1062F00070617573656400506175736500726573D4
:10630000756D656400526573756D696E670047321F
:10631000362043616E63656C656400473236204801
:10632000656174696E67204E6F7A7A6C65004732DA
:10633000362048656174696E672042656400576164
:106340006974696E6720666F722068656174757024
:106350002E0A004669786564204C656E6774682073
:106360005072696D6500446F6E65205072696D6989
:106370006E67004D616E75616C207072696D696E3B
:10638000672E2E2E004C656176696E672047323687
:10639000003F53706563696669656420582C592015
:1063A000636F6F7264696E617465206F7574206FBE
:1063B0006620626F756E64732E0A003F285229654D
:1063C000706561742076616C7565206E6F742070E5
:1063D0006C61757369626C653B206D7573742062C6
:1063E00065206174206C6561737420312E0A003F52
:1063F000537065636966696564206E6F7A7A6C654F
:106400002074656D7065726174757265206E6F744D
:1064100020706C61757369626C652E0A003F537061
:10642000656369666965642066696C616D656E7433
:106430002073697A65206E6F7420706C6175736962
:10644000626C652E0A003F53706563696669656416
:10645000207072696D65206C656E677468206E6F60
:106460007420706C61757369626C652E0A003F530D
:106470007065636966696564206E6F7A7A6C652001
:1064800073697A65206E6F7420706C6175736962D0
:106490006C652E0A003F52657472616374696F6E99
:1064A000204D756C7469706C696572206D757374BC
:1064B000206265207370656369666965642E0A00F1
:1064C0003F537065636966696564205265747261E3
:1064D0006374696F6E204D756C7469706C69657258
:1064E000206E6F7420706C61757369626C652E0A22
:1064F000003F537065636966696564206C61796506
:106500007220686569676874206E6F7420706C61B2
:10651000757369626C652E0A0043292E0A003F5389
:106520007065636966696564206265642074656D81
:106530007065726174757265206E6F7420706C6125
:10654000757369626C65202834302D00473236201F
:106550007374617274696E672E2E2E0A0041425365
:1065600000504C41002E0A006F70656E2066616914
:106570006C65642C2046696C653A200046696C6540
:106580002073656C65637465640A002053697A65DD
:106590003A200046696C65206F70656E65643A202C
:1065A00000454E4420535542524F5554494E450ADA
:1065B000002220706F73002220706172656E743A41
:1065C0002200535542524F5554494E452043414CA9
:1065D0004C207461726765743A220053756263617E
:1065E0006C6C204F766572666C6F770045786365DA
:1065F00065646564206D617820535542524F55544F
:10660000494E452064657074683A002E0A0044655E
:106610006C6574696F6E206661696C65642C2046D8
:10662000696C653A200046696C652064656C657428
:1066300065643A005344207072696E74696E672015
:106640006279746520004E6F742053442070726923
:106650006E74696E670A002F6175746F25632E670B
:106660000057726974696E6720746F2066696C6583
:106670003A2000667265736800646F696E67002077
:1066800066696C653A20004E6F77200002FD555513
:106690005555555FFFFFFFFFFFFFFFFFFFFE0000A7
:1066A0000000003FFFFFFFFFFFFFFFFFFFFD0000B7
:1066B00007FFFFFFFFFFFFFFFFFFFFFFFFFE07C01A
:1066C0000555555555555FFFFFFFFFFFFFFC0A209D
:1066D0000600000000003FFFFFFFFFFFFFFE141059
:1066E00005000007FFFFFFFFFFFFFFFFFFFC28087B
:1066F0000607C00555555555555FFFFFFFFE54046D
:10670000040A200600000000003FFFFFFFFC6004B9
:1067100006141005000007FFFFFFFFFFFFFE5004F7
:106720000428080607C00555555555555FFC6004FB
:10673000065404040A200600000000003FFE540432
:106740001C60040614100500000000001FFC28084F
:106750002E50040428080607C00001F03FFE141064
:10676000546004065404040A200002081FFC0A2096
:106770006654041C60040614100005043FFE07C0A4
:106780005428082E5004042808000A021FFC0000A8
:106790002E14105460040654040015013FFE00003E
:1067A0001C0A206654041C60040018011FFC000031
:1067B0000607C05428082E50040014013FFE0000B4
:1067C0000400002E14105460040018011FFCFFFF89
:1067D000FE00001C0A206654041C15013FFED5551E
:1067E0005400000607C05428082A0A021FFC84101F
:1067F0004600000400002E14105105043FFEC41092
:1068000044FFFFFE00001C0A206102881FFC841068
:1068100046D5555400000607C05101F03FFE8410D4
:106820004484104600000400002A00001FFCC4102D
:1068300046C41044FFFFFE00001C00003FFE841011
:1068400044841046D5555400000000001FFCD55567
:106850005684104484104600000000003FFCFFFFF7
:10686000FCC41046C41044FFFFFFFFFF9FFE000062
:1068700006841044841046D555555555BFFD5555D1
:1068800054D5555684104484104104109FFFFFFFD7
:10689000FCFFFFFCC41046C410410411BFFFFFFF02
:1068A000FE00000684104484104104109FFFFFFF87
:1068B000FD555554D5555684104104109FFFFFFFD8
:1068C000FFFFFFFCFFFFFCC410410411BFFFFFFFEF
:1068D000FFFFFFFE00000684104104109FFFFFFF32
:1068E000FFFFFFFD555554D555555555BFFFFFFFCB
:1068F000FFFFFFFFFFFFFCFFFFFFFFFF9FFFFFFF0B
:10690000FFFFFFFFFFFFFE00000000003FFFFFFF53
:10691000FFFFFFFFFFFFFD55555555555FFFFFFF7B
:10692000FFFFFFFFFFFFFFFFFFFFFFFFFFFFFFFF77
:10693000FFFFFFFFFFFFFFFFFFFFFFFFFFFFFFFF67
:10694000FFFFFFFFFFFFFFFFFFFFFFFFFFFFFFFF57
:10695000FFFFFFFFFFFFFFFFFFFFFFFFFFE02EFB3B
:106960007DFBFBCFC1DFBB3EC0E1FE3C1FFDEE7BEC
:1069700039F9F3CF9EDFBB3EDFDEFCDDE7FDEE3B0A
:10698000BBF9EBD7BF5FBB5EDFDEFDEDF7FDEEBB16
:10699000D3FAEBB73FDFBB4EDFDFFFCDF3FDEEDB1E
:1069A000C7FAEBBB7FC03B6EC0E3FF1DF3FDEECB30
:1069B000EFFADBBB7FDFBB66DFF8FFCDF3FDEEEB6D
:1069C000EFFB5B033F5FBB76DFFE7FEDF3FDEEF396
:1069D000EFFB5B79BEDFBB7ADFDE7DEDF7FDEEF32B
:1069E000EFFBBAFD9EDFBB7CDFDEFDCDE7FDEEFBFE
:1069F000EFFBBAFDC1DFBB7EC0E0FE1C1F6D617204
:106A00006C696E66772E6F726700322E302E375F9C
:106A10004457372E33001FFFFFFFFFFFFF600000CA
:106A2000000001FF400000000000FF8000000000A7
:106A3000007F83CF00000C303F87FF80000C301FA9
:106A4000867980000C000F8C30C7838C30E78C3047
:106A5000CFC7CC31F38C30DCECEC33B98C30D86C54
:106A60006C33198C30D06C0C33198C30D86C0C33DF
:106A7000198C30DC6C0E3B198C30CF7C079F198C45
:106A800030C77C038F194000000000000260000046
:106A9000000000061FFFFFFFFFFFF870012C0190B0
:106AA000012701B0012201C0011D01F001180110F0
:106AB00002130130020E016002090190020401C0BC
:106AC00002FF000003FA004003F5008003F000D04D
:106AD00003EB002004E6007004E100E004DC004069
:106AE00005D700C005D2004006CD00D006C8008002
:106AF00007C3003008BE00F008B900C009B400B0F8
:106B00000AAF00B00BAA00D00CA500000EA00050E8
:106B10000F9B00C01096005012910000148C00C012
:106B2000158700B0178200B0197D00D01B780000D7
:106B30001E730040206E0090226900F02464004023
:106B4000275F0090295A00E02B5500102E5000209E
:106B5000304B0010324600E033410090353C0010CD
:106B600037370070383200A0392D00B03A2800A025
:106B70003B2300603C1E00103D1900903D140010A6
:106B80003E0F00703E0A00C03E0500003F0000407E
:106B90003FFBFF803FF6FFC03FF1FF2020506C61BC
:106BA0006E6E657242756666657242797465733A97
:106BB00020002046726565204D656D6F72793A2020
:106BC00000436F6D70696C65643A204170722032C9
:106BD0003520323032310A00204C617374205570F8
:106BE00064617465643A20323032312D30342D3195
:106BF00038207C20417574686F723A2054696E7930
:106C00004D616368696E657333440A00322E302E1D
:106C1000375F4457372E330A004D61726C696E003E
:106C200020536F6674776172652052657365740ACC
:106C300000205761746368646F67205265736574E0
:106C40000A002042726F776E206F75742052657350
:106C500065740A002045787465726E616C20526517
:106C60007365740A00506F77657255700A0073740B
:106C70006172740A004732385859004D3130303152
:106C8000006572726F722077726974696E67207422
:106C90006F2066696C650A00446F6E6520736176CB
:106CA000696E672066696C652E0A004D32390045B1
:106CB0006E6473746F707300255320256320256301
:106CC00020256320256300205A3A0020593A0020ED
:106CD000583A00656E6473746F7073206869743A13
:106CE000200000000A0B02090C0D0E080703040126
:106CF0000000000000000000000000000000000094
:106D00000000000000000000000000000000121160
:106D10001000000000000000000000000000000063
:106D20000000000000000000004D6F766520257314
:106D30006D6D004D6F766520302E316D6D004D6F9D
:106D4000766520316D6D004D6F76652031306D6D4B
:106D5000004D6F76652041786973004578747275CF
:106D6000646572004D6F7665205A004D6F76652020
:106D700059004D6F766520580061655D6543686117
:106D80006E67652046696C616D656E7400556E6C4A
:106D90006F61642046696C616D656E74004C6F6153
:106DA000642046696C616D656E740050726568653B
:106DB000617420437573746F6D005072656865610E
:106DC000742024004261636B0073686F7700627502
:106DD00074746F6E00626567696E00446973616206
:106DE0006C6552756E6F75740050757267654D6F86
:106DF00072650050617573656400436F6E74696EEF
:106E00007565004C6F61642046696C616D656E74D8
:106E1000205400496E736572742066696C616D65FB
:106E20006E7420616E642073656E64204D3130385D
:106E30000A00220A00556E6B6E6F776E20636F6DCD
:106E40006D616E643A2022002042002050006F6B7A
:106E500000204500205A00205900204D393220588A
:106E60000020453A00205A3A0020593A00583A008A
:106E700020746F6F206C6F6E672065787472757305
:106E8000696F6E2070726576656E7465640A0020A5
:106E9000636F6C6420657874727573696F6E2070AF
:106EA000726576656E7465640A00526573656E641A
:106EB0003A20006E6F74696669636174696F6E2051
:106EC0000000002200250028002B002E0031003495
:106ED0000002010000050108010B0100002100244F
:106EE0000027002A002D00300033000101000004BB
:106EF0000107010A0105050505070508080808023C
:106F00000202020A0A080804040404010101010142
:106F10000101010303030303030303040707070C31
:106F20000C0C0C0C0C0C0C020202020606060606E7
:106F30000606060B0B0B0B0B0B0B0B010210202094
:106F400008081020401020408002010201080402BD
:106F50000101020408102040808040201008040233
:106F6000018004020180402010080402010804028C
:106F70000101020408102040800102040810204092
:106F8000800045026D0111241FBECFEFD1E2DEBFAC
:106F9000CDBF00E00CBF17E0A0E0B2E0E4E9FCE9FF
:106FA00003E00BBF02C007900D92A033B107D9F7E1
:106FB00020E2A0E3B7E001C01D92AB33B207E1F7D6
:106FC00017E3C2ECD7E300E006C021970109802F48
:106FD000FE010F944DC9C13CD10780E00807A9F715
:106FE0000F943BB70D9438CE0C9400006091390299
:106FF00070913A02072E000C880B990B0F946BC20C
:107000002AE037ED43E25CE30F94CAC220912709DE
:10701000309128094091290950912A090F94CAC238
:1070200060938E0270938F028093900290939102EE
:107030000895E0916D0FE23030F4F0E0E852FF4E39
:1070400080915B0F808308958091241E8823C1F076
:1070500081508093241EE0E5FEE1882351F08150A9
:10706000990B2BE1289FF001299FF00D1124EA577D
:10707000F14E8BE1ABE6BEE101900D928A95E1F70E
:107080002091241E211105C080912F1E80628093C3
:107090002F1E81E090E0A0E0B0E0211103C080E06D
:1070A00090E0DC018093530F9093540FA093550F01
:1070B000B093560F1092580F81E08093520F83E0E7
:1070C0008093820208950E94568E8BE69DE09093F5
:1070D000FB0E8093FA0E0895CF93DF93EC01CB0162
:1070E000BA010F946BC229EC38EC48EC5EE30F94C4
:1070F00050CA20E030E040E05FE30F9456C90F949F
:10710000C9CA6883DF91CF910895E0916D0F86E041
:10711000E802F0011124E25CF04F80915B0F90E0F7
:107120009583848308958F929F92AF92BF92CF925E
:10713000DF92EF92FF92CF936B017C0120E030E071
:10714000A9010F9464C287FD9FC06DEB77E386E0D1
:1071500095E3A70196010F9456C96B017C0120E0CD
:1071600030E040E251E40F94CAC220E030E048EC45
:1071700052E40F94CAC24B015C0120E030E0A90147
:10718000C701B6010F9464C220E030E040EA50E449
:1071900087FF04C020E030E040EA50ECC501B401B4
:1071A0000F9456C920E030E040E251E40F9450CAF9
:1071B0000F94C2CA6B017C018BE2F7FE09C0F09408
:1071C000E094D094C094C11CD11CE11CF11C8DE250
:1071D0008093640FC701B60120E137E240E050E040
:1071E0000F94CAC88AE0882E912CA12CB12CCA0118
:1071F000B901A50194010F94CAC8605D6093650F41
:10720000C701B60128EE33E040E050E00F94CAC851
:10721000CA01B901A50194010F94CAC8605D6093C9
:10722000660FC701B60124E630E040E050E00F945D
:10723000CAC8CA01B901A50194010F94CAC8605D0A
:107240006093670F8EE28093680FC701B601A501B6
:1072500094010F94CAC8C62FCA01B901A5019401AF
:107260000F94CAC8605D6093690FC05DC0936A0FD8
:1072700084E69FE0CF91FF90EF90DF90CF90BF909A
:10728000AF909F908F9008956DEB77E386E095EB3C
:1072900060CF8F929F92AF92BF92CF92DF92EF9288
:1072A000FF926B017C0120E030E0A9010F9464C2E1
:1072B00087FD6BC06DEB77E386E095E3A701960150
:1072C0000F9456C96B017C0120E030E040E251E4AC
:1072D0000F94CAC220E030E040E251E40F94CAC2E9
:1072E0004B015C0120E030E0A901C701B6010F9419
:1072F00064C220E030E040EA50E487FF04C020E0B0
:1073000030E040EA50ECC501B4010F9456C920E0CA
:1073100030E040E251E40F9450CA0F94C2CA9B017E
:107320008BE237FF05C022273327261B370B8DE260
:107330008093660FC90164E670E00F9439C9CB01F0
:10734000EAE0F0E0BF010F9439C9805D8093670FD8
:10735000C901BF010F9439C9282FCB01BF010F9478
:1073600039C9805D8093680F8EE28093690F205D3C
:1073700020936A0F86E69FE0FF90EF90DF90CF901A
:10738000BF90AF909F908F9008956DEB77E386E06C
:1073900095EB94CF8F929F92AF92BF92CF92DF9254
:1073A000EF92FF92CF936B017C0120E030E0A901C6
:1073B0000F9464C287FDAAC06DEB77E386E095E386
:1073C000A70196010F9456C96B017C0120E030E0C3
:1073D000A9010F9464C287FF9EC0C701B6019058EF
:1073E00020E030E040E251E40F94CAC220E030E0F7
:1073F00040E251E40F94CAC220E030E040EA50E499
:107400000F9456C920E030E040E251E40F9450CA96
:107410000F94C2CA6B017C0180E28093640F60E22A
:1074200080E1C81687E2D806E104F1048CF0C701B8
:10743000B60120E137E240E050E00F94CAC8CA012B
:10744000B9012AE030E040E050E00F94CAC8605D26
:107450006093650F60E288EEC81683E0D806E10409
:10746000F1048CF0C701B60128EE33E040E050E0B3
:107470000F94CAC8CA01B9012AE030E040E050E0E8
:107480000F94CAC8605D6093660F60E284E6C81618
:10749000D104E104F1048CF0C701B60124E630E028
:1074A00040E050E00F94CAC8CA01B9012AE030E0B8
:1074B00040E050E00F94CAC8605D6093670F8AE0B7
:1074C000882E912CA12CB12CC701B601A5019401E5
:1074D0000F94CAC8C62FCA01B901A50194010F941F
:1074E000CAC8605D6093680F8EE28093690FC05DCB
:1074F000C0936A0F84E69FE0CF91FF90EF90DF90FA
:10750000CF90BF90AF909F908F9008956DEB77E3F1
:1075100086E095EB55CF20E030E040E251E4C70132
:10752000B60162CFCF93DF93EC01CB01BA010F9488
:107530006BC220E030E040E251E40F9450CA20E0FA
:1075400030E0A9010F9456C9688379838A839B83AD
:10755000DF91CF910895CF93DF93EC01CB01BA0176
:107560000F946BC220E030E040E251E40F9450CA27
:1075700020E030E0A9010F9456C9688379838A839B
:107580009B83DF91CF9108950F946BC220E030E090
:1075900040E251E40F9450CA20E030E0A9010F947A
:1075A00056C90C94CA39CF93DF93EC01CB01BA01D1
:1075B0000F946BC220E030E040E251E40F9450CAD7
:1075C00020E030E0A9010F9456C9688379838A834B
:1075D0009B83DF91CF9108950F946BC220E030E040
:1075E00040E251E40F9450CA20E030E0A9010F942A
:1075F00056C90C944939CF93DF93EC01CB01BA0102
:107600000F946BC22AE037ED43E25DE30F9450CA5A
:1076100020E030E0A9010F9456C90F94C9CA6883CD
:1076200079838A839B83DF91CF910895CF93DF93F2
:10763000EC01CB01BA010F946BC22AE037ED43E2B3
:107640005DE30F9450CA20E030E0A9010F9456C9C1
:10765000688379838A839B83DF91CF910895CF9349
:10766000DF93EC01CB01BA010F946BC220E030E054
:10767000A9010F9456C9688379838A839B83DF911C
:10768000CF910895CF93DF93EC01CB01BA010F9412
:107690006BC220E030E0A9010F9456C9688379835A
:1076A0008A839B83DF91CF910895CF93DF93EC0181
:1076B000CB01BA010F946BC220E030E048EC52E4F9
:1076C0000F9450CA20E030E0A9010F9456C9688396
:1076D00079838A839B83DF91CF910895CF93DF9342
:1076E000EC01CB01BA010F946BC220E030E048EC12
:1076F00052E40F9450CA20E030E0A9010F9456C91B
:10770000688379838A839B83DF91CF9108950F9457
:107710006BC220E030E048EC52E40F9450CA20E005
:1077200030E0A9010F9456C90C949338CF93DF939E
:10773000EC01CB01BA010F946BC220E030E0A9014B
:107740000F9456C90F94C2CA79836883DF91CF9191
:107750000895CF93DF93EC01CB01BA010F946BC274
:1077600020E030E0A9010F9456C9688379838A83A9
:107770009B83DF91CF910895CF93DF93EC01CB01F1
:10778000BA010F946BC220E030E04AE754E40F9452
:1077900050CA20E030E0A9010F9456C9688379836C
:1077A0008A839B83DF91CF9108952CEA35EC47E2E1
:1077B0005EE36091300770913107809132079091BC
:1077C00033070F9450CA60931A1D70931B1D80934A
:1077D0001C1D90931D1D08952CEA35EC47E25EE3D5
:1077E0006091340770913507809136079091370783
:1077F0000F94CAC26093161D7093171D8093181DB5
:107800009093191D08950F946BC220E030E0A901F8
:107810000F9456C90F94C2CACB010D94881D809154
:10782000AD1D9091AE1D891B8F70B9F48091F70E3C
:107830008770873051F01092F70E1092260980E180
:1078400094E19093FB0E8093FA0E20E040E070E00C
:1078500060E08BE291E40C94D38D089520E040E049
:1078600070E060E08FE69CE40C94D38D8091EA1088
:10787000811114C0809192029091930201972091FE
:107880000D1D30910E1D2817390744F420E040E00B
:1078900070E060E084E79CE40C94D38D0C942E3C63
:1078A00021E020934507FC0180819181A281B38171
:1078B0008093110290931202A0931302B0931402CA
:1078C00020E040E070E060E080914E0F90914F0F1B
:1078D0000C94D38DCF93DF9300D01F92CDB7DEB73A
:1078E0008DEC9CECACECBCE389839A83AB83BC83CA
:1078F000CE0101960E94503C0F900F900F900F9078
:10790000DF91CF910895CF93DF9300D01F92CDB731
:10791000DEB78DEC9CECACECBDE389839A83AB8342
:10792000BC83CE0101960E94503C0F900F900F90A7
:107930000F90DF91CF910895CF93DF9300D01F92E6
:10794000CDB7DEB780E090E0A0E8BFE389839A83FB
:10795000AB83BC83CE0101960E94503C0F900F90E8
:107960000F900F90DF91CF910895CF93DF9300D0C8
:107970001F92CDB7DEB780E090E0A0E2B1E489834A
:107980009A83AB83BC83CE0101960E94503C0F903A
:107990000F900F900F90DF91CF9108958FEF80930C
:1079A0005B0F20E040E070E060E083E499E70C9436
:1079B000D38D8F929F92AF92BF92CF92DF92EF9230
:1079C000FF920F931F93CF93DF9361E081E00E94BA
:1079D000758DC091580F85E0982E9C0E97E2E92E88
:1079E00094E1F92ED3E0DC1B2DE3C22E24E1D22E4C
:1079F00012E01C1B33E5A32E34E1B32E01E00C1B77
:107A00008C2E8194C11133C08091570F8823B1F01F
:107A100080918202882359F081E09091570F911153
:107A200080E024E04DE455E1682D0F94799ECF5F0E
:107A3000C911E8CF84E08093510F0CC08091500FA2
:107A40001092500F882321F30E94BB8E8091520F19
:107A50008823F1F2DF91CF911F910F91FF90EF906A
:107A6000DF90CF90BF90AF909F908F900895C130DE
:107A700001F59091570F913069F08091820288232F
:107A8000B1F281E0913009F080E020E243E454E17A
:107A9000602FCBCF8091500F1092500F882369F345
:107AA000B092FB0EA092FA0E8091520F882329F318
:107AB000D1CFC23081F59091570F923071F0809103
:107AC0008202882309F4B3CF81E0923009F080E08C
:107AD00020E24EE254E1612FA8CF8091500F109226
:107AE000500F882361F3D092FB0EC092FA0E809162
:107AF000520F882321F3AECF8091500F1092500F78
:107B0000882381F0F092FB0EE092FA0E8091520FE2
:107B1000882341F09FCFC33009F089CF9091570F50
:107B2000933051F380918202882309F480CF81E061
:107B3000933009F080E020E244E154E16D2F75CFED
:107B40003F924F925F926F927F928F929F92AF92ED
:107B5000BF92CF92DF92EF92FF920F931F93CF933A
:107B6000DF9361E081E00E94758DC091580F85E040
:107B7000482E4C0E96E5E92E9EE8F92E2EEAC22EEE
:107B800022E1D22ED4E0DC1B3DE6A32E32E1B32E5F
:107B900083E0782E7C1A44E8842E42E1942E82E021
:107BA000682E6C1A81E0582E5C1A3C2E3194C1115B
:107BB00033C08091570F882389F0809182028823F7
:107BC00009F448C081E09091570F911180E024E0C2
:107BD00044EA54E1632D0F94799E3CC08091500F8C
:107BE0001092500F882349F30E94BB8E8091520F50
:107BF000882319F3DF91CF911F910F91FF90EF90A0
:107C0000DF90CF90BF90AF909F908F907F906F90BC
:107C10005F904F903F900895C130D1F58091570FFC
:107C20008130F9F0809182028823A1F011E08091E7
:107C3000570F813009F010E080910E0290910F02F1
:107C40000F94881D00E09C014CE852E1652D812FC6
:107C50000E94FB9BCF5FC411AACF85E08093510F98
:107C6000C9CF8091500F1092500F8823D9F20CE5A4
:107C700013E429E030E050E040E06EE072E08CE890
:107C800092E10F944CA18091520F882359F2B2CF08
:107C9000C23009F04EC09091570F923069F0809138
:107CA00082028823B9F281E0923009F080E020E27C
:107CB00046E752E1662D8FCF8091500F1092500F02
:107CC000882369F39092FB0E8092FA0E8091520FF6
:107CD000882329F38FCF9091570F933071F08091C3
:107CE0008202882309F4B6CF81E0933009F080E066
:107CF00020E24EE552E1672D6ECF8091500F109239
:107D0000500F882361F3B092FB0EA092FA0E80917F
:107D1000520F882321F36ECF8091500F1092500F95
:107D2000882381F00E94568E8091520F882351F053
:107D300061CFC33081F2C43009F08CCF8091570FEE
:107D4000843051F380918202882309F483CFFF921B
:107D5000EF92DF92CF92DF9381E09091570F9430B2
:107D600009F080E08F930E943F8D0F900F900F904D
:107D70000F900F900F906ECF9F92AF92BF92CF92C5
:107D8000DF92EF92FF920F931F93CF93DF9361E007
:107D900081E00E94758DC091580F85E0E82EEC0EB1
:107DA00096E5C92E9EE8D92E2EEAA22E22E1B22E09
:107DB000D2E0DC1B81E0F82EFC1A9C2E9194C111BC
:107DC00032C08091570F8823B1F0809182028823BE
:107DD00059F081E09091570F911180E024E047E63F
:107DE00054E1692D0F94799ECF5FCE11E8CF83E0E7
:107DF0008093510F0CC08091500F1092500F882328
:107E000021F30E94BB8E8091520F8823F1F2DF9103
:107E1000CF911F910F91FF90EF90DF90CF90BF9087
:107E2000AF909F900895C130A1F58091570F813098
:107E3000C9F0809182028823B9F211E08091570F36
:107E4000813009F010E080910602909107020F94B2
:107E5000881D00E09C0149E651E16F2D812F0E94B1
:107E6000FB9BC2CF8091500F1092500F882309F3D3
:107E700003EA18E429E030E047EF5FEF66E072E0E4
:107E800089E691E10F944CA18091520F882389F2E9
:107E9000BECFC23009F0A8CF8091570F8230D1F009
:107EA00080918202882309F49FCFDF92CF92BF9204
:107EB000AF92DF9381E09091570F923009F080E00C
:107EC0008F930E943F8D0F900F900F900F900F9007
:107ED0000F908ACF8091500F1092500F882301F39A
:107EE0000E94568E8091520F8823D1F290CF5F92DC
:107EF0006F927F928F929F92AF92BF92CF92DF92BA
:107F0000EF92FF920F931F93CF93DF9361E081E095
:107F10000E94758DC091580F85E0982E9C0ED1E07F
:107F200093EAE92E9AE0F92E882483947D2E7C1A18
:107F30006C2E619425E8C22E2AE0D22E12E01C1B82
:107F400033E0532E43E0A42E41E0B42EC11141C0D2
:107F5000DD23D9F08091570F1816BCF04091530FD4
:107F60005091540F6091550F7091560F4F5F5F4FB6
:107F70006F4F7F4F4093530F5093540F6093550FA3
:107F80007093560F8F5F8093570F809182028823E2
:107F900041F030E020E041E06EEA7AE0862D0E9478
:107FA000C6998091960F882309F487C0C23051F496
:107FB0008091570F823009F445C08091820281116F
:107FC0005AC0D0E0CF5F9C12C1CF83E08093510FA5
:107FD00018C0C13031F79091570F913031F0809136
:107FE000820281111EC0D0E0DCCF8091500F109230
:107FF000500F8823A1F3C093970F8091520F8823CD
:1080000071F3DF91CF911F910F91FF90EF90DF906F
:10801000CF90BF90AF909F908F907F906F905F9028
:1080200008951F92FF92EF927F9281E0913009F0C4
:1080300080E08F930E943F8D0F900F900F900F90D4
:108040000F90D1CF8091500F1092500F882309F4D8
:10805000B4CF8091590288258093590250928202B0
:10806000A114B10411F00F94E3358091520F8823CD
:1080700009F4A3CFC6CF81E09091570F923009F059
:1080800080E09091590222E93AE0911102C02EE875
:108090003AE001E045E95AE0612F0E94FB9B91CF55
:1080A0008091500F1092500F882371F0C093970F5A
:1080B0008091520F882341F0A4CFC23009F082CFC3
:1080C0009091570F923061F380918202882309F4D6
:1080D00078CF1F92DF92CF921F9381E0923009F008
:1080E00080E08F930E943F8D0F900F900F900F9024
:1080F0000F9067CF69EA7BE38FE490E60C945F9B77
:108100006CE678E381E799E40C945F9B6BEA7AE391
:1081100084EC9AE30C945F9B63ED7AE38CEE9AE334
:108120000C945F9B6BEF7AE385E199E50C945F9B80
:1081300066E17BE387E599E50C945F9B62E47BE372
:1081400086E699E50C945F9B6EE67BE387E89BE30C
:108150000C945F9B62E97AE38CEB9FE40C945F9B49
:1081600066E97BE383E09CE30C945F9B6FE27BE337
:108170008BEE93E80C945F9B6CEB7BE387E294E8D7
:108180000C945F9B65E57BE389E09FE70C945F9B24
:1081900061E08BE59FE00D9440468F929F92AF92F5
:1081A000BF92CF92DF92EF92FF92CF93DF9300D0F6
:1081B00000D01F921F92CDB7DEB7809150070F9469
:1081C000953F4B015C0189829A82AB82BC8280918F
:1081D00051070F94FF3E6B017C01CD82DE82EF825E
:1081E000F886CE0101960F940B45882319F18092F1
:1081F0009B1090929C10A0929D10B0929E10C092E5
:108200009F10D092A010E092A110F092A2108EEFD9
:1082100028960FB6F894DEBF0FBECDBFDF91CF9189
:10822000FF90EF90DF90CF90BF90AF909F908F9096
:108230000C94D69028960FB6F894DEBF0FBECDBF33
:10824000DF91CF91FF90EF90DF90CF90BF90AF90F4
:108250009F908F90089581E08093450780918202DE
:10826000882341F030E020E041E065E074E182E005
:108270000E94C699809126098770873049F581E070
:1082800080934407809151076091500770E09FE010
:10829000899F600D711D112420E040E089E691E482
:1082A0000E94D38D109211021092120210921302AA
:1082B000109214020E94CD4080E090E0A0E8BFE35D
:1082C0008093110290931202A0931302B0931402B0
:1082D00008953F924F925F926F927F928F929F92FA
:1082E000AF92BF92CF92DF92EF92FF920F931F93C4
:1082F000CF93DF93CDB7DEB7C654D1090FB6F8944C
:10830000DEBF0FBECDBF80914307882309F4A1C013
:108310008091500F1092500F882309F450C0809123
:1083200050070F94953F7E012DE3E20EF11C87016B
:1083300022E040E00F94F4BC809151070F94FF3E7F
:108340006E01E3E3CE0ED11C860122E040E00F94E3
:10835000F4BC809110021F928F93DF92CF92FF9214
:10836000EF9289EE93E19F938F931F9282E38F9315
:10837000025311091F930F930F94BEC1C8010E94AD
:108380004D8D0FB6F894DEBF0FBECDBFCA5BDF4F79
:108390000FB6F894DEBF0FBECDBFDF91CF911F9116
:1083A0000F91FF90EF90DF90CF90BF90AF909F9094
:1083B0008F907F906F905F904F903F90089581E0F5
:1083C000809345078091530F9091540FA091550FC2
:1083D000B091560FB7FF0CC080EE90E0A0E0B0E087
:1083E0008093530F9093540FA093550FB093560F53
:1083F0008091530F9091540FA091550FB091560F4B
:10840000813E9105A105B10544F01092530F1092E1
:10841000540F1092550F1092560F6091530F709198
:10842000540F8091550F9091560F2FE030E040E0AF
:1084300050E00F94A8C8615021502D3028F489E0F5
:108440006D3028F086E003C084E06D30D8F380936F
:1084500010026091530F7091540F8091550F9091BD
:10846000560F2FE030E040E050E00F94A8C8322EC5
:108470006B0180918202882309F4FEC080911D1E49
:108480008C3308F580911F1E8830E8F081E08093DE
:10849000091E01E321E348E065E289EE9DE10F94C6
:1084A000F6AC80911D1E883370F480911F1E8A30B7
:1084B00050F01092091E0DE22DE24AE067E289EECB
:1084C0009DE10F94F6AC81E08093091E1BE0809142
:1084D0001D1E181798F080911F1E811778F098E2E2
:1084E000A92E01E021E0412F6A2D89EE9DE10F9434
:1084F000F6AC93E0A90EE5E5AE12F3CF1D5F18339D
:1085000031F78EE08319482F440F480F465F842FC0
:1085100090E0039620911D1E2817190609F074F4A7
:1085200080911F1E841750F06C2D660F6C0D695DD5
:1085300003E023E089EE9DE10F94F6AC81E08093A7
:10854000091E80911D1E883008F047C08C2D0F94A5
:10855000953F4B015C01832D0F94FF3E20919310BA
:108560003091941040919510509196100F9456C9E7
:108570002B013C01A501940160918F107091901026
:1085800080919110909192100F9456C969837A83CB
:108590008B839C834D825E826F82788685E0809398
:1085A000201E17E01093211E8DE69EE60E94859600
:1085B000CE0101960F943B1C0E944D9A8AE4809351
:1085C000201E1093211E82E094E10E948596CE0128
:1085D00005960F943B1C0E944D9A80911D1E81347C
:1085E00008F04AC080911F1E873308F445C085E01B
:1085F0008093201E10E41093211E68E270E080E05A
:1086000090E00E94B5938C2D0F94559F6CE270E022
:1086100080E090E00E94B593832D0F94559F69E20E
:1086200070E080E090E00E94B5938AE48093201E81
:108630001093211E8FEF93E10E9485968FE08C9D11
:1086400080018D9D100D1124030D111D000F111FB0
:10865000000F111F0C5C164FF8016081718182813F
:1086600093819B01AC010F94A3CC811120C0C80160
:108670000F94BA9E0E944D9A80915007082E000CCC
:10868000990B8C159D0549F480915107082E000C1B
:10869000990B3816190609F479CEC092500730921A
:1086A00051070E94CD4082E0809382026FCE88EF16
:1086B00093E10E948596E0CF0F931F93CF93DF93B2
:1086C000CDB7DEB762970FB6F894DEBF0FBECDBF51
:1086D00080910F028F9380910E028F9383E592E138
:1086E0009F938F938E010F5F1F4F1F930F930F94D4
:1086F000FBC1C8010E94FCD10F900F900F900F900A
:108700000F900F9062960FB6F894DEBF0FBECDBFEC
:10871000DF91CF911F910F9108955F926F927F9299
:108720008F929F92AF92BF92CF92DF92EF92FF9281
:108730000F931F93CF93DF93CDB7DEB72C970FB670
:10874000F894DEBF0FBECDBF61E081E00E94758D61
:10875000F090580F85E0C82ECF0C9BE0A92E92E137
:10876000B92ECE0101964C0122E1622E22E1722E39
:1087700082E0E82EEF1881E0D82EDF185F2C5194AC
:10878000F1103CC08091570F8823B1F08091820294
:10879000882359F081E09091570F911180E024E0F7
:1087A00043E855E1652D0F94799EF394FC10E8CFD2
:1087B00083E08093510F0CC08091500F1092500FA6
:1087C000882321F30E94BB8E8091520F8823F1F2FF
:1087D0002C960FB6F894DEBF0FBECDBFDF91CF91C0
:1087E0001F910F91FF90EF90DF90CF90BF90AF90CF
:1087F0009F908F907F906F905F90089591E0F91215
:1088000034C08091570F8130C9F080918202882353
:1088100061F211E08091570F813009F010E08091F2
:108820000C0290910D020F94881D00E09C014DE117
:1088300052E16D2D812F0E94FB9BB7CF8091500F8D
:108840001092500F882309F310E000E026E030E09A
:1088500042E050E06CE072E08DE192E10F944CA1B7
:108860008091520F882389F2B3CF82E0F8129DCF16
:108870008091570F8230C1F080918202882309F4E1
:1088800094CF1F927F926F92EF9281E09091570F59
:10889000923009F080E08F930E943F8D0F900F90EF
:1088A0000F900F900F9081CF8091500F1092500F2A
:1088B000882311F380910D028F9380910C028F9386
:1088C000BF92AF929F928F920F94FBC1C4010E94FE
:1088D0004D8D0F900F900F900F900F900F908091F3
:1088E000520F882349F274CF0F931F93CF93DF93D6
:1088F000CDB7DEB764970FB6F894DEBF0FBECDBF1D
:1089000080910B028F9380910A028F9380910902CC
:108910008F93809108028F938CEB91E19F938F93BB
:108920008E010F5F1F4F1F930F930F94FBC1C80160
:108930000E944D8D0FB6F894DEBF0FBECDBF64967A
:108940000FB6F894DEBF0FBECDBFDF91CF911F9160
:108950000F9108952F923F924F925F926F927F9264
:108960008F929F92AF92BF92CF92DF92EF92FF923F
:108970000F931F93CF93DF9361E081E00E94758D89
:10898000C091580F3C2E85E0482E4C0E06E51EE89F
:108990009EEAE92E92E1F92ED4E0DC1B5524539493
:1089A00024E7C22E24E4D22E3CECA32E31E1B32ED8
:1089B00083E0782E7C1A4BE7842E4DE6942E82E0DD
:1089C000682E6C1A252C2C1AC1113AC08091570FB1
:1089D0008823B9F080918202882361F0632D61952C
:1089E00081E09091570F911180E024E043E855E138
:1089F0000F94799ECF5FC411E7CF85E08093510F2C
:108A00000CC08091500F1092500F882319F30E94D0
:108A1000BB8E8091520F8823E9F2DF91CF911F9195
:108A20000F91FF90EF90DF90CF90BF90AF909F900D
:108A30008F907F906F905F904F903F902F90089510
:108A4000C13061F5E9E7FDE68591949110926D0FD3
:108A500090936F0F80936E0F9091570F913069F044
:108A600080918202882331F281E0913009F080E028
:108A700020E24DEE51E1622DBBCF8091500F10925C
:108A8000500F882369F32FEF31E13093FB0E2093D1
:108A9000FA0E8091520F882319F3BFCFC23009F02C
:108AA0005BC0F4018591949150926D0F90936F0F7C
:108AB00080936E0F9091570F923071F080918202E7
:108AC000882309F497CF81E0923009F080E020E21A
:108AD0004DEE51E1662D8CCF8091500F1092500FCA
:108AE000882361F321EE31E13093FB0E2093FA0EDF
:108AF0008091520F882311F390CF8091570F8330CC
:108B000089F080918202882309F474CFDF92CF929A
:108B1000BF92AF927F9281E09091570F9330A1F175
:108B200080E032C08091500F1092500F882349F39B
:108B30000E9474448091520F882319F36ECF809164
:108B4000500F1092500F882381F00E94568E809112
:108B5000520F882351F061CFC33079F2C43009F04D
:108B600049CF8091570F843051F38091820288233E
:108B700009F440CF1F930F93FF92EF92DF9381E0B0
:108B80009091570F943061F68F930E943F8D0F9014
:108B90000F900F900F900F900F902CCF0F931F936B
:108BA000CF93DF93CDB7DEB7C054D1090FB6F89499
:108BB000DEBF0FBECDBF809109028F938091080266
:108BC0008F9380910B028F9380910A028F938BE297
:108BD00091E19F938F938E010F5F1F4F1F930F9310
:108BE0000F94FBC1C8010E944D8D0FB6F894DEBFF3
:108BF0000FBECDBFC05CDF4F0FB6F894DEBF0FBE17
:108C0000CDBFDF91CF911F910F9108958F929F92C9
:108C1000AF92BF92CF92DF92EF92FF920F931F938A
:108C2000CF93DF9361E081E00E94758DC091580F72
:108C300085E0982E9C0E9EECC92E95E4D92E2EE14F
:108C4000A22E23E1B22ED3E0DC1B82E0F82EFC1A28
:108C500081E0E82EEC1A8C2E8194C11133C08091F2
:108C6000570F8823B1F080918202882359F081E068
:108C70009091570F911180E024E044EA54E1682D6F
:108C80000F94799ECF5FC911E8CF84E08093510F94
:108C90000CC08091500F1092500F882321F30E9436
:108CA000BB8E8091520F8823F1F2DF91CF911F91FB
:108CB0000F91FF90EF90DF90CF90BF90AF909F907B
:108CC0008F900895C130A1F58091570F8130C9F080
:108CD000809182028823B1F211E08091570F813098
:108CE00009F010E080910802909109020F94881D0C
:108CF00000E09C0141E551E16E2D812F0E94FB9B1C
:108D0000C1CF8091500F1092500F882309F310E0CB
:108D100000E02CE231E04AEA50E068E072E081E5F0
:108D200091E10F944CA18091520F882389F2BDCF1D
:108D3000C23009F03FC08091570F8230B9F0809166
:108D40008202882309F49ECF11E08091570F823070
:108D500009F010E080910A0290910B020F94881D97
:108D600000E09C0148E451E16F2DC7CF8091500F86
:108D70001092500F882319F310E000E02CE830E047
:108D800045E050E06AE072E088E491E10F944CA184
:108D90008091520F882399F288CF8091500F1092C2
:108DA000500F882371F00E94CE458091520F882386
:108DB00041F07BCFC33009F065CF8091570F8330EE
:108DC00061F380918202882309F45CCFDF92CF9215
:108DD000BF92AF92DF9381E09091570F933009F0EB
:108DE00080E08F930E943F8D0F900F900F900F9017
:108DF0000F900F9047CFEF92FF920F931F93CF9357
:108E0000DF93CDB7DEB7A8970FB6F894DEBF0FBEDD
:108E1000CDBFF62EE72E90914F079F9390914E076E
:108E20009F93282F082E000C330B3F938F938BE8D2
:108E300093E19F938F938E010F5F1F4F1F930F93AB
:108E40000F94FBC1F80101900020E9F7CF012091B8
:108E50004F072F9320914E072F93EF92FF92019788
:108E60009F938F930F94FBC1C8010E94FCD10FB652
:108E7000F894DEBF0FBECDBFA8960FB6F894DEBF44
:108E80000FBECDBFDF91CF911F910F91FF90EF905B
:108E9000089568EA73E183E50C94FB4669E973E1A0
:108EA0008CE40C94FB462F923F924F925F926F920C
:108EB0007F928F929F92AF92BF92CF92DF92EF926A
:108EC000FF920F931F93CF93DF9300D01F92CDB7E4
:108ED000DEB70E948AE99C838B8361E081E00E9477
:108EE000758D5090580F25E0250D298311E0352D03
:108EF00031953A83212E251889E4682E87E4782E4F
:108F000096EBE92E93E1F92E83E0482E45182EE4E6
:108F1000C22E27E4D22E34ECA32E33E1B32E82E00E
:108F2000382E35188B809C8081E0881A910851106A
:108F30000AC08091570F882309F445C080918202AE
:108F4000811166C010E080914E0790914F0797FD08
:108F500006C02B813C81821793070CF465C031E079
:108F6000531229C01123D9F08091570F8230BCF4DD
:108F70004091530F5091540F6091550F7091560FBF
:108F80004F5F5F4F6F4F7F4F4093530F5093540F7E
:108F90006093550F7093560F8F5F8093570F80919A
:108FA0008202882341F030E020E041E06EED73E181
:108FB000822D0E94C69982E0539439813511B7CF32
:108FC0008093510F0EC08091500F1092500F882344
:108FD00009F4B4CF0E94BB8E8091520F882309F40C
:108FE000ADCF0F900F900F900F90DF91CF911F9109
:108FF0000F91FF90EF90DF90CF90BF90AF909F9038
:109000008F907F906F905F904F903F902F9008953A
:1090100081E09091570F911180E024E04DE455E1FB
:109020006A810F94799E8ECF81E0581235C080916D
:10903000570F8130D9F0809182028823A1F011E08E
:109040008091570F813009F010E080914E07909188
:109050004F070F94881D00E09C0142ED53E1622D03
:10906000812F0E94FB9B10E084E0A6CF8091500FDF
:109070001092500F8823F9F210E000E0940150E0C4
:1090800040E06EE477E082ED93E10F944CA1809193
:10909000520F882381F2A5CF92E0591221C080910E
:1090A000570F823081F0809182028823E1F2DF92B3
:1090B000CF92BF92AF923F9281E09091570F923042
:1090C00029F180E023C08091500F1092500F882327
:1090D00051F30E944E478091520F882321F381CF94
:1090E00023E05212C1CF8091570F8330C9F0809195
:1090F0008202882309F4B7CF7F926F92FF92EF929A
:109100004F9281E09091570F9330D9F68F930E9440
:109110003F8D0F900F900F900F900F900F90A3CF57
:109120008091500F1092500F882309F30E944947F5
:109130008091520F8823D9F254CF0F94FB458BE9CD
:1091400092E10D94D54A0F931F93CF93DF93CDB740
:10915000DEB72D970FB6F894DEBF0FBECDBF80915E
:1091600006029091070207E010E01816190614F4A1
:1091700006E010E061E671E1CE0101960F946DC149
:10918000809106029091070297FF03C09195819507
:1091900091099F938F938DE591E19F938F9381E048
:1091A00090E08C0F9D1F080F191F1F930F930F94B2
:1091B000FBC1CE0101960E944D8D0F900F900F9034
:1091C0000F900F900F902D960FB6F894DEBF0FBE44
:1091D000CDBFDF91CF911F910F910895CF92DF9274
:1091E000EF92FF92CF93DF9300D01F92CDB7DEB7FF
:1091F00081E0809345078091410790914207892B38
:1092000041F180914107909142072AE037ED43EA0E
:109210005BEB1816190624F42AE037ED43EA5BE30A
:1092200060914A0770914B0780914C0790914D07D0
:109230000F9456C960934A0770934B0780934C076D
:1092400090934D07109242071092410782E080935D
:109250008202809182028823C9F120E030E04AE74F
:1092600054E460914A0770914B0780914C079091AC
:109270004D070F94CAC20F94C2CA6B017C0125E04E
:1092800030E040E050E00F94CAC8A7019601261BC9
:10929000370B480B590BCA01B9010F946BC220E080
:1092A00030E04AE754E40F9450CA69837A838B8391
:1092B0009C83CE0101960F94BA9EBC0183E291E19A
:1092C0000E94519ACE0101960E9446920F900F90F3
:1092D0000F900F90DF91CF91FF90EF90DF90CF90A4
:1092E00008950F946BC229EC38EC48EC5EE30F94C0
:1092F00050CA20E030E040E05FE30F9456C90F947D
:10930000C9CA862F0D94BD1D2F923F924F925F9236
:109310006F927F928F929F92AF92BF92CF92DF9285
:10932000EF92FF920F931F93CF93DF9300D000D063
:109330001F921F92CDB7DEB720916D0F288761E095
:1093400081E00E94758D3091580F3F83E8858E2F04
:1093500090E0880F991F9C01275832493C832B834A
:1093600036E0E39FC0011124FC01E05CF04FFA837A
:10937000E9839C01225C304F79015F8035E0432E08
:10938000450C11E0312E3518252C2194FE82ED82FA
:10939000570134E0A30EB11C49E6C42E4DE8D42E8B
:1093A00085E0782E75184701E2E08E0E911C82E070
:1093B000682E6518FF81F1115BC01123D9F08091EF
:1093C000570F1816BCF04091530F5091540F6091F5
:1093D000550F7091560F4F5F5F4F6F4F7F4F409308
:1093E000530F5093540F6093550F7093560F8F5F28
:1093F0008093570F80918202882351F0EB81FC818A
:109400006591749130E020E043E0822D0E94C6997E
:10941000F501808180935B0FFF81F23009F07AC003
:10942000288520936D0F8091570F823009F45FC01B
:1094300080918202882391F011E08091570F823051
:1094400009F010E080915B0F0F94BD1D00E09C01BE
:1094500042EA59E0662D812F0E94FB9B10E02F818C
:109460002F5F2F832411A6CF86E08093510F19C060
:109470002F81213069F68091570F813031F0809132
:109480008202811127C010E0C3CF8091500F10924B
:10949000500F8823A1F30E94BB8E8091520F882326
:1094A00071F328960FB6F894DEBF0FBECDBFDF91E3
:1094B000CF911F910F91FF90EF90DF90CF90BF90D1
:1094C000AF909F908F907F906F905F904F903F9064
:1094D0002F90089581E09091570F913009F080E02E
:1094E00024E04CEA59E0632D0F94799ECCCF809113
:1094F000500F1092500F882309F49ACF65E878E353
:1095000082EA99E00F948BA28091520F882309F48C
:109510008FCFC7CF3F81333091F58091570F833084
:10952000C1F080918202882309F498CF11E08091E4
:10953000570F833009F010E0ED81FE818081918129
:109540000F94881D63E0651900E09C014BE959E028
:1095500082CF8091500F1092500F882311F310E0AA
:1095600000E02CE231E045E050E0B7018BE999E002
:109570000F944CA18091520F882399F292CFFF81D2
:10958000F43091F58091570F8430B9F080918202C8
:10959000882309F463CF11E08091570F843009F0DC
:1095A00010E0F401808191810F94881D64E06519B9
:1095B00000E09C0147E959E04ECF8091500F109296
:1095C000500F882319F310E000E02CE830E045E06C
:1095D00050E069817A8187E999E00F944CA18091EC
:1095E000520F882399F25DCFFF81F53009F037CF14
:1095F0008091570F8530E1F080918202882309F431
:109600002DCFDF92CF9289ED99E09F938F937F9238
:1096100081E09091570F953009F080E08F930E9480
:109620003F8D0F900F900F900F900F900F9016CFCF
:109630008091500F1092500F8823F1F20E94698D93
:109640008091520F8823C1F22CCF0D94E1A50D9487
:10965000E1A50F9404480E9413E60C94568E6FEF18
:1096600080915B0F0D94FFA34F925F926F927F9258
:109670008F929F92AF92BF92CF92DF92EF92FF9222
:109680000F931F93CF93DF9300915B0F61E081E015
:109690000E94758DC091580F10E0000F111F0758E0
:1096A000124995E0592E5C0E2AE9E22E20E1F22EB5
:1096B000D3E0DC1B3FE2C32E3BE4D32E4CE8A42EC8
:1096C00040E1B42E82E0782E7C1A5DEB852E50E1CD
:1096D000952E81E0682E6C1A4C2E4194C11137C032
:1096E0008091570F8823B1F080918202882359F02E
:1096F00081E09091570F911180E024E048EA50E119
:10970000642D0F94799ECF5F5C12E8CF84E0809344
:10971000510F0CC08091500F1092500F882321F3ED
:109720000E94BB8E8091520F8823F1F2DF91CF917E
:109730001F910F91FF90EF90DF90CF90BF90AF906F
:109740009F908F907F906F905F904F900895C13061
:1097500059F5F8018591949190936F0F80936E0F56
:109760008091570F813081F080918202882359F2D5
:109770001F929F928F926F9281E09091570F91303C
:1097800009F474C080E072C08091500F1092500FA5
:10979000882351F380915B0F682F0F94FFA3809172
:1097A000520F882309F3C2CFC23009F042C0F8013A
:1097B0008591949190936F0F80936E0F8091570FC6
:1097C0008230D1F080918202882309F49CCFDF920D
:1097D000CF92BF92AF927F9281E09091570F9230DB
:1097E00009F080E08F930E943F8D0F900F900F90B3
:1097F0000F900F900F9087CF8091500F1092500FC5
:10980000882301F30E942F4B8091520F8823D1F2BD
:109810008DCF8091500F1092500F8823C1F060912E
:109820005B0F8FEF0F94FFA38091520F882379F085
:109830007DCFC33009F067CFF80185919491909363
:109840006F0F80936E0F8091570F833011F38091CB
:109850008202882309F457CF1F92FF92EF92DF9381
:1098600081E09091570F933009F08CCF8F930E9435
:109870003F8D0F900F900F900F900F9044CF81E08D
:10988000809345078091F70E8770873051F01092D2
:10989000F70E1092260980E194E19093FB0E8093DD
:1098A000FA0E8091AA0F8093470780E00F94CF456E
:1098B00020E040E070E060E08BED98E50C94D38D03
:1098C0006AE77FE482E00D9476B36FE77FE481E09E
:1098D0000D9476B364E87FE480E00D9476B361E3A1
:1098E0007DE483E00D9476B3CF92DF92EF92FF9206
:1098F0000F931F938AECC82E8FE0D82EF12CE12C09
:109900000CEC1FE02BED30E04EE25CE36CED7FE011
:1099100081EE9FE00E94F6941F910F91FF90EF90CF
:10992000DF90CF900895CF92DF92EF92FF920F9346
:109930001F938DEBC82E8EE0D82EF12CE12C0DE676
:109940001FE02BED30E047E050E96FEB7EE084EC68
:109950009EE00E94F6941F910F91FF90EF90DF9090
:10996000CF900895CF92DF92EF92FF920F931F93C3
:10997000CF93DF9300D01F92CDB7DEB720916D0F4C
:109980001C821B8280E2898380E22A302CF0822FA5
:109990006AE00F9417C9805D8A83822F6AE00F9472
:1099A00017C9905D9B8387E4C82E89E0D82ECE012D
:1099B00001967C0109E419E02BED30E04DE358E518
:1099C00067E579E08AE599E00E94F6940F900F90A0
:1099D0000F900F90DF91CF911F910F91FF90EF901B
:1099E000DF90CF900895CF92DF92EF92FF920F9386
:1099F0001F9380E3C82E89E0D82EF12CE12C02E3DE
:109A000019E027E438E54FE558E56DE379E082E4B5
:109A100099E00E94F6941F910F91FF90EF90DF90D4
:109A2000CF900895CF92DF92EF92FF920F931F9302
:109A300085EAC82E88E0D82EF12CE12C08EB18E03E
:109A400030E020E04FE95EE867EA78E08EEA98E0EF
:109A50000E94F6941F910F91FF90EF90DF90CF90AE
:109A60000895CF93DF9300D01F92CDB7DEB78091DA
:109A7000500F1092500F882359F0109245070E9402
:109A8000BB8E0F900F900F900F90DF91CF910895A4
:109A90006091530F7091540F8091550F9091560F14
:109AA000611571058105910561F10F946BC22091DB
:109AB00011023091120240911302509114020F943E
:109AC000CAC22091A7103091A8104091A9105091BE
:109AD000AA100F9456C96093A7107093A810809392
:109AE000A9109093AA1083E00E94D69081E0809301
:109AF00082021092530F1092540F1092550F109231
:109B0000560F80918202882309F4BBCF20914A0F1F
:109B100030914B0F40914C0F50914D0F6091A71019
:109B20007091A8108091A9109091AA100F9455C916
:109B300069837A838B839C83CE0101960F94BF1B2C
:109B4000BC018BE59DE60E94519A9BCF2F923F92DC
:109B50004F925F926F927F928F929F92AF92BF923D
:109B6000CF92DF92EF92FF921F93CF93DF93CDB707
:109B7000DEB72C970FB6F894DEBF0FBECDBF1C0129
:109B8000162F8091500F1092500F8823E1F0109201
:109B900045070E94BB8E2C960FB6F894DEBF0FBE11
:109BA000CDBFDF91CF911F91FF90EF90DF90CF90CD
:109BB000BF90AF909F908F907F906F905F904F90ED
:109BC0003F902F9008958091530F9091540FA09142
:109BD000550FB091560F8D839E83AF83B887892B25
:109BE0008A2B8B2B09F460C080913B02882309F4F7
:109BF000BDC080913C028111B9C0613009F494C0AC
:109C0000623009F4A2C080903D0290903E02A09084
:109C10003F02B0904002C0904902D0904A02E090CA
:109C20004B02F0904C02612E712C6D817E818F81F0
:109C300098850F946BC220911102309112024091CD
:109C40001302509114020F94CAC2D301AA0FBB1F72
:109C5000AA0FBB1FBC87AB87A556BF4EBA87A98783
:109C60002D913D914D915C910F9456C92B013C0172
:109C70008D819E81AF81B885B7FF8FC0A50194010A
:109C8000C301B2010F9464C287FD7FC0EB85FC85E0
:109C9000E556FF4E4082518262827382812F0E947C
:109CA000D69081E0809382021092530F1092540F4D
:109CB0001092550F1092560F80918202882309F45A
:109CC0006ACFF4E01F9FC0011124FC01E556FF4E4E
:109CD00081579F4EDC012D913D914D915C916081AA
:109CE0007181828193810F9456C96B017C01C98275
:109CF000DA82EB82FC822DEC3CEC4CEC5DE3609173
:109D000011027091120280911302909114020F942B
:109D1000B6CB87FD52C0CE0101960F94BF1BBC018C
:109D2000C1010E94519A37CF809041029090420227
:109D3000A0904302B0904402C0904D02D0904E02D9
:109D4000E0904F02F09050026ECF809045029090CC
:109D50004602A0904702B0904802C0905102D090B5
:109D60005202E0905302F09054025DCF812C30E516
:109D7000932E33ECA32E37ECB32EC12C40E5D42E1A
:109D800043ECE42E47E4F42E4ECFA985BA858D929C
:109D90009D92AD92BC92139781CFA7019601C3010A
:109DA000B2010F94B6CB18160CF070CFE985FA8586
:109DB000C082D182E282F38271CF20E030E040E2C3
:109DC00051E4C701B6010F94CAC220E030E04AE76F
:109DD00054E40F94CAC24B015C0120E030E0A901B9
:109DE000C701B6010F9464C220E030E040EA50E4BD
:109DF00087FF04C020E030E040EA50ECC501B40128
:109E00000F9456C920E030E040E251E40F9450CA6C
:109E10000F94C2CA6B017C01F7FC62C020EA36E8ED
:109E200041E050E00F94CAC8CA01B9012AE030E00D
:109E300040E050E00F94CAC8605D6093640FC701B2
:109E4000B60120E137E240E050E00F94CAC88AE052
:109E5000882E912CA12CB12CCA01B901A501940125
:109E60000F94CAC8605D6093650FC701B60128EE04
:109E700033E040E050E00F94CAC8CA01B901A5011F
:109E800094010F94CAC8605D6093660F8EE2809360
:109E9000670FC701B60124E630E040E050E00F94C0
:109EA000CAC8CA01B901A50194010F94CAC8605D6E
:109EB0006093680FC701B601A50194010F94CAC849
:109EC000162FCA01B901A50194010F94CAC8605D9B
:109ED0006093690F105D10936A0F84E69FE01FCFB7
:109EE000F094E094D094C094C11CD11CE11CF11CEE
:109EF0006DE2A3CF62E084E69DE60C94A64D61E09E
:109F00008BE69DE60C94A64D60E082E79DE60C94FE
:109F1000A64DCF92DF92EF92FF92CF93DF9300D0C6
:109F20001F92CDB7DEB76B017C0120E030E0A901C4
:109F30000F9464C287FD1BC06DEB77E386E095E369
:109F4000A70196010F9456C969837A838B839C83FA
:109F5000CE0101960F94BF1B0F900F900F900F90A2
:109F6000DF91CF91FF90EF90DF90CF9008956DEB50
:109F700077E386E095EBE4CF0F946BC220E030E00E
:109F800040E251E40F9450CA20E030E0A9010F9460
:109F900056C90C94894FAF92BF92CF92DF92EF9245
:109FA000FF920F931F93CF93DF93CDB7DEB7ADB67C
:109FB000BEB680915B1A62E77FE0882311F06BE503
:109FC0007AE1FB0101900020E9F7CF01861B970B96
:109FD00001962DB73EB7281B390B0FB6F8943EBF3C
:109FE0000FBE2DBF8DB79EB701967C0180E2EDB705
:109FF000FEB78183C70101960F9409CE80E9C82E70
:10A000008FE0D82E02E91FE02BED30E04EE150E565
:10A010006EE97FE085EA9FE00E94F6940FB6F8941F
:10A02000BEBE0FBEADBEDF91CF911F910F91FF90CD
:10A03000EF90DF90CF90BF90AF90089582E79FE0C0
:10A040000E9483DB0E94568E80E00C9423903F9206
:10A050004F925F926F927F928F929F92AF92BF9238
:10A06000CF92DF92EF92FF920F931F93CF93DF93E4
:10A0700061E081E00E94758DC091580F3C2E85E013
:10A08000482E4C0E9EE6C92E9EE0D92E03EA1EE015
:10A09000D4E0DC1B2DE3A22E2EE0B22E38E8E32E16
:10A0A0003EE0F32E83E0782E7C1A4EE0842E4EE0C4
:10A0B000942E82E0682E6C1A81E0582E5C1AC11131
:10A0C00039C08091570F8823B9F08091820288238C
:10A0D00061F0632D619581E09091570F911180E0BF
:10A0E00024E048EB5EE00F94799ECF5FC411E7CF88
:10A0F00085E08093510F0CC08091500F1092500F4B
:10A10000882319F30E94BB8E8091520F8823E9F2B5
:10A11000DF91CF911F910F91FF90EF90DF90CF9043
:10A12000BF90AF909F908F907F906F905F904F9077
:10A130003F900895C13051F58091570F813089F0DB
:10A1400080918202882389F21F9282EB9EE09F9386
:10A150008F935F9281E09091570F913071F180E081
:10A160002CC08091500F1092500F882349F386E93C
:10A170009DE09093FB0E8093FA0E0E94548D0E94F6
:10A18000568E8091520F8823D9F2C2CFC23009F087
:10A190006AC08091570F8230C9F080918202882373
:10A1A00009F4A3CF1F928AE99EE09F938F936F9249
:10A1B00081E09091570F923091F68F930E943F8DDE
:10A1C0000F900F900F900F900F908FCF8091500FA6
:10A1D0001092500F882309F39092FB0E8092FA0E92
:10A1E0000E94548D0E94568E8091520F8823A9F2AE
:10A1F0008FCF8091570F833081F080918202882326
:10A2000009F473CF1F92FF92EF927F9281E09091B9
:10A21000570F933009F0A3CFD0CF8091500F1092F9
:10A22000500F882351F3B092FB0EA092FA0E0E94B9
:10A23000548D0E94568E8091520F8823F1F268CF80
:10A240008091500F1092500F8823B1F0D092FB0EE6
:10A25000C092FA0E0E94548D0E94568E8091520F29
:10A26000882351F055CFC33021F2C43009F03DCFDF
:10A270008091570F843021F380918202882309F462
:10A2800034CF1F921F930F93DF9381E09091570F6C
:10A29000943009F064CF91CF0F94B03A0F9470B11D
:10A2A00081E08093251E0F94B2B10C94568E6F926C
:10A2B0007F928F929F92AF92BF92CF92DF92EF9256
:10A2C000FF920F931F93CF93DF9381E08093450715
:10A2D00061E00E94758DC091580F85E0882E8C0E2C
:10A2E000D1E00CE411E591E7E92E9DE0F92E82E042
:10A2F000982E9C1A23E6C22E28E3D22E3CE7A32EEA
:10A300003DE0B32E7D2E7C1A6C2E6194C11130C0BD
:10A31000DD23D9F08091570F1816BCF04091530FF0
:10A320005091540F6091550F7091560F4F5F5F4FD2
:10A330006F4F7F4F4093530F5093540F6093550FBF
:10A340007093560F8F5F8093570F809182028823FE
:10A3500041F030E020E041E069E87DE0862D0E9498
:10A36000C699CF5F8C12D2CF83E08093510F23C068
:10A37000C13081F58091570F813089F08091820240
:10A38000882309F444C0DF92CF92BF92AF927F92AC
:10A3900081E09091570F913089F180E02FC080913A
:10A3A000500F1092500F882349F30E946338809118
:10A3B000520F882319F3DF91CF911F910F91FF90D6
:10A3C000EF90DF90CF90BF90AF909F908F907F9055
:10A3D0006F900895C23029F68091570F8230C9F0EE
:10A3E00080918202882399F01F930F93FF92EF923E
:10A3F0009F9281E09091570F923079F68F930E944F
:10A400003F8D0F900F900F900F900F900F90D0E016
:10A41000A8CF8091500F1092500F882309F30E940B
:10A420004C518091520F8823D9F2C5CFEF92FF9201
:10A430000F931F93CF93DF93CDB7DEB765970FB61A
:10A44000F894DEBF0FBECDBF8091500F1092500F19
:10A45000882379F00E94BB8E65960FB6F894DEBF14
:10A460000FBECDBFDF91CF911F910F91FF90EF9065
:10A47000089560E085E00E94758D0091580F10E00E
:10A480008AE3F82E90E2E92E011130C08091820219
:10A49000882341F030E020E043E06DE27DE0812F51
:10A4A0000E94C699F982EA8242E150E067EF7CE0BF
:10A4B000CE0103960F9495C18C8987FD1C8A0530C7
:10A4C000C1F580918202882349F09E012F5F3F4FA2
:10A4D00041E06DEE7CE0812F0E94C6990F5F1F5F07
:10A4E000153091F687E08093510FB6CF013051F4CB
:10A4F000809182028823B1F230E020E041E061E205
:10A500007DE0CDCF023009F580918202882351F29F
:10A5100030E020E041E066E17DE0C1CF8091820241
:10A52000882309F4BFCF30E020E041E06CE07DE01B
:10A53000B6CF063099F680918202882379F230E016
:10A5400020E041E068ED7CE0C6CF033039F3043011
:10A5500009F0A8CF80918202882309F4A3CF30E0CC
:10A5600020E041E069EF7CE09ACFEF92FF920F93F9
:10A570001F93CF93DF93CDB7DEB765970FB6F894EF
:10A58000DEBF0FBECDBF8091500F1092500F8823B9
:10A5900079F00E94BB8E65960FB6F894DEBF0FBEB1
:10A5A000CDBFDF91CF911F910F91FF90EF90089554
:10A5B00060E085E00E94758D0091580F10E08AE3FD
:10A5C000F82E90E2E92E01110CC0809182028823BE
:10A5D00041F030E020E043E067EC7CE0812F0E9416
:10A5E000C699F982EA8242E150E060EC7CE0CE015B
:10A5F00003960F9495C18C8987FD1C8A013069F4FC
:10A6000080918202882349F09E012F5F3F4F41E0F5
:10A610006BEB7CE0812F0E94C699F982EA8242E1CD
:10A6200050E067EB7CE0CE0103960F9495C18C89D6
:10A6300087FD1C8A023069F480918202882349F0E8
:10A640009E012F5F3F4F41E06EEA7CE0812F0E9428
:10A65000C699F982EA8242E150E066EA7CE0CE01E6
:10A6600003960F9495C18C8987FD1C8A033069F489
:10A6700080918202882349F09E012F5F3F4F41E085
:10A6800062EA7CE0812F0E94C6990F5F1F5F153040
:10A6900009F099CF84E08093510F7DCFEF92FF9224
:10A6A0000F931F93CF93DF93CDB7DEB765970FB6A8
:10A6B000F894DEBF0FBECDBF8091500F1092500FA7
:10A6C000882379F00E94BB8E65960FB6F894DEBFA2
:10A6D0000FBECDBFDF91CF911F910F91FF90EF90F3
:10A6E000089560E085E00E94758D0091580F10E09C
:10A6F0008AE3F82E90E2E92E01110CC080918202CB
:10A70000882341F030E020E042E063E97CE0812FE3
:10A710000E94C699F982EA8242E150E061E97CE058
:10A72000CE0103960F9495C18C8987FD1C8A013058
:10A7300069F480918202882349F09E012F5F3F4F88
:10A7400040E068E87CE0812F0E94C699F982EA82A5
:10A7500042E150E064E87CE0CE0103960F9495C19D
:10A760008C8987FD1C8A023009F04EC080918202DC
:10A77000882349F09E012F5F3F4F40E06BE77CE06C
:10A78000812F0E94C699F982EA8242E150E066E593
:10A790007CE0CE0103960F9495C18C8987FD1C8ABD
:10A7A000053069F480918202882349F09E012F5F71
:10A7B0003F4F40E068E87CE0812F0E94C699F98213
:10A7C000EA8242E150E062E57CE0CE0103960F941C
:10A7D00095C18C8987FD1C8A063089F5809182029B
:10A7E000882349F09E012F5F3F4F40E06BE77CE0FC
:10A7F000812F0E94C6990F5F1F5F153009F07CCF33
:10A8000088E08093510F60CF033059F48091820229
:10A81000882309F4B8CF30E020E040E069E67CE02E
:10A82000AFCF043009F0AFCF80918202882309F4C2
:10A83000AACF30E020E042E068E57CE0A1CF07301D
:10A84000D1F6809182028823B1F230E020E040E02E
:10A8500069E67CE0CDCF2F923F924F925F926F924C
:10A860007F928F929F92AF92BF92CF92DF92EF92A0
:10A87000FF920F931F93CF93DF93CDB7DEB7E2978D
:10A880000FB6F894DEBF0FBECDBF8091500F10926F
:10A89000500F8823D9F00E94BB8EE2960FB6F89431
:10A8A000DEBF0FBECDBFDF91CF911F910F91FF9003
:10A8B000EF90DF90CF90BF90AF909F908F907F9060
:10A8C0006F905F904F903F902F9008958091E40E8D
:10A8D0009091E50E9CA78BA7A091E60EB091E70E94
:10A8E000BEA7ADA74090E80E5090E90E6090EA0E2A
:10A8F0007090EB0E8091EC0E9091ED0EA091EE0E0B
:10A90000B091EF0E8FA798ABA9ABBAAB8090F00EC9
:10A910009090F10EA090F20EB090F30E60E085E002
:10A920000E94758D0091580F10E0DE0156967D0152
:10A930008AE0C82ED12C97EF292E9BE0392E6FE4A8
:10A940007CE0CE0101960F946DC18BA59CA50F9460
:10A950005D1DBC01CE0103960F9409CE01110DC0FF
:10A9600080918202882349F09E012F5F3F4F40E093
:10A9700063E47CE0812F0E94C69960E47CE0CE0114
:10A9800001960F946DC18DA59EA50F945D1DBC0110
:10A99000CE0103960F9409CE013009F04CC080918E
:10A9A0008202882349F09E012F5F3F4F40E066E31B
:10A9B0007CE0812F0E94C69920E030E048EC52E410
:10A9C000C501B4010F9450CA0F94C2CACB01B6019D
:10A9D0000F9439C99F938F9320E030E04AE754E405
:10A9E000C501B4010F9450CA0F94C2CA9F938F93AC
:10A9F0007F936F933F922F92FF92EF920F94FBC140
:10AA00000FB6F894DEBF0FBECDBF073059F480916A
:10AA10008202882339F0970140E064EF7BE0812FC8
:10AA20000E94C6990F5F1F5F153009F088CF88E03C
:10AA30008093510F32CF023059F4809182028823E3
:10AA400009F4BACF30E020E040E065E27CE0B1CF2D
:10AA5000033099F480918202882309F4ADCF4982B2
:10AA60005A826B827C82B701CE0101960E947CA53E
:10AA70009C0140E062E27CE09CCF043009F04CC0D5
:10AA800080918202882341F030E020E040E061E1E3
:10AA90007CE0812F0E94C69920E030E048EC52E42F
:10AAA000C501B4010F9450CA0F94C2CACB01B601BC
:10AAB0000F9439C99F938F9320E030E04AE754E424
:10AAC000C501B4010F9450CA0F94C2CA9F938F93CB
:10AAD0007F936F933F922F92FF92EF920F94FBC15F
:10AAE0000FB6F894DEBF0FBECDBF9CCF809182021F
:10AAF000882391F28FA598A9A9A9BAA989839A83D5
:10AB0000AB83BC83B701CE0101960E947CA59C015A
:10AB100040E06EE07CE04DCF053041F3063009F0B7
:10AB20004BCF80918202882309F4B6CF30E020E039
:10AB300040E06FEF7BE03DCF2F923F924F925F92CC
:10AB40006F927F928F929F92AF92BF92CF92DF923D
:10AB5000EF92FF920F931F93CF93DF934C010F94CB
:10AB600074C101968401080F191FC8010F9474C1A4
:10AB700001966801C80ED91EF8016080C1E061101D
:10AB800001C0C0E0F6013080D1E0311001C0D0E05A
:10AB9000AA24A3946110A12C60E085E00E94758D29
:10ABA0005090580F752C9EE0E92EF12C252C219405
:10ABB0008A2D90E001965C01AC0EB11CAD0EB11C6B
:10ABC00071101DC0809182028823A1F0E0910502DE
:10ABD000E2506EEB7AE0E33038F4F0E0EE0FFF1F66
:10ABE000E054FD4F6081718130E020E043E0822D30
:10ABF0000E94C699D1E0611013C0D2E011C0D2E02A
:10AC00006110D1E0D7110CC080918202882341F0FD
:10AC100030E020E041E0B4018D2F85190E94C699F3
:10AC2000C1E0CD0F472C4518662079F0C7110BC045
:10AC300080918202882339F030E020E041E0B801C1
:10AC4000842D0E94C699C2E0CD0F332071F0C71148
:10AC50000BC080918202882339F030E020E041E08F
:10AC6000B601842D0E94C699CF5FF3E0AF16B10400
:10AC70000CF4CF5FC71162C080918202882309F46F
:10AC80005AC030E020E042E06BEC7AE0842D0E9474
:10AC9000C699D0913F0793EF9E0D90933E078EEF9C
:10ACA0008E0D80936C0F20911D1E2E151F0411F028
:10ACB0000CF041C020911F1E9217E8F59EE390937F
:10ACC000201E8093211E65E470E080E090E00E94E9
:10ACD000B59361E36D0F062E000C770B880B990B73
:10ACE0000E94B59360E270E080E090E00E94B5932E
:10ACF00080910D1D90910E1D0F94881D0E944D9AFC
:10AD00006FE270E080E090E00E94B5930E94359180
:10AD1000811109C085E08D9FF0011124EF52F34F9E
:10AD20008481811108C080910F1D9091101D0F9496
:10AD3000881D0E944D9A92E090938202ECE0EE0E04
:10AD4000F11C7394FAE4EF16F10409F039CFCF5FE8
:10AD5000C093510FDF91CF911F910F91FF90EF9012
:10AD6000DF90CF90BF90AF909F908F907F906F902B
:10AD70005F904F903F902F90089586ED9AE00C944D
:10AD80009C5583EE9AE00C949C5585E09BE00C94D6
:10AD90009C5580EA9BE00C949C558BE59BE00C94C1
:10ADA0009C5588E89BE00C949C558BED9BE00C94A3
:10ADB0009C558EEB9BE00C949C558EE39BE00C9491
:10ADC0009C558FE19BE00C949C5584E00D94CFA2A0
:10ADD00083E00D94CFA282E00D94CFA2CF93DF93B6
:10ADE00000D01F92CDB7DEB784EF91E0A0E0B0E0D5
:10ADF00089839A83AB83BC83BE016F5F7F4F88E7F3
:10AE00000F9460490F900F900F900F90DF91CF91AA
:10AE100008956F927F928F929F92AF92BF92CF923E
:10AE2000DF92EF92FF920F931F93CF93DF9361E036
:10AE300081E00E94758DC091580F6C2E85E0782EB0
:10AE40007C0E99E9E92E91E0F92E28E7C22E29E03F
:10AE5000D22ED5E0DC1B39E0A32E32E0B32E14E075
:10AE60001C1B03E00C1B82E0982E9C1A81E0882EAC
:10AE70008C1AC11136C08091570F8823B9F0809188
:10AE80008202882361F0662D619581E09091570FD1
:10AE9000911180E024E04CEA59E00F94799ECF5F55
:10AEA000C711E7CF86E08093510F0CC08091500FFF
:10AEB0001092500F882319F30E94BB8E8091520F7D
:10AEC0008823E9F2DF91CF911F910F91FF90EF90CE
:10AED000DF90CF90BF90AF909F908F907F906F90BA
:10AEE0000895C13029F58091570F8130A1F08091EC
:10AEF00082028823A1F28BEE91E09F938F9381E9E8
:10AF000099E09F938F938F9281E09091570F9130AA
:10AF100049F180E027C08091500F1092500F882394
:10AF200031F30F94D1498091520F882301F3CACF96
:10AF3000C23009F085C08091570F8230E9F08091CE
:10AF40008202882309F4ABCF8EEE96E59F938F9310
:10AF500087E899E09F938F939F9281E09091570F9C
:10AF60009230B9F68F930E943F8D0F900F900F9003
:10AF70000F900F900F9093CF8091500F1092500F21
:10AF80008823E9F20E94EE568091520F8823B9F28D
:10AF900099CF8091570F8330A9F080918202882346
:10AFA00009F47DCF8BEC91E09F938F9380E899E03B
:10AFB0009F938F930F9381E09091570F933009F0F7
:10AFC000A8CFD0CF8091500F1092500F882329F333
:10AFD0000F949B498091520F8823F9F273CF80918F
:10AFE000570F843099F080918202882309F457CF5B
:10AFF000BF92AF9283E799E09F938F931F9381E075
:10B000009091570F943009F084CFACCF8091500FBE
:10B010001092500F882339F30F9480498091520F7A
:10B02000882309F34FCF8091500F1092500F88233F
:10B0300099F00F94B6498091520F882369F042CF5E
:10B04000C33009F4A6CFC43051F2C53009F027CF80
:10B050008091570F853039F380918202882309F45B
:10B060001ECFFF92EF92DF92CF92DF9381E090911B
:10B07000570F953009F04DCF75CF80916D0F80320D
:10B0800010F40F94533B0E94548D0C94BB8E80E0BF
:10B0900090E0A0E8B0E48093A3109093A410A09354
:10B0A000A510B093A61088EB92E00F949B0C8091B2
:10B0B00047070F94CF45109245070C94BB8E80E054
:10B0C00090E0A0E8B0E48093A3109093A410A09324
:10B0D000A510B093A61088EB92E00F949B0CE09122
:10B0E000460780E090E0AAE7B3E4E43009F44AC000
:10B0F00080E090E0A0EBB1E480939B1090939C10D3
:10B10000A0939D10B0939E1080939F109093A010D9
:10B11000A093A110B093A210EE0FFF0BE856FD4FC5
:10B12000808191818330910549F184309105D9F175
:10B13000029761F480E090E0AFEEB3E480939B105F
:10B1400090939C10A0939D10B0939E1080EA92E083
:10B150000F949B0C1092A3101092A4101092A510A3
:10B160001092A61088EB92E00F949B0C80914607FA
:10B170008F5F8530ECF480934607089580E090E07F
:10B18000AFEEB3E480939B1090939C10A0939D101E
:10B19000B0939E1080939F109093A010A093A11045
:10B1A000B093A210D3CF80E090E0AFEEB3E4F2CF43
:10B1B00010924607089580918202882341F030E082
:10B1C00020E041E065E074E182E00E94C699809150
:10B1D00026098770873079F41092460720E040E016
:10B1E00070E060E083EF9CE40E94D38D81E0809367
:10B1F00038070C945F580895CF93DF9300D01F92C7
:10B20000CDB7DEB70F94C9CA0F9469C269837A8338
:10B210008B839C83CE0101960F943C1B0F900F9063
:10B220000F900F90DF91CF9108950F946BC22AE099
:10B2300037ED43E25DE30F9450CA20E030E0A9010E
:10B240000F9456C90C94FC58CF92DF92EF92FF9264
:10B25000CF93DF9300D01F92CDB7DEB76B017C0197
:10B2600020E030E0A9010F9464C287FD1BC06DEBA4
:10B2700077E386E095E3A70196010F9456C96983A9
:10B280007A838B839C83CE0101960F943C1B0F9095
:10B290000F900F900F90DF91CF91FF90EF90DF9084
:10B2A000CF9008956DEB77E386E095EBE4CF0F94B4
:10B2B0006BC22AE037ED43E25DE30F9450CA20E011
:10B2C00030E0A9010F9456C90C9424590F946BC215
:10B2D00020E030E0A9010F9456C90C9424597F92C4
:10B2E0008F929F92AF92BF92CF92DF92EF92FF9296
:10B2F0000F931F93CF93DF9361E081E00E94758DE0
:10B30000C091580F65E0862E8C0ED6E0DC1B85E0E0
:10B31000D82EDC1A84E0C82ECC1A83E0B82EBC1AD2
:10B3200082E0A82EAC1A81E0982E9C1A7C2E719493
:10B33000C11134C08091570F8823B1F080918202EF
:10B34000882359F081E09091570F911180E024E01B
:10B3500043E958E0672D0F94799ECF5FC811E8CF7D
:10B3600087E08093510F0CC08091500F1092500FC6
:10B37000882321F30E94BB8E8091520F8823F1F223
:10B38000DF91CF911F910F91FF90EF90DF90CF90C1
:10B39000BF90AF909F908F907F900895C130E9F556
:10B3A0008091570F8130E9F0809182028823A9F2C1
:10B3B00011E08091570F813009F010E06091C117C2
:10B3C0007091C2178091C3179091C4170E9424599D
:10B3D00000E09C014EED57E0692D812F0E94FB9B00
:10B3E000BCCF8091500F1092500F8823E9F20F9438
:10B3F000D49FE12C1CE3F12E0CE116E420E030E0B8
:10B4000040E85FE361EC77E18EED97E00F94E09F19
:10B410008091520F882341F2B3CFC23009F006C1A8
:10B420008091570F8230D9F080918202882309F4ED
:10B4300094CF11E08091570F823009F010E06091B5
:10B44000C5177091C6178091C7179091C8170E94B1
:10B45000245900E09C0147ED57E06A2DBECF809152
:10B46000500F1092500F8823F9F20F94D49FE12CC3
:10B470001CE3F12E0CE116E420E030E040E85FE34D
:10B4800065EC77E187ED97E00F94E09F8091520F94
:10B49000882351F275CF8091570F8330D9F0809176
:10B4A0008202882309F459CF11E08091570F83302D
:10B4B00009F010E06091C9177091CA178091CB17FD
:10B4C0009091CC170E94245900E09C0140ED57E078
:10B4D0006B2D83CF8091500F1092500F8823F9F27B
:10B4E0000F94D49FE12C1CE3F12E0CE116E420E034
:10B4F00030E040E85FE369EC77E180ED97E00F949E
:10B50000E09F8091520F882351F23ACF8091570FDC
:10B510008430D9F080918202882309F41ECF11E093
:10B520008091570F843009F010E06091CD17709131
:10B53000CE178091CF179091D0170E94245900E028
:10B540009C0149EC57E06C2D48CF8091500F109230
:10B55000500F8823F9F20F94D49FE12C1CE3F12EB5
:10B560000CE116E420E030E040E85FE36DEC77E1C9
:10B5700089EC97E00F94E09F8091520F882351F25D
:10B58000FFCE8091570F8530D9F0809182028823B9
:10B5900009F4E3CE11E08091570F853009F010E0F7
:10B5A0006091DD177091DE178091DF179091E017A1
:10B5B0000E94245900E09C0144EC57E06D2D0DCF12
:10B5C0008091500F1092500F8823F9F20F94D49F5E
:10B5D000E12C1CE3F12E0CE116E420E030E0A9019F
:10B5E0006DED77E184EC97E00F94E09F8091520F2E
:10B5F000882359F2C5CE8091500F1092500F8823A6
:10B6000029F10F94D49FE12C1CE3F12E0CE116E4F8
:10B6100020E030E0A90161EE77E18AEB97E00F943A
:10B62000E09F8091520F882389F0AACEC33009F49D
:10B6300032CFC43009F46ACFC53009F4A2CFC63086
:10B6400009F08BCE8091570F8630A9F2809182024B
:10B65000882309F482CE11E08091570F863009F0DB
:10B6600010E06091E1177091E2178091E3179091DB
:10B67000E4170E94245900E09C014AEB57E06D2F2B
:10B68000ACCE2F923F924F925F926F927F928F92A9
:10B690009F92AF92BF92CF92DF92EF92FF920F9361
:10B6A0001F93CF93DF93CDB7DEB72C970FB6F894E7
:10B6B000DEBF0FBECDBFC090A117D090A217E09003
:10B6C000A317F090A4178091A5179091A617A091A9
:10B6D000A717B091A8178C159D05AE05BF0510F4EE
:10B6E000D701C601C0909D17D0909E17E0909F177C
:10B6F000F090A017BC01CD016C157D058E059F054E
:10B7000010F4C701B6010F9469C22B013C0161E03E
:10B7100081E00E94758D2091580F2B872E83822FF8
:10B720008B5F8D8387E0922F821B8F8386E0821B45
:10B73000888785E0821B898784E0821B8A8783E073
:10B74000282E221A82E0382E321A91959C872B855A
:10B75000211142C08091570F8823C9F08091820245
:10B76000882359F081E09091570F911180E024E0F7
:10B7700043E958E06C850F94799E8B858F5F8B87AA
:10B780009D819813E4CF88E08093510F0CC0809185
:10B79000500F1092500F882309F30E94BB8E8091A6
:10B7A000520F8823D9F22C960FB6F894DEBF0FBE45
:10B7B000CDBFDF91CF911F910F91FF90EF90DF9060
:10B7C000CF90BF90AF909F908F907F906F905F9041
:10B7D0004F903F902F9008958B85813009F08BC05A
:10B7E0008091570F8130F9F080918202882329F2ED
:10B7F00011E08091570F813009F010E06091D1176E
:10B800007091D2178091D3179091D4170E94245928
:10B8100061E02E81621B00E09C0144E158E0812F31
:10B820000E94FB9BAACF8091500F1092500F88234B
:10B83000D9F20F94D49F2AE037ED43E25DE3C301D0
:10B84000B2010F94CAC220E030E0A9010F9456C99A
:10B850004B015C0120E030E040E05FE40F9464C203
:10B8600087FD05C0812C912CA12C3FE4B32E2AE04A
:10B8700037ED43E25DE36091D1177091D21780916B
:10B88000D3179091D4170F94CAC220E030E0A901D9
:10B890000F9456C920E030E040E85FE30F9455C9AB
:10B8A0000F94C9CA69837A838B839C83C501B401D1
:10B8B0000F94C2CA7B018C0121E0E21AF108010950
:10B8C00011091F92912C812C28E9A22E20E4B22E7E
:10B8D000C980DA8021E030E040E050E061ED77E1BE
:10B8E00084E198E00E94F98E0F908091520F882396
:10B8F00009F47ACF58CF8B85823009F090C18091BE
:10B90000570F8230D9F080918202882309F435CF15
:10B9100011E08091570F823009F010E06091D51747
:10B920007091D6178091D7179091D8170E942459FB
:10B9300000E09C014AE058E0632D71CF8091500FE8
:10B940001092500F8823F9F20F94D49F6091A91799
:10B950007091AA178091AB179091AC170F9469C2A0
:10B960007B018C0120E030E048EC52E465ED77E1AA
:10B970008AE098E00F94E09F8091520F882319F29B
:10B9800012CF8091570F8330D9F0809182028823A3
:10B9900009F4F3CE11E08091570F833009F010E0E5
:10B9A0006091D9177091DA178091DB179091DC17AD
:10B9B0000E94245900E09C0141E058E0622D2FCF05
:10B9C0008091500F1092500F8823F9F20F94D49F5A
:10B9D0002AE037ED43E25DE3C301B2010F94CAC22E
:10B9E00020E030E0A9010F9456C94B015C0120E032
:10B9F00030E040E05FE40F9464C287FD05C0812C15
:10BA0000912CA12C9FE4B92E2AE037ED43E25DE3AF
:10BA10006091D9177091DA178091DB179091DC173C
:10BA20000F94CAC220E030E0A9010F9456C920E06B
:10BA300030E040E85FE30F9455C90F94C9CA6983A9
:10BA40007A838B839C83C501B4010F94C2CA7B01A6
:10BA50008C0121E0E21AF108010911091F92912CD1
:10BA6000812C88E9A82E80E4B82EC980DA8021E0F4
:10BA700030E040E050E069ED77E181E098E00E943D
:10BA8000F98E0F908091520F882309F47ECF8BCED0
:10BA90008091570F8430E9F080918202882309F465
:10BAA0006CCE11E08091570F843009F010E0609166
:10BAB0009D1770919E1780919F179091A0170F94DA
:10BAC00069C20E94FC5800E09C014AEF57E06A8579
:10BAD000A6CE8091500F1092500F8823E9F20F9458
:10BAE000D49F0FE71FE524E630E040E050E06DE929
:10BAF00077E18AEF97E00F947EA08091520F882320
:10BB000059F251CE8091570F8530E9F08091820231
:10BB1000882309F432CE11E08091570F853009F067
:10BB200010E06091A1177091A2178091A3179091D6
:10BB3000A4170F9469C20E94FC5800E09C0143EFD7
:10BB400057E069856CCE8091500F1092500F88237A
:10BB5000E9F20F94D49F0DE71FE524E630E040E0C2
:10BB600050E061EA77E183EF97E00F947EA0809147
:10BB7000520F882359F217CE8091570F8630E9F083
:10BB800080918202882309F4F8CD11E08091570F4B
:10BB9000863009F010E06091A5177091A61780918A
:10BBA000A7179091A8170F9469C20E94FC5800E053
:10BBB0009C014CEE57E0688532CE8091500F109278
:10BBC000500F8823E9F20F94D49F0BE71FE52AE07A
:10BBD00030E040E050E065EA77E18CEE97E00F94CA
:10BBE0007EA08091520F882359F2DDCD8091500FB5
:10BBF0001092500F882339F10F94D49F09E71FE565
:10BC000024E630E040E050E069EA77E185EE97E035
:10BC10000F947EA08091520F8823A9F0C4CD2B856C
:10BC2000233009F4AECE243009F432CF253009F4A4
:10BC300069CF263009F4A0CF273009F09ECD80913E
:10BC4000570F873099F280918202882309F495CDAD
:10BC500011E08091570F873009F010E06091A9172B
:10BC60007091AA178091AB179091AC170F9469C28D
:10BC70000E94FC5800E09C0145EE57E06F81CFCD5B
:10BC8000BF92CF92DF92EF92FF920F931F93CF93C9
:10BC9000DF9361E081E00E94758DC091580F85E0CF
:10BCA000C82ECC0ED4E0DC1B13E01C1B82E0F82E67
:10BCB000FC1A81E0E82EEC1ABC2EB194C11130C000
:10BCC0008091570F8823B1F080918202882359F028
:10BCD00081E09091570F911180E024E043E958E012
:10BCE0006B2D0F94799ECF5FCC11E8CF85E08093C8
:10BCF000510F0CC08091500F1092500F882321F3E8
:10BD00000E94BB8E8091520F8823F1F2DF91CF9178
:10BD10001F910F91FF90EF90DF90CF90BF9008950B
:10BD2000C130B9F58091570F8130F1F080918202D6
:10BD30008823C9F2DD24D3948091570F813009F014
:10BD4000D12C6091B1177091B2178091B317909177
:10BD5000B4170E94CA3900E09C0148E858E06E2DF3
:10BD60008D2D0E94FB9BBFCF8091500F1092500FE2
:10BD70008823E1F20F94D49F47E75FE561EB77E119
:10BD800088E898E00F9400A18091520F882371F207
:10BD9000BDCFC23009F07FC08091570F8230E1F0F3
:10BDA00080918202882309F49ECFDD24D394809170
:10BDB000570F823009F0D12C6091B5177091B617EA
:10BDC0008091B7179091B8170E94CA3900E09C0182
:10BDD0004DE758E06F2DC4CF8091500F1092500F57
:10BDE0008823F1F20F94D49F45E75FE565EB77E197
:10BDF0008DE798E00F9400A18091520F882381F283
:10BE000085CF8091570F8330E1F0809182028823A3
:10BE100009F469CFDD24D3948091570F833009F062
:10BE2000D12C6091B9177091BA178091BB1790917E
:10BE3000BC170E94CA3900E09C0142E758E0612F1C
:10BE40008FCF8091500F1092500F8823F1F20F94F2
:10BE5000D49F43E75FE569EB77E182E798E00F94D1
:10BE600000A18091520F882381F250CF8091500F12
:10BE70001092500F8823C9F00F94D49F41E75FE5DB
:10BE80006DEB77E187E698E00F9400A18091520F67
:10BE9000882359F03BCFC33009F4B3CFC43009F045
:10BEA00022CF8091570F843009F38091820288233A
:10BEB00009F419CFDD24D3948091570F843009F011
:10BEC000D12C6091BD177091BE178091BF179091D2
:10BED000C0170E94CA3900E09C0147E658E06D2F68
:10BEE0003FCF0C943BEE0C943BEE0C943BEE0C9449
:10BEF0003BEE0C94EDED0C94EDED0C94EDED0C940B
:10BF0000EDED8FEF0C945E8E80916D0F0C945E8E34
:10BF1000EF92FF920F931F93CF93DF9300D000D047
:10BF200000D01F921F92CDB7DEB77C012091590F30
:10BF3000422F022E000C550B80915A0F833079F15D
:10BF4000843031F180E59AE05F932F939F938F9334
:10BF50008E010F5F1F4F1F930F930F94FBC1C701FB
:10BF60000E94E1EDC8010E944D8D0F900F900F903F
:10BF70000F900F900F902B960FB6F894DEBF0FBE68
:10BF8000CDBFDF91CF911F910F91FF90EF9008955A
:10BF90008CE59AE027FDD8CF87E49AE0D5CF85E6F7
:10BFA0009AE0D2CFE0916D0F85E1E802F001112413
:10BFB000E75FF24E868197810C94885FE0916D0F68
:10BFC00086E0E802F0011124E25CF04F808191816B
:10BFD0000C94885F0F931F93CF93DF938C01EB0139
:10BFE0009091D11D2091D21D921305C00F94612014
:10BFF0000F94F30EF5CF8091D01D34E0839FF001B4
:10C000001124ED52F24E11830083D383C2839F5FCC
:10C010009093D11D8F5F281739F08093D01DDF9149
:10C02000CF911F910F9108951092D01DF8CFCF920C
:10C03000DF92EF92FF926B017C0120E030E0A901DA
:10C040000F9464C287FD26C06DEB77E386E095E32D
:10C05000A70196010F9456C96B017C0120E030E0E6
:10C06000A9010F9464C220E030E040E05FE387FF65
:10C0700004C020E030E040E05FEBC701B6010F9460
:10C0800056C90F94C2CACB01FF90EF90DF90CF90BA
:10C090000D94881D6DEB77E386E095EBD9CF0F9477
:10C0A0006BC220E030E0A9010F9456C90C941760D0
:10C0B0003F924F925F926F927F928F929F92AF9238
:10C0C000BF92CF92DF92EF92FF920F931F93CF9385
:10C0D000DF9361E081E00E94758DC091580FA5E06B
:10C0E0004A2E4C0ED4E0DC1B83E0782E7C1A82E0D2
:10C0F000682E6C1A81E0582E5C1A3C2E3194C111C6
:10C1000038C08091570F8823B1F080918202882334
:10C1100059F081E09091570F911180E024E043E9BC
:10C1200058E0632D0F94799ECF5FC411E8CF85E06E
:10C130008093510F0CC08091500F1092500F8823A4
:10C1400021F30E94BB8E8091520F8823F1F2DF9180
:10C15000CF911F910F91FF90EF90DF90CF90BF9004
:10C16000AF909F908F907F906F905F904F903F9097
:10C170000895C13009F05DC08091570F8130E9F01A
:10C1800080918202882381F211E08091570F8130E3
:10C1900009F010E06091C0107091C1108091C21040
:10C1A0009091C3100E94176000E09C0142E358E0A8
:10C1B000652D812F0E94FB9BB7CF8091500F10926D
:10C1C000500F8823E9F20F94D49F20E030E0A901BA
:10C1D0006091C0107091C1108091C2109091C310F5
:10C1E0000F9456C920E030E040E85FE30F9455C952
:10C1F0000F94C9CA1F92912C812CEAE7AE2EE0E47D
:10C20000BE2E6B011DEDE12E13E0F12E00E010E0DB
:10C2100021E030E040E050E060EC70E182E398E043
:10C220000E94F98E0F908091520F882309F4A8CFB5
:10C230008ECFC23009F0FEC08091570F8230D9F006
:10C2400080918202882309F46FCF11E08091570F0B
:10C25000823009F010E06091C4107091C510809197
:10C26000C6109091C7100E94176000E09C014AE23E
:10C2700058E0662D9ECF8091500F1092500F88236A
:10C28000F9F20F94D49F20E030E0A9016091C4102E
:10C290007091C5108091C6109091C7100F9456C927
:10C2A00020E030E040E85FE30F9455C90F94C9CA1D
:10C2B0001F92912C812C4AE7A42E40E4B42E6B01EE
:10C2C0001DEDE12E13E0F12E00E010E021E030E062
:10C2D00040E050E064EC70E18AE298E00E94F98E60
:10C2E0000F908091520F882309F4AACF30CF80910C
:10C2F000570F8330D9F080918202882309F414CF3C
:10C3000011E08091570F833009F010E06091C81060
:10C310007091C9108091CA109091CB100E949338EF
:10C3200000E09C0142E258E0672D43CF8091500F1E
:10C330001092500F8823F9F20F94D49F20E030E040
:10C3400048EC52E46091C8107091C9108091CA10F5
:10C350009091CB100F94CAC220E030E0A9010F9455
:10C3600056C920E030E040E251E40F9455C90F94E3
:10C37000C9CA1F92912C812C24EAA22E20E4B22E4D
:10C380006B011EEAE12E12E8F12E01E010E02AE036
:10C3900030E040E050E068EC70E182E298E00E941A
:10C3A000F98E0F908091520F882309F4A4CFCFCE3D
:10C3B0008091500F1092500F882309F446C00F94BB
:10C3C000D49F20E030E048EC52E46091CC107091B2
:10C3D000CD108091CE109091CF100F94CAC220E062
:10C3E00030E0A9010F9456C920E030E040E251E46A
:10C3F0000F9455C90F94C9CA1F92912C812C84EABD
:10C40000A82E80E4B82E6B011EEAE12E12E8F12E70
:10C4100001E010E02AE030E040E050E06CEC70E138
:10C420008AE198E00E94F98E0F908091520F882344
:10C4300061F08DCEC33009F45ACFC43009F074CE08
:10C440008091570F843009F4B3CF80918202882302
:10C4500009F46ACE11E08091570F843009F010E0A2
:10C460006091CC107091CD108091CE109091CF1032
:10C470000E94933800E09C014AE158E06D2F99CE6C
:10C48000CF93DF93EC010E94D28E20E040E070E079
:10C4900060E0CE01DF91CF910C94D38D2F923F922B
:10C4A0004F925F926F927F928F929F92AF92BF92C4
:10C4B000CF92DF92EF92FF920F931F93CF93DF9370
:10C4C00000D01F92CDB7DEB761E081E00E94758D8C
:10C4D0008091580F8B83282E8B5F8983922D9195A5
:10C4E0009A8388E0782E721887E0682E621886E0BA
:10C4F000582E521885E0482E421882E0382E321805
:10C5000081E082198C839B81911113C08091570F18
:10C51000882361F180918202882359F081E0909113
:10C52000570F911180E024E04BEE55E16A810F94A2
:10C53000799E8091AA0F882309F44DC08B818130A8
:10C5400009F06EC09091570F913099F1809182025D
:10C55000882309F4B2C081E0913009F080E020E244
:10C5600047ED55E16C810F94799EA7C08091500FE3
:10C570001092500F882371F20E94BB8E8091520F4F
:10C58000882341F20F900F900F900F90DF91CF9181
:10C590001F910F91FF90EF90DF90CF90BF90AF90E1
:10C5A0009F908F907F906F905F904F903F902F90D3
:10C5B00008958091500F1092500F882339F226EE83
:10C5C00035E13093FB0E2093FA0E8091520F8823B1
:10C5D00009F4BCCFD7CF9B81913011F59091570FC3
:10C5E000913069F080918202882309F466C081E06D
:10C5F000913009F080E020E245EC55E1B3CF809125
:10C60000500F1092500F882369F322ED35E13093DB
:10C61000FB0E2093FA0E8091520F882319F3B2CFAC
:10C620008B81823019F58091570F823081F0809193
:10C630008202882309F441C081E09091570F923023
:10C6400009F080E023E044EB55E1632D8CCF80912D
:10C65000500F1092500F882351F38EE894E60E94F9
:10C6600040628091520F882311F38CCF9B819330CD
:10C6700009F034C18091570F833009F45CC0809178
:10C6800082028823D1F08FE09CE39F938F938AEA04
:10C6900095E19F938F9383E082198F9381E090912E
:10C6A000570F933009F080E08F930E943F8D0F90D9
:10C6B0000F900F900F900F900F908091A60F909178
:10C6C000A70FA091A80FB091A90F80935B0F909333
:10C6D0005C0FA0935D0FB0935E0F8B81883009F5DE
:10C6E0008091570F883009F4C2C08091820288235C
:10C6F000C1F011E08091570F883009F010E060918F
:10C700005B0F70915C0F80915D0F90915E0F0E94A6
:10C71000176000E09C0142E655E1672D812F0E94E1
:10C72000FB9B9B819F5F9B8389819813ECCE89E063
:10C730008093510F27CF8091500F1092500F882374
:10C7400009F49DCF0E940F3C8091520F882309F479
:10C7500096CF18CF8091570F843089F08091820254
:10C76000882309F4AACF64E0621981E09091570F01
:10C77000943009F080E023E04DE955E1F4CE80915A
:10C78000500F1092500F882349F383E597E40E94DD
:10C7900040628091520F882309F3F4CE8091570FA5
:10C7A000853009F180918202882361F081E09091C7
:10C7B000570F953009F080E023E04DE855E1642DF6
:10C7C0000F94799E8091A60F9091A70FA091A80F2A
:10C7D000B091A90F80935B0F90935C0FA0935D0FB6
:10C7E000B0935E0F9ECF8091500F1092500F882310
:10C7F000C9F289ED9CE30E9440628091520F882328
:10C8000089F2C0CE8091570F863079F080918202F4
:10C810008823C1F281E09091570F963009F080E0B3
:10C8200023E043E855E1652D9ECE8091500F109294
:10C83000500F882359F38DEF95E60E944062809156
:10C84000520F882319F39ECE8091500F1092500FF3
:10C85000882309F455C02EE735E13093FB0E209371
:10C86000FA0E8091520F882309F44AC08BCE809132
:10C87000500F1092500F882309F437CF0F94D49F94
:10C8800020E030E0A90160915B0F70915C0F809116
:10C890005D0F90915E0F0F9456C90F94C9CA1F92F5
:10C8A00088EC882E80E4982E9AE7A92E90E4B92E81
:10C8B0006B0114E6E12EF12C00E010E020E030E006
:10C8C000A9016BE57FE082E695E10E94F98E0F9069
:10C8D0008091520F882309F408CF54CE9B81943065
:10C8E00009F438CF953009F459CF963009F48ACF3E
:10C8F000973009F0E2CE9091570F973009F4A4CF0A
:10C9000080918202882309F45DCF81E0973009F09D
:10C9100080E020E24EE655E1662D25CE9F92AF9253
:10C92000BF92CF92DF92EF92FF920F931F93CF931C
:10C93000DF9361E081E00E94758DC091580FCC2E8D
:10C9400085E0982E9C0E99E4A92E97E4B92ED7E0A5
:10C95000DC1B16E01C1B05E00C1B84E0F82EFC1A07
:10C9600082E0E82EEC1A81E0D82EDC1AC11133C027
:10C970008091570F8823B9F080918202882361F05B
:10C980006C2D619581E09091570F911180E024E02A
:10C990004DE455E10F94799ECF5FC911E7CF88E050
:10C9A0008093510F0CC08091500F1092500F88232C
:10C9B00019F30E94BB8E8091520F8823E9F2DF9118
:10C9C000CF911F910F91FF90EF90DF90CF90BF908C
:10C9D000AF909F900895C13011F59091570F91300D
:10C9E00069F0809182028823B9F281E0913009F0E8
:10C9F00080E020E243E355E16D2DCCCF8091500FD4
:10CA00001092500F882369F326E435E13093FB0E32
:10CA10002093FA0E8091520F882319F3D0CFC230A1
:10CA200009F0BDC09091570F923071F08091820251
:10CA3000882309F4B1CF81E0923009F080E020E250
:10CA40004AE155E16E2DA6CF8091500F1092500F04
:10CA5000882361F32BE235E13093FB0E2093FA0E2D
:10CA60008091520F882311F3AACF8091570F833002
:10CA700089F080918202882309F48ECF63E06C19DB
:10CA800081E09091570F933009F080E023E049E076
:10CA900055E180CF8091500F1092500F882349F3B9
:10CAA0008AEA94E40E9440628091520F882309F33D
:10CAB00086CF9091570F943071F080918202882335
:10CAC00009F46ACF81E0943009F080E020E24DEE75
:10CAD00054E16F2D5FCF8091500F1092500F88233B
:10CAE00061F32EEF34E13093FB0E2093FA0E809128
:10CAF000520F882311F363CF8091570F853081F057
:10CB000080918202882309F447CF81E09091570FEA
:10CB1000953009F080E023E04CED54E1602F3ACFEE
:10CB20008091500F1092500F882351F38AEA94E4B9
:10CB30000E9440628091520F882311F340CF909160
:10CB4000570F963071F080918202882309F424CF28
:10CB500081E0963009F080E020E240EC54E1612F62
:10CB600019CF8091500F1092500F882361F321ED5F
:10CB700034E13093FB0E2093FA0E8091520F8823FC
:10CB800011F31DCF8091500F1092500F8823C9F0E0
:10CB90000E9449478091520F882399F010CFC330EB
:10CBA00009F463CFC43009F484CFC53009F4A4CFAD
:10CBB000C63029F2C73009F0EFCE8091570F873089
:10CBC00009F380918202882309F4E6CEBF92AF92E6
:10CBD0008FEA94E19F938F93DF9381E09091570FB9
:10CBE000973009F080E08F930E943F8D0F900F9057
:10CBF0000F900F900F900F90CFCEAF92BF92CF9229
:10CC0000DF92EF92FF920F931F93CF93DF9361E038
:10CC100081E00E94758DC091580F85E0B82EBC0E42
:10CC2000D5E0DC1B14E01C1B03E00C1B93E9C92EB0
:10CC300094E1D92E82E0F82EFC1A81E0E82EEC1A5D
:10CC4000AC2EA194C11131C08091570F8823B1F04F
:10CC500080918202882359F081E09091570F9111C1
:10CC600080E024E04DE455E16A2D0F94799ECF5F7A
:10CC7000CB11E8CF86E08093510F0CC08091500F0C
:10CC80001092500F882321F30E94BB8E8091520F87
:10CC90008823F1F2DF91CF911F910F91FF90EF90D8
:10CCA000DF90CF90BF90AF900895C13011F5809183
:10CCB000570F813079F0809182028823C1F281E0A0
:10CCC0009091570F913009F080E023E044EA54E15D
:10CCD0006E2DCBCF8091500F1092500F882359F3B7
:10CCE0008EE097E60E9440628091520F882319F3EC
:10CCF000D1CFC23009F076C09091570F923071F0C9
:10CD000080918202882309F4B2CF81E0923009F049
:10CD100080E020E24FE754E16F2DA7CF8091500FC4
:10CD20001092500F882361F3D092FB0EC092FA0E3E
:10CD30008091520F882321F3ADCF8091570F83301C
:10CD400081F080918202882309F491CF81E0909153
:10CD5000570F933009F080E023E041E754E1602F62
:10CD600084CF8091500F1092500F882351F38AEA9C
:10CD700094E40E9440628091520F882311F38ACF7D
:10CD80008091570F843081F080918202882309F4CA
:10CD90006ECF81E09091570F943009F080E023E04E
:10CDA00047E654E1612F61CF8091500F1092500FF0
:10CDB000882351F38DED98E60E9440628091520FD6
:10CDC000882311F367CF8091500F1092500F882362
:10CDD000A9F081EE99E60E9440628091520F88236B
:10CDE00069F058CFC33009F4A8CFC43049F2C53038
:10CDF00009F03DCF8091570F853029F38091820251
:10CE0000882309F434CF81E09091570F953009F0D1
:10CE100080E023E049E554E16D2F27CF9F92AF9248
:10CE2000BF92CF92DF92EF92FF920F931F93CF9317
:10CE3000DF9361E081E00E94758DC091580FDC2F77
:10CE400085E0982E9C0E96E5A92E9EE8B92E19E055
:10CE50001C1B08E00C1B87E0F82EFC1A86E0E82E6D
:10CE6000EC1A85E0D82EDC1A84E0C82ECC1AC11149
:10CE700033C08091570F8823B9F0809182028823B4
:10CE800061F06D2F619581E09091570F911180E0D5
:10CE900024E043E855E10F94799ECF5FC911E7CFB5
:10CEA0008AE08093510F0CC08091500F1092500F68
:10CEB000882319F30E94BB8E8091520F8823E9F2D8
:10CEC000DF91CF911F910F91FF90EF90DF90CF9066
:10CED000BF90AF909F900895C13041F5E9E7FDE61E
:10CEE0008591949190936F0F80936E0F9091570F4F
:10CEF000913059F080918202882379F261E06D1BB4
:10CF000081E0913061F180E02AC08091500F109251
:10CF1000500F882379F325E633E13093FB0E2093FD
:10CF2000FA0E8091520F882329F3CACFC23009F03C
:10CF30000FC1EBE7FDE68591949190936F0F80937D
:10CF40006E0F9091570F923071F08091820288237A
:10CF500009F4A3CF62E06D1B81E09230A1F620E2DC
:10CF600046E553E198CF8091500F1092500F8823DF
:10CF700061F320E333E13093FB0E2093FA0E8091AE
:10CF8000520F882311F39CCF8091570F833089F083
:10CF900080918202882309F480CF63E06D1B81E0D9
:10CFA0009091570F933009F080E023E04EE153E178
:10CFB00072CF8091500F1092500F882349F386E072
:10CFC00096E40E9440628091520F882309F378CF43
:10CFD0009091570F943071F080918202882309F468
:10CFE0005CCF81E0943009F080E020E247E053E13B
:10CFF0006C2D51CF8091500F1092500F882361F308
:10D0000027E133E13093FB0E2093FA0E8091520F0B
:10D01000882311F355CF8091570F853081F080918F
:10D020008202882309F439CF81E09091570F95301F
:10D0300009F080E023E04AEF52E16D2D2CCF809182
:10D04000500F1092500F882351F380EA9DE30E9405
:10D0500040628091520F882311F332CF9091570F85
:10D06000963071F080918202882309F416CF81E016
:10D07000963009F080E020E241EE52E16E2D0BCFB8
:10D080008091500F1092500F882361F323EF32E10B
:10D090003093FB0E2093FA0E8091520F882311F3E8
:10D0A0000FCF8091570F8730B1F080918202882393
:10D0B00009F4F3CE8DE998E49F938F9382ED92E18A
:10D0C0009F938F93FF9281E09091570F973009F4CF
:10D0D0006AC080E068C08091500F1092500F882382
:10D0E00021F30E949D488091520F8823F1F2E8CEEF
:10D0F0009091570F983071F080918202882309F443
:10D10000CCCE81E0983009F080E020E24AEB52E199
:10D11000602FC1CE8091500F1092500F882361F381
:10D120002DEC32E13093FB0E2093FA0E8091520FDA
:10D13000882311F3C5CE8091500F1092500F882391
:10D1400001F10E94568E8091520F8823D1F0B8CE03
:10D15000C33009F419CFC43009F43ACFC53009F40B
:10D160005ACFC63009F47ACFC73009F49ACFC83005
:10D1700009F4BECFC93009F090CE8091570F8930A5
:10D18000D1F280918202882309F487CEBF92AF92B8
:10D190008EEA92E19F938F931F9381E09091570FB6
:10D1A000993009F096CF8F930E943F8D0F900F908A
:10D1B0000F900F900F900F9070CE5F926F927F92B2
:10D1C0008F929F92AF92BF92CF92DF92EF92FF9297
:10D1D0000F931F93CF93DF9361E081E00E94758DE1
:10D1E000C091580F85E0682E6C0E96E5E92E9EE8FA
:10D1F000F92E2EEAC22E22E1D22ED4E0DC1B13E05F
:10D200001C1B3CE9A32E31E1B32E02E00C1B41EBC9
:10D21000842E41E1942E81E0782E7C1A5C2E51946C
:10D22000C11136C08091570F8823B1F080918202DE
:10D23000882359F081E09091570F911180E024E00C
:10D2400043E855E1652D0F94799ECF5FC611E8CF75
:10D2500085E08093510F0CC08091500F1092500FB9
:10D26000882321F30E94BB8E8091520F8823F1F214
:10D27000DF91CF911F910F91FF90EF90DF90CF90B2
:10D28000BF90AF909F908F907F906F905F90089528
:10D29000C13001F59091570F913069F08091820271
:10D2A000882399F281E0913009F080E020E243EA9E
:10D2B00051E1672DC8CF8091500F1092500F8823F5
:10D2C00069F39092FB0E8092FA0E8091520F8823A0
:10D2D00029F3CECFC23009F051C09091570F923050
:10D2E00071F080918202882309F4AFCF81E09230FF
:10D2F00009F080E020E24AE851E1602FA4CF80915C
:10D30000500F1092500F882361F3B092FB0EA09241
:10D31000FA0E8091520F882321F3AACF8091570FE4
:10D32000833081F080918202882309F48ECF81E0DE
:10D330009091570F933009F080E023E047E751E1E7
:10D34000612F81CF8091500F1092500F882351F39D
:10D350008CEB9EE30E9440628091520F882311F370
:10D3600087CF8091500F1092500F882381F00E9438
:10D37000568E8091520F882351F07ACFC33071F2CC
:10D38000C43009F062CF8091570F843051F38091FF
:10D390008202882309F459CFFF92EF92DF92CF9255
:10D3A000DF9381E09091570F943009F080E08F93E4
:10D3B0000E943F8D0F900F900F900F900F900F9045
:10D3C00044CF8F929F92AF92BF92CF92DF92EF9213
:10D3D000FF920F931F93CF93DF9361E081E00E9450
:10D3E000758DC091580F85E0982E9C0E96E5E92E1C
:10D3F0009EE8F92E2EEAC22E22E1D22ED3E0DC1BCB
:10D4000012E01C1B3DE4A32E32E1B32E01E00C1B05
:10D410008C2E8194C11133C08091570F8823B1F0B5
:10D4200080918202882359F081E09091570F9111E9
:10D4300080E024E043E855E1682D0F94799ECF5FAA
:10D44000C911E8CF84E08093510F0CC08091500F38
:10D450001092500F882321F30E94BB8E8091520FAF
:10D460008823F1F2DF91CF911F910F91FF90EF9000
:10D47000DF90CF90BF90AF909F908F900895C13074
:10D4800001F59091570F913069F0809182028823C5
:10D49000B1F281E0913009F080E020E24CE352E10A
:10D4A000602FCBCF8091500F1092500F882369F3DB
:10D4B000B092FB0EA092FA0E8091520F882329F3AE
:10D4C000D1CFC23081F58091570F823081F08091A9
:10D4D0008202882309F4B3CF81E09091570F9230F4
:10D4E00009F080E023E049E252E1612FA6CF80916C
:10D4F000500F1092500F882351F38DE893E40E944F
:10D5000040628091520F882311F3ACCF8091500F6D
:10D510001092500F882371F00E94568E8091520F06
:10D52000882341F09FCFC33009F089CF8091570FF6
:10D53000833061F380918202882309F480CFFF92C7
:10D54000EF92DF92CF92DF9381E09091570F93306B
:10D5500009F080E08F930E943F8D0F900F900F9005
:10D560000F900F900F906BCF5F926F927F928F9280
:10D570009F92AF92BF92CF92DF92EF92FF920F9362
:10D580001F93CF93DF93FF24F39480910F1D90910D
:10D59000101D892B09F4F12C61E081E00E94758D4A
:10D5A000C091580F8C2E95E0992E9C0EAA24A3941E
:10D5B00084E0E82EEC1A83E0D82EDC1A82E0C82E34
:10D5C000CC1A7A2C7C1A6C2E619487E0B82EBC1A87
:10D5D000C111B8C08091570F882309F495C080917C
:10D5E0008202882359F081E09091570F911180E0D9
:10D5F00024E04EED50E1662D0F94799E8091D91074
:10D6000080935B0FC430E9F4A0926D0F8091570FA7
:10D61000843009F445C180918202882391F0D1E0E1
:10D620008091570F843009F0D0E080915B0F0F9408
:10D63000BD1D00E09C0147EC50E16E2D8D2F0E9436
:10D64000FB9B10E000E0D5E05C2E581800935B0FC8
:10D65000CD131FC0F801EE0FFF1FE758F249859167
:10D66000949190936F0F80936E0F8091570F8C174A
:10D6700009F42BC180918202882359F081E09091B6
:10D68000570F9D1380E023E04DEB50E1652D0F9483
:10D69000799E8D2F0F5F1F4FD6E08630B9F68091AF
:10D6A000B10F9091B20F892B19F4FF2009F42DC10D
:10D6B000C73009F58091570F873009F417C1809161
:10D6C00082028823C1F089E29BE49F938F9384EBCD
:10D6D00090E19F938F93BF9281E09091570F973085
:10D6E00009F080E08F930E943F8D0F900F900F9074
:10D6F0000F900F900F9088E0FF24F394CF5FC91133
:10D7000067CF8093510F0EC08091500F1092500F31
:10D71000882309F464CF0E94BB8E8091520F882326
:10D7200009F45DCFDF91CF911F910F91FF90EF90A2
:10D73000DF90CF90BF90AF909F908F907F906F9031
:10D740005F900895C13009F05FC08091570F81301C
:10D7500009F43FC080918202882309F44FCFD1E0C1
:10D760008091570F813009F0D0E080910F1D90918A
:10D77000101D0F94881D00E09C0147ED50E1672DBE
:10D780008D2F0E94FB9B8091D81080935B0FC3303C
:10D7900009F034CF10926D0F8091570F833009F448
:10D7A0006AC080918202882309F44BCFD1E0809136
:10D7B000570F833009F0D0E080915B0F0F94BD1DAF
:10D7C00000E09C0147EC50E16D2D8D2F0E94FB9BEA
:10D7D00015CF8091500F1092500F882309F4BACFC3
:10D7E0000F94D49F07E21BE42CE231E050E040E0CC
:10D7F0006FE07DE187ED90E10F944CA18091520F95
:10D80000882309F4A7CF8ECFC23009F0BCCF809116
:10D81000570F8230B9F080918202882309F4EECE4E
:10D82000D1E08091570F823009F0D0E08091B10FA4
:10D830009091B20F0F94881D00E09C0143ED50E1E0
:10D840006C2D9ECF8091500F1092500F882319F3AA
:10D850000F94D49F03E417ED2CE830E050E040E053
:10D8600061EB7FE083ED90E10F944CA18091520F2A
:10D87000882389F257CF8091500F1092500F882340
:10D8800009F48FCF0F94D49F69E178E387EC90E19E
:10D890000F948BA28091520F882309F482CF42CF3C
:10D8A0008091500F1092500F882309F4B4CE0F943A
:10D8B000D49F69E178E387EC90E10F948BA280918B
:10D8C000520F882309F4A7CE2DCF8091500F1092CC
:10D8D000500F882309F4CECE84E39BE40E9440627B
:10D8E0008091520F882309F4C5CE1CCF8091500F30
:10D8F0001092500F882309F4E2CE0E94294B8091A8
:10D90000520F882309F4DBCE0DCF87E0F7CE9F922C
:10D91000AF92BF92CF92DF92EF92FF920F931F933D
:10D92000CF93DF9361E081E00E94758DC091580F25
:10D93000DC2F85E0982E9C0E96E1A92E90E1B92E61
:10D9400019E01C1B08E00C1B87E0F82EFC1A86E08F
:10D95000E82EEC1A85E0D82EDC1A84E0C82ECC1A0A
:10D96000C11133C08091570F8823B9F08091820292
:10D97000882361F06D2F619581E09091570F91118F
:10D9800080E024E047E850E10F94799ECF5FC91111
:10D99000E7CF8AE08093510F0CC08091500F109216
:10D9A000500F882319F30E94BB8E8091520F882359
:10D9B000E9F2DF91CF911F910F91FF90EF90DF90EF
:10D9C000CF90BF90AF909F900895C13019F580918E
:10D9D000570F813081F0809182028823B9F261E093
:10D9E0006D1B81E09091570F913009F080E023E0AA
:10D9F00041E55DE6C9CF8091500F1092500F88230A
:10DA000051F38AE39EE60E9440628091520F882380
:10DA100011F3CFCFC23009F006C19091570F923069
:10DA200079F080918202882309F4B0CF62E06D1B07
:10DA300081E0923009F080E020E24DE750E1A4CF90
:10DA40008091500F1092500F882359F320E134E158
:10DA50003093FB0E2093FA0E8091520F882309F326
:10DA6000A8CF9091570F933079F08091820288234C
:10DA700009F48CCF63E06D1B81E0933009F080E006
:10DA800020E241E750E180CF8091500F1092500F7B
:10DA9000882359F328E730E13093FB0E2093FA0EE8
:10DAA0008091520F882309F384CF9091570F9430BF
:10DAB00071F080918202882309F468CF81E094306C
:10DAC00009F080E020E245E650E16C2D5DCF8091C9
:10DAD000500F1092500F882361F32CE630E1309301
:10DAE000FB0E2093FA0E8091520F882311F361CF21
:10DAF0009091570F953071F080918202882309F43C
:10DB000045CF81E0953009F080E020E249E550E121
:10DB10006D2D3ACF8091500F1092500F882361F3F2
:10DB200020E630E13093FB0E2093FA0E8091520FE5
:10DB3000882311F33ECF8091570F863081F080917A
:10DB40008202882309F422CF81E09091570F96300A
:10DB500009F080E023E044E450E16E2D15CF809180
:10DB6000500F1092500F882351F38EE492E60E94DA
:10DB700040628091520F882311F31BCF8091570F81
:10DB8000873081F080918202882309F4FFCE81E002
:10DB90009091570F973009F080E023E046E350E181
:10DBA0006F2DF2CE8091500F1092500F882351F3B9
:10DBB0008FE39CE40E9440628091520F882311F30E
:10DBC000F8CE9091570F983071F08091820288239F
:10DBD00009F4DCCE81E0983009F080E020E24AE1EF
:10DBE00050E1602FD1CE8091500F1092500F8823BA
:10DBF00061F329E230E13093FB0E2093FA0E80911D
:10DC0000520F882311F3D5CE8091500F1092500FF0
:10DC1000882311F1B092FB0EA092FA0E8091520F60
:10DC20008823D1F0C6CEC33009F41BCFC43009F429
:10DC30003CCFC53009F45CCFC63009F47CCFC73087
:10DC400009F49CCFC83009F4BCCFC93009F09ECE8E
:10DC50009091570F9930C1F280918202882309F484
:10DC600095CE81E0993009F080E020E245E050E176
:10DC7000612F8ACEAF92BF92CF92DF92EF92FF9246
:10DC80000F931F93CF93DF9361E081E00E94758D26
:10DC9000C091580F85E0C82ECC0ED5E0DC1B93E078
:10DCA000D92E14E01C1BBD2CBC1A82E0F82EFC1AE5
:10DCB00081E0E82EEC1AAC2EA194C1112BC080910A
:10DCC000570F882381F080918202882369F181E0D7
:10DCD0009091570F911180E024E04EEF5FE06A2DA4
:10DCE0000F94799E21C08091500F1092500F88237D
:10DCF00051F30E94BB8E8091520F882321F3DF9154
:10DD0000CF911F910F91FF90EF90DF90CF90BF9038
:10DD1000AF900895C130A1F59091570F913059F00F
:10DD200080918202811119C0CF5FCC11C6CF86E0ED
:10DD30008093510FE4CF8091500F1092500F8823A1
:10DD400079F380913B028C2780933B02D092820230
:10DD50008091520F882321F3D2CF81E0913009F0D6
:10DD600080E090913B022DEE3FE0911102C029EE40
:10DD70003FE001E040EF5FE06E2D0E94FB9BD4CFBF
:10DD8000C23009F077C08091570F823079F08091CE
:10DD90008202882349F281E09091570F923009F076
:10DDA00080E023E042E75DE66F2D9ACF8091500F2F
:10DDB0001092500F882359F38AE69CE40E94406237
:10DDC0008091520F882319F39ACF8091570F833097
:10DDD00081F080918202882309F4A6CF81E090919E
:10DDE000570F933009F080E023E04BE65DE66B2DA2
:10DDF00077CF8091500F1092500F882351F385E612
:10DE00009CE40E9440628091520F882311F377CFE7
:10DE10008091570F843081F080918202882309F429
:10DE200083CF81E09091570F943009F080E023E098
:10DE300044E65DE6612F54CF8091500F1092500F51
:10DE4000882351F380E69CE40E9440628091520F47
:10DE5000882311F354CF8091500F1092500F8823D4
:10DE6000A9F086E39CE30E9440628091520F8823D0
:10DE700069F045CFC33009F4A8CFC43049F2C530AA
:10DE800009F052CF8091570F853029F3809182029B
:10DE9000882309F449CF81E09091570F953009F01C
:10DEA00080E023E04BE55DE66D2F1ACF3F924F9265
:10DEB0005F926F927F928F929F92AF92BF92CF921A
:10DEC000DF92EF92FF920F931F93CF93DF93CDB723
:10DED000DEB7EB970FB6F894DEBF0FBECDBF8091D3
:10DEE0004307882369F180912F1E00E010E083FF33
:10DEF00023C08BE69EE10E94F6E38BE1EBE6FEE1B8
:10DF0000DE01919601900D928A95E1F710E000E014
:10DF1000BE016F5F7F4FCE0181960F94CE89181698
:10DF20003CF4CE0101960E94DDDB080F111DF0CFFD
:10DF3000CE0181960F94D83A009348071093490771
:10DF400061E081E00E94758D1091580F412E85E0AF
:10DF5000582E510E312E319494E2A92E98E3B92E09
:10DF600021EC822E2FE0922E81E0682E611A111191
:10DF700013C08091570F882339F180918202882342
:10DF800059F081E09091570F911180E024E045EC29
:10DF90005FE0632D0F94799E80912F1E85FD5BC0FD
:10DFA00083FF59C0113009F054C08091570F813060
:10DFB00079F180918202811138C082E01F5F511295
:10DFC000D6CF8093510F0CC08091500F1092500FFC
:10DFD000882399F20E94BB8E8091520F882369F2A8
:10DFE000EB960FB6F894DEBF0FBECDBFDF91CF9199
:10DFF0001F910F91FF90EF90DF90CF90BF90AF9067
:10E000009F908F907F906F905F904F903F9008957A
:10E010008091500F1092500F882359F20E9424389B
:10E020008091520F882329F2DBCFBF92AF929F924B
:10E030008F926F9281E09091570F913009F080E0BC
:10E040008F930E943F8D0F900F900F900F900F9025
:10E050000F9082E001C081E090918202992309F43F
:10E06000ADCF082FD12CC12C712E7418802FE090C9
:10E070004807F0904907CE14DF0408F09FCF011342
:10E08000ACC081E0E81AF108EC18FD088BE69EE1CF
:10E090000E94F6E38BE1EBE6FEE1DE019196019052
:10E0A0000D928A95E1F7F12CBE016F5F7F4FCE0193
:10E0B00081960F94CE8918167CF4CE0101960E94A9
:10E0C000DDDB882389F3EF106BC0BE016F5F7F4FEC
:10E0D00082E79FE00E94F8DBCE0181960F94D83A48
:10E0E00090912F1E8091570F94FF7CC0811366C0C2
:10E0F0009091500F1092500F992309F45FC019822C
:10E100001C8280916E1E60E57EE1882311F06BE633
:10E110007EE121E042E75FE0CE0101960F94F92312
:10E12000882309F43FC08BE1FE013196ABE6BEE1E6
:10E1300001900D928A95E1F780912F1E8F7D80933B
:10E140002F1EA091241EAA3080F481E08A0F8093B4
:10E15000241E8BE18A9FD0011124AA57B14EEBE611
:10E16000FEE101900D928A95E1F7CE0101960F94A0
:10E17000D83A1092580F82E090E0A0E0B0E080938F
:10E18000530F9093540FA093550FB093560F81E007
:10E190008093520F1092400783E08093820220CF39
:10E1A000F39482CF0F941A5E62E77FE08BEA9FE0E0
:10E1B0000F9403568AE00F94484AD7CF9091820279
:10E1C000992359F0FF24F3948113F12C6F2D872D9F
:10E1D0000E94F69241E0811118C08FEFC81AD80A48
:10E1E0000F5F44CF8117B1F0809182028823A9F399
:10E1F000FF24F3948091570F8113F12C6F2D872DFD
:10E200000E94F692882349F340E0672D8F2D0F94EA
:10E21000199EE3CF8091500F1092500F882321F365
:10E220008BEC9FE40E9440628091520F8823E1F2C0
:10E23000D7CE2F923F924F925F926F927F928F92A2
:10E240009F92AF92BF92CF92DF92EF92FF920F9385
:10E250001F93CF93DF9300D000D0CDB7DEB70F94DC
:10E260009D47582E80912F1E83FB222720F929835A
:10E27000212C83FF03C00F94CA47282E61E081E060
:10E280000E94758D8091580F8D83782E8B5F8A83C5
:10E290000DEA12E099E3E92E9FE0F92E2CE4C22E5C
:10E2A00020E9D22E3DE4A32E3FE0B32E81E0482E9C
:10E2B000471884E087198B8383E087198C8382E079
:10E2C000382E37184BEC842E4FE8942E9D819111F7
:10E2D00043C18091570F882309F417C180918202AE
:10E2E000882361F0672D619581E09091570F91111E
:10E2F00080E024E044E85FE00F94799E511050C123
:10E300000F94D847882309F4E5C18D81813009F045
:10E3100007C28091570F813009F4B6C18091820203
:10E320008111C1C192E09E838E818F5F9D8189138F
:10E3300016C08091570F891709F402C2809182029A
:10E34000882369F06D81671981E09091570F2D81C5
:10E35000921380E023E042E35FE00F94799E8E8188
:10E360008E5F8E839E812D81921316C08091570FF0
:10E37000891709F4F6C180918202882369F06D81C2
:10E38000671981E09091570F2D81921380E023E06F
:10E3900046E25FE00F94799E8E818F5F9D818913A5
:10E3A00016C08091570F891709F4ECC18091820241
:10E3B000882369F06D81671981E09091570F2D8155
:10E3C000921380E023E048E15FE00F94799E6E8035
:10E3D0006394639451101EC08D81681217C08091A0
:10E3E000570F9D81891709F4DEC18091820288232D
:10E3F00069F06D81671981E09091570F2D8192131B
:10E4000080E023E049E05FE00F94799E83E0682E8E
:10E410008E81680E9D81691216C08091570F8615F6
:10E4200009F4D2C180918202882369F06D81671955
:10E4300081E09091570F2D81921380E023E049EF06
:10E440005EE00F94799E81E0860D9D81891316C050
:10E450008091570F891709F4C8C1809182028823DF
:10E4600069F06D81671981E09091570F2D819213AA
:10E4700080E023E04BEE5EE00F94799E82E0860D13
:10E4800051103AC09981992309F4E4C1211034C094
:10E490002D81821314C09091570F921709F4B6C1C1
:10E4A00080918202882359F06D81671981E02D8166
:10E4B000921380E020E24AED5EE00F94799E83E0C3
:10E4C000860D9D81891316C08091570F891709F415
:10E4D000B0C180918202882369F06D81671981E063
:10E4E0009091570F2D81921380E023E049EC5EE07C
:10E4F0000F94799E84E0860D9D819F5F9D832A8184
:10E500009213E4CE8093510F0EC08091500F109261
:10E51000500F882309F4E2CE0E94BB8E8091520FE7
:10E52000882309F4DBCE26960FB6F894DEBF0FBE23
:10E53000CDBFDF91CF911F910F91FF90EF90DF90B2
:10E54000CF90BF90AF909F908F907F906F905F9093
:10E550004F903F902F900895552009F4D1CE2D81F2
:10E56000213071F58091570F8130E9F0809182025E
:10E570008823B1F09F928F9288E79FE09F938F93BB
:10E580004F9281E09091570F913009F080E08F9386
:10E590000E943F8D0F900F900F900F900F900F9053
:10E5A00095E09E83DFCE8091500F1092500F88230C
:10E5B000E9F20E94CB8F8091520F8823B9F2B3CF3A
:10E5C0008D81823031F58091570F823099F08091A2
:10E5D0008202882361F081E09091570F923009F018
:10E5E00080E023E04DE65FE0632D0F94799E25E007
:10E5F0002E83D2CE8091500F1092500F882339F382
:10E6000083E99CE40E9440628091520F8823F9F2D2
:10E610008ACF9D81933009F043C18091570F833099
:10E6200099F080918202882361F081E09091570FE8
:10E63000933009F080E023E048E65FE06C810F94BE
:10E64000799E85E08E83C3CE8091500F1092500F3B
:10E65000882339F386EF9CE70E9440628091520F35
:10E660008823F9F260CF8091500F1092500F8823C9
:10E6700009F41FC18EEC9CE30E9440628091520F0E
:10E68000882309F416C14FCF8091500F1092500F7C
:10E69000882309F443CE0E944C908091520F882326
:10E6A00009F43CCE40CFDF92CF92BF92AF924F920F
:10E6B00081E09091570F913009F080E08F930E9494
:10E6C0003F8D0F900F900F900F900F900F9022E0C2
:10E6D0002E832ACE81E08E832E818D81281324CE35
:10E6E0008091570F8217F9F080918202882309F4F4
:10E6F0001BCE1F930F93FF92EF928D8187198F93FB
:10E7000081E09091570F2D81921380E08F930E94AA
:10E710003F8D0F900F900F900F900F900F9004CEA1
:10E7200092E09E83D9CF8091500F1092500F882392
:10E73000D9F20F946E4B8091520F8823A9F2F3CE39
:10E740008091500F1092500F882309F4F7CD87E87D
:10E750009CE60E9440628091520F882309F4EECD1E
:10E76000E2CE8091500F1092500F882309F403CE0F
:10E7700084EB9AE60E9440628091520F882309F44C
:10E78000FACDD1CE8091500F1092500F882309F40A
:10E790000DCE83ED96E70E9440628091520F882350
:10E7A00009F404CEC0CE8091500F1092500F8823F0
:10E7B00009F41BCE87E290E50E9440628091520FDF
:10E7C000882309F412CEAFCE8091500F1092500FD3
:10E7D000882309F427CE89E495E70E94406280915E
:10E7E000520F882309F41ECE9ECE8091500F1092B6
:10E7F000500F882309F431CE89E694E70E944062E5
:10E800008091520F882309F428CE8DCE8091500F2D
:10E810001092500F882309F443CE27EE3EE0309348
:10E82000FB0E2093FA0E8091520F882309F438CE04
:10E830007ACE8091500F1092500F882309F449CE60
:10E8400086E59FE60E9440628091520F882309F47A
:10E8500040CE69CE9D81891321C09091570F2D81A3
:10E86000921302C01092500F809182028823B1F05F
:10E870001F921F9224E43FE03F932F938D818719CD
:10E880008F9381E02D81921380E08F930E943F8DC2
:10E890000F900F900F900F900F900F9083E02BCE62
:10E8A0008D81843009F07CCE8091570F843009F43B
:10E8B000DACE80918202882309F4C3CE81E0909160
:10E8C000570F943009F080E023E04AE55FE06B8168
:10E8D0008CCEDF92EF92FF920F931F93CF93DF9333
:10E8E00061E081E00E94758DC091580F85E0E82EAF
:10E8F000EC0ED4E0DC1B13E01C1B02E00C1B81E0DF
:10E90000F82EFC1ADC2ED194C1112EC08091570F25
:10E910008823B1F080918202882359F081E09091A0
:10E92000570F911180E024E046E65DE06D2D0F94D5
:10E93000799ECF5FCE11E8CF85E08093510F0CC058
:10E940008091500F1092500F882321F30E94BB8EAC
:10E950008091520F8823F1F2DF91CF911F910F9197
:10E96000FF90EF90DF900895C13011F58091570F1F
:10E97000813079F0809182028823D9F281E09091F0
:10E98000570F913009F080E023E049E55DE06F2DFD
:10E99000CECF8091500F1092500F882359F386E10B
:10E9A00092E50E9440628091520F882319F3D4CFE0
:10E9B000C23009F055C08091570F823081F08091AC
:10E9C0008202882309F4B5CF81E09091570F9230ED
:10E9D00009F080E023E04EE45DE0602FA8CF809155
:10E9E000500F1092500F882351F385EB92E50E944F
:10E9F00040628091520F882311F3AECF8091570F60
:10EA0000833081F080918202882309F492CF81E0E3
:10EA10009091570F933009F080E023E042E45DE0ED
:10EA2000612F85CF8091500F1092500F882351F3A2
:10EA30008EE493E50E9440628091520F882311F387
:10EA40008BCF8091500F1092500F882391F08BE262
:10EA500094E50E9440628091520F882351F07CCF50
:10EA6000C33061F2C43009F064CF8091570F843015
:10EA700041F380918202882309F45BCF81E0909179
:10EA8000570F943009F080E023E044E35DE06D2F00
:10EA90004ECF7F928F929F92AF92BF92CF92DF9292
:10EAA000EF92FF920F931F93CF93DF930F94D8476A
:10EAB000882309F46CC081E080935B0F0E94B08EC4
:10EAC000982E61E081E00E94758DC091580F85E01D
:10EAD000882E8C0E7C2E71949EE6E92E9AE0F92EFB
:10EAE000D3E0DC1B23E7C22E2AE0D22E12E01C1B4F
:10EAF00038E7A32E3AE0B32E01E00C1BC11114C07D
:10EB00008091570F882309F444C0809182028823A2
:10EB100059F081E09091570F911180E024E040E896
:10EB20005AE0672D0F94799E8091EA1081115DC0A3
:10EB300080910F1D9091101D2091920230919302AF
:10EB400021503109821793070CF04FC0C13009F0F2
:10EB5000FCC08091570F8130C1F1809182028823DF
:10EB600061F081E09091570F913009F080E023E04F
:10EB70004DE75DE6602F0F94799E992009F455C00A
:10EB800082E0CF5F8C12BACF8093510F10C082E029
:10EB900093CF8091500F1092500F882309F4B5CF76
:10EBA0000E94BB8E8091520F882309F4AECFDF9173
:10EBB000CF911F910F91FF90EF90DF90CF90BF907A
:10EBC000AF909F908F907F9008958091500F1092FA
:10EBD000500F882311F28BEE96E50E9440628091DF
:10EBE000520F882309F4B9CFE2CFC13031F69091AA
:10EBF000570F913059F080918202882309F4BDCFDC
:10EC000081E0913009F080E020E2B2CF8091500F96
:10EC10001092500F882379F3B092FB0EA092FA0E57
:10EC20008091520F882339F3C2CF8091EA1081116D
:10EC3000A6C080910F1D9091101D209192023091DD
:10EC4000930221503109821793070CF081C0C23022
:10EC5000A1F48091570F823029F18091820288239C
:10EC600061F081E09091570F923009F080E023E04D
:10EC70004DE95DE6612F0F94799E20910F1D309133
:10EC8000101D8091EA1081117CC0809192029091B8
:10EC900093020197281739070CF073C0C33011F1A4
:10ECA00084E06FCF8091500F1092500F8823A9F20B
:10ECB00088EE96E50E9440628091520F882369F2A7
:10ECC00076CF8091500F1092500F882309F44CC0DA
:10ECD000D092FB0EC092FA0E8091520F882309F455
:10ECE00043C065CF8091570F833089F080918202B5
:10ECF0008823B1F281E09091570F933009F080E0C2
:10ED000023E04DE85DE66D2F0F94799EC9CF809189
:10ED1000500F1092500F882349F385EE96E50E941C
:10ED200040628091520F882309F341CF8091500FA8
:10ED30001092500F882361F1F092FB0EE092FA0ED0
:10ED40008091520F882321F132CF911019CF75CFC6
:10ED500020910F1D3091101DC23009F096CF909177
:10ED6000570F923009F4ADCF80918202882309F4C5
:10ED700084CF81E0923009F080E020E279CFC23088
:10ED800071F3C33009F08CCF9091570F933071F22B
:10ED900080918202882309F483CF81E0933009F0C7
:10EDA00080E020E2AECF2F923F924F925F926F921F
:10EDB0007F928F929F92AF92BF92CF92DF92EF920B
:10EDC000FF920F931F93CF93DF9300D01F92CDB785
:10EDD000DEB70E94B08EE82E61E081E00E94758D62
:10EDE0002091580F2B8363E0F62EE11002C054E00F
:10EDF000F52E1B81812F8B5F898323E0722E972D47
:10EE0000911B9A836624639433E0C32E31E0D32EA2
:10EE100082E0582E511A462C411A312E319443E982
:10EE2000A42E42E0B42E8B81811111C18091570F25
:10EE3000882309F4E7C080918202882359F081E099
:10EE40009091570F911180E024E042E45AE0632D45
:10EE50000F94799EE11013C18B81833009F00FC1AB
:10EE60008091570F833009F44EC180918202811145
:10EE70005BC194E09C838C818F5F9B81891309C067
:10EE80008091570F891709F48DC1809182028111F9
:10EE9000A2C18C818E5F8C83912C812C2B80211AB6
:10EEA0009B812C81921323C0F401EE0FFF1FE758C2
:10EEB000F2498591949180926D0F90936F0F80939A
:10EEC0006E0F8091570F9B81891709F49EC1809125
:10EED0008202882361F081E09091570F2C81921378
:10EEE00080E023E048EE59E0622D0F94799E0C817A
:10EEF00081E0800F8C838A94892809F082C12B815C
:10EF0000821323C08091570F821709F48FC180911B
:10EF100082028823D1F089E69DE89F938F9389ED43
:10EF200099E09F938F938B81811B8F9381E09091C8
:10EF3000570F2B81921380E08F930E943F8D0F908B
:10EF40000F900F900F900F900F9082E0800FE110C4
:10EF500050C09B81891323C08091570F891709F4F2
:10EF600074C1809182028823D1F08DE69DE89F9341
:10EF70008F938BEC99E09F938F938B81811B8F9361
:10EF800081E09091570F2B81921380E08F930E9424
:10EF90003F8D0F900F900F900F900F900F9083E088
:10EFA000800F9B81891323C08091570F891709F423
:10EFB0005BC1809182028823D1F081E79DE89F9315
:10EFC0008F938AEB99E09F938F938B81811B8F9313
:10EFD00081E09091570F2B81921380E08F930E94D4
:10EFE0003F8D0F900F900F900F900F900F9084E037
:10EFF000800F9B819F5F9B832981921314CF809305
:10F00000510F0EC08091500F1092500F882309F4B9
:10F0100012CF0E94BB8E8091520F882309F40BCF30
:10F020000F900F900F900F90DF91CF911F910F9144
:10F03000FF90EF90DF90CF90BF90AF909F908F9018
:10F040007F906F905F904F903F902F9008959B819D
:10F05000913091F58091570F8130F9F080918202C3
:10F06000882309F4F7CE81E09091570F913009F091
:10F0700080E023E040E35AE0642D0F94799E8B8179
:10F08000F81209C08091570F8F1509F45CC0809168
:10F090008202811171C0FC82EECE8091500F1092DD
:10F0A000500F8823D9F289ED99E70E944062809140
:10F0B000520F882399F2B4CF2B81223009F0CACEA7
:10F0C0008091570F823081F080918202882309F469
:10F0D000C1CE81E09091570F923009F080E023E09B
:10F0E00041E25AE0652DC9CF8091500F1092500F28
:10F0F000882351F380ED9AE90E9440628091520F7B
:10F10000882311F38DCF8091500F1092500F8823D8
:10F1100009F4ABCE89E097E50E9440628091520FDE
:10F12000882309F4A2CE7CCF81E09091570F9330D1
:10F1300009F080E023E049E15AE06A810F94799E6A
:10F1400024E02C8398CE8091500F1092500F88238A
:10F1500009F49DCF809159028625809359027092BF
:10F160008202C114D10411F00F94E3358091520F43
:10F17000882309F48CCF54CF6B81611B81E090917F
:10F18000570F2B81921380E09091590228E03AE0CA
:10F19000911102C024E03AE001E04BE05AE00E9405
:10F1A000FB9B79CF8091500F1092500F882309F468
:10F1B0006CCE8091C00C86258093C00C7092820228
:10F1C000A114B10411F00F94B83A8091520F882322
:10F1D00009F45BCE25CF6B81611B81E09091570FC5
:10F1E0002B81921380E09091C00C28E03AE09111BD
:10F1F00002C024E03AE001E047EF59E00E94FB9BA7
:10F2000048CE88248394912C4BCE8091500F10923D
:10F21000500F882309F45BCE84E899E40E94406291
:10F220008091520F882309F452CEFACE8091500F6C
:10F230001092500F882309F46ACE0E94698D809144
:10F24000520F882309F463CEEBCE8091500F1092B9
:10F25000500F882309F485CE0E946D8D8091520F46
:10F26000882309F47ECEDCCE8091500F1092500F8F
:10F27000882309F49ECE0E94718D8091520F8823BD
:10F2800009F497CECDCECF92DF92EF92FF920F93FB
:10F290001F93CF93DF930091040261E081E00E940D
:10F2A000758DC091580FEC2E85E0F82EFC0EDC2EEB
:10F2B000D194C11114C08091570F882309F44BC019
:10F2C00080918202882359F081E09091570F91112B
:10F2D00080E024E04EE659E06D2D0F94799E1FEFFB
:10F2E000D1E0CC2ECE1880913D0718170CF05BC0F2
:10F2F000011779F1812F17FD802F40913907509127
:10F300003A0760913B0770913C07082E04C0769540
:10F310006795579547950A94D2F740FD1AC0DC13BC
:10F3200015C080936D0F8091570F8D1759F1809103
:10F330008202882359F081E09091570F9D1380E05D
:10F3400023E04EE559E06C2D0F94799E17FD29C0FE
:10F35000DF5F1F5FC8CF8091500F1092500F88233E
:10F3600009F4AECF0E94BB8E8091520F882309F41E
:10F37000A7CFDF91CF911F910F91FF90EF90DF907A
:10F38000CF9008958091500F1092500F882379F2FA
:10F3900082EB9CE40E9440628091520F882339F2F4
:10F3A000E8CFDE5FD6CFCF5FFC1283CFD093510F73
:10F3B000E0CF7F928F929F92AF92BF92CF92DF92D7
:10F3C000EF92FF920F931F93CF93DF930E94B08E23
:10F3D000182F61E081E00E94758DC091580F0C2FAD
:10F3E00085E0782E7C0E85E0F82EFC1A86E0E82E6B
:10F3F000EC1A84E0D82EDC1A83E0C82ECC1A82E006
:10F40000982E9C1A93EBA92E98E0B92E81E0882EB5
:10F410008C1AC1114AC08091570F882361F18091E5
:10F420008202882361F0602F619581E09091570FEF
:10F43000911180E024E042E259E00F94799E11118D
:10F4400093C1C53009F022C18091570F853009F46E
:10F45000BBC080918202882361F081E09091570FB8
:10F46000953009F080E023E048EE58E06F2D0F94CE
:10F47000799ED7E07AC18091500F1092500F882367
:10F4800071F20E94BB8E8091520F882341F2DF916E
:10F49000CF911F910F91FF90EF90DF90CF90BF9091
:10F4A000AF909F908F907F900895C13079F58091B3
:10F4B000570F8130D1F080918202882309F4BFCFA9
:10F4C0001F9281E199E09F938F938F9281E09091B9
:10F4D000570F913009F080E08F930E943F8D0F907D
:10F4E0000F900F900F900F90AACF8091500F109215
:10F4F000500F882301F3B092FB0EA092FA0E0E94E7
:10F50000568E8091520F8823B1F2C1CFC23009F0DC
:10F510000EC18091570F8230A1F080918202882322
:10F5200061F081E09091570F923009F080E023E084
:10F5300048E059E0692D0F94799E112309F499CF81
:10F5400013C18091500F1092500F882331F38FE632
:10F5500099E50E9440628091520F8823F1F297CF83
:10F560008091570F833081F080918202882309F4C3
:10F57000F8C081E09091570F933009F080E023E0CC
:10F580004BEF58E06C2DD7CF8091500F1092500F59
:10F59000882351F381E49BE50E9440628091520FE1
:10F5A000882311F374CF8091500F1092500F88234D
:10F5B00009F4C8C088E590E60E9440628091520F2D
:10F5C000882309F4BFC063CF8091500F1092500F71
:10F5D000882309F43ECF86E394E80E94406280913C
:10F5E000520F882309F435CF52CF8091500F1092DB
:10F5F000500F882309F452C080E49EE50E944062C7
:10F600008091520F882309F449C041CF8091500F57
:10F610001092500F882309F4AFC088E19FE70E9441
:10F6200040628091520F882309F4A6C030CF8091A8
:10F63000500F1092500F882309F44BC087EB9CE9C0
:10F640000E9440628091520F882309F442C01FCF6C
:10F650008091500F1092500F882309F453C00E94DC
:10F66000D28E20E040E070E060E082E19DE4DF9136
:10F67000CF911F910F91FF90EF90DF90CF90BF90AF
:10F68000AF909F908F907F900C94D38DC63009F0EF
:10F69000F0CE8091570F863009F4A7CF8091820277
:10F6A000882309F4E6CE81E09091570F963009F057
:10F6B00080E023E04FED58E06E2D0F94799ED7E067
:10F6C00081E08D0F8C1315C08091570F8C1709F4B2
:10F6D000AECF80918202882361F06C2F601B81E0A5
:10F6E0009091570F9C1380E023E04AEC58E00F9470
:10F6F000799E82E08D0F8C1313C09091570F9C1749
:10F7000009F4A6CF80918202882351F06C2F601BF0
:10F7100081E09C1380E023E048EB58E00F94799E51
:10F72000CF5FC71176CEDD5FD093510FB0CEC3301F
:10F7300009F416CFC43009F082CE8091570F84307F
:10F7400009F431CF80918202882359F081E09091B1
:10F75000570F943009F080E023E046EF58E06D2D1C
:10F76000EACE112309F492CFD5E0DC13A9CF809122
:10F77000570F8D1709F44ACF80918202882309F42C
:10F780009FCF6C2F601B81E09091570F9C1380E0FE
:10F7900023E043ED58E00F94799E92CFCF92DF9211
:10F7A000EF92FF9220E030E04AE754E460914A078C
:10F7B00070914B0780914C0790914D070F94CAC2EE
:10F7C0000F94C2CA6B017C0125E030E040E050E0BC
:10F7D0000F94CAC8A7019601261B370B480B590B7B
:10F7E000CA01B9010F946BC220E030E04AE754E44B
:10F7F0000F9450CAFF90EF90DF90CF900895FC01D6
:10F8000080819181A281B38180934A0790934B07B5
:10F81000A0934C07B0934D0720E040E070E060E01B
:10F820008EEE98E40C94D38D8F929F92AF92BF92FC
:10F83000CF92DF92EF92FF921F93CF93DF9300D08E
:10F840001F92CDB7DEB76B017C0120E030E0A9014B
:10F850000F9464C287FD34C06DEB77E386E095E3D7
:10F86000A70196010F9456C96B017C01C982DA8207
:10F87000EB82FC8220E030E040E251EC0F9464C265
:10F88000181654F420E030E048EC52E4C701B60109
:10F890000F94B6CB87FD19C0CE0101960F943B1C87
:10F8A0000F900F900F900F90DF91CF911F91FF90CD
:10F8B000EF90DF90CF90BF90AF909F908F90089582
:10F8C0006DEB77E386E095EBCBCF20E030E040E2D4
:10F8D00051E4C701B6010F94CAC220E030E048EC01
:10F8E00052E40F94CAC24B015C0120E030E0A90150
:10F8F000C701B6010F9464C220E030E040EA50E452
:10F9000087FF04C020E030E040EA50ECC501B401BC
:10F910000F9456C920E030E040E251E40F9450CA01
:10F920000F94C2CA4B015C0120E030E0A901C7017D
:10F93000B6010F94B6CB87FD0BC020E030E040E26B
:10F9400051E4C701B6010F9464C260E287FD13C0A1
:10F95000B7FC42C0C501B40128EE33E040E050E0FE
:10F960000F94CAC8CA01B9012AE030E040E050E073
:10F970000F94CAC8605D6093660FC501B40124E6A8
:10F9800030E040E050E00F94CAC88AE0C82ED12C85
:10F99000E12CF12CCA01B901A70196010F94CAC844
:10F9A000605D6093670F8EE28093680FC501B401BC
:10F9B000A70196010F94CAC8162FCA01B901A70161
:10F9C00096010F94CAC8605D6093690F105D109333
:10F9D0006A0F86E69FE064CFB094A09490948094E0
:10F9E000811C911CA11CB11C6DE2C5CF8F929F920E
:10F9F000AF92BF92CF92DF92EF92FF920F931F933D
:10FA0000CF93DF9361E081E00E94758DC091580F24
:10FA1000AC2E85E0982E9C0ED8E0DC1B87E0F82EFB
:10FA2000FC1A86E0E82EEC1A85E0D82EDC1A84E079
:10FA3000C82ECC1A82E0B82EBC1A8C2E8194C1112B
:10FA40004FC08091570F882391F1809182028823C3
:10FA500059F081E09091570F911180E024E04EE140
:10FA600051E1682D0F94799E8091D81080935B0F9F
:10FA7000C43009F056C010926D0F8091570F84303A
:10FA800009F4E9C080918202882309F4BDC111E024
:10FA90008091570F843009F010E080915B0F0F9434
:10FAA000BD1D00E09C0141E051E16C2D37C080910B
:10FAB000500F1092500F882341F20E94BB8E80910C
:10FAC000520F882311F2DF91CF911F910F91FF9078
:10FAD000EF90DF90CF90BF90AF909F908F90089560
:10FAE000C13009F063C08091570F813009F445C0DF
:10FAF000809182028823A9F011E08091570F813014
:10FB000009F010E080918402909185020F94881D85
:10FB100061E06A1900E09C0148E151E1812F0E94F7
:10FB2000FB9B8091D91080935B0FC53009F0BDC05D
:10FB300081E080936D0F8091570F853009F4A0C04C
:10FB400080918202882391F011E08091570F8530D7
:10FB500009F010E080915B0F0F94BD1D00E09C0147
:10FB600041E051E16D2D812F0E94FB9BCF5F9C12E4
:10FB700066CF89E08093510FA6CF8091500F1092ED
:10FB8000500F882309F4B4CF10E000E027EE33E0F3
:10FB90004AE050E064E872E088E191E10F944CA102
:10FBA0008091520F882309F4A3CF8DCFC23009F082
:10FBB000F2C08091570F8230D1F080918202882369
:10FBC00009F4AFCF11E08091570F823009F010E0B7
:10FBD00080910F1D9091101D0F94881D00E09C01D5
:10FBE00041E151E16B2D812F0E94FB9B3DCF809124
:10FBF000500F1092500F882301F30F94D49F05E209
:10FC00001BE42CE231E050E040E06FE07DE181E177
:10FC100091E10F944CA18091520F882371F253CF40
:10FC20008091500F1092500F882309F4BCC00F949C
:10FC3000D49F03E417ED2CE830E050E040E061EBA6
:10FC40007FE08DE091E10F944CA18091520F8823C9
:10FC500009F4A9C038CF8091500F1092500F88231B
:10FC600009F410CF0F94D49F69E178E381E091E12A
:10FC70000F948BA28091520F882309F403CF23CFD6
:10FC80008091500F1092500F882309F459CF0F9490
:10FC9000D49F69E178E381E091E10F948BA2809198
:10FCA000520F882309F44CCF0ECFC63091F58091C6
:10FCB000570F8630B9F080918202882309F456CF1D
:10FCC00011E08091570F863009F010E080913902E1
:10FCD00090913A020F94881D00E09C014CEF50E196
:10FCE0006E2D41CF8091500F1092500F882319F341
:10FCF00006EF17E327EE33E04AE050E069E372E0F5
:10FD00008CEF90E10F944CA18091520F882399F2CF
:10FD1000DACEC73009F05FC08091570F8730D9F035
:10FD200080918202882309F421CF11E08091570F3E
:10FD3000873009F010E06091D0107091D11080915F
:10FD4000D2109091D3100E94147C00E09C0142EFED
:10FD500050E16F2D08CF8091500F1092500F8823E3
:10FD6000F9F260ED70E182EF90E10F9445A280918D
:10FD7000520F8823A9F2A7CE8091500F1092500FF6
:10FD8000882381F180ED9AE90E9440628091520FB0
:10FD9000882341F198CEC33009F066CE8091570F89
:10FDA000833009F43DCF80918202882309F4B9CED3
:10FDB00011E08091570F833009F010E08091B10F6E
:10FDC0009091B20F0F94881D63E06A1900E09C01C6
:10FDD0004DE051E108CFC83009F0C8CE8091570FEF
:10FDE000883051F280918202882309F4BFCE81E0ED
:10FDF0009091570F983009F080E023E043EE50E1F6
:10FE00006D2F0F94799EB2CE8091D91080935B0FA5
:10FE1000ADCE0F946BC220E030E048EC52E40F947A
:10FE200050CA20E030E0A9010F9456C90C94147C0C
:10FE30002F923F924F925F926F927F928F929F92FA
:10FE4000AF92BF92CF92DF92EF92FF920F931F93E8
:10FE5000CF93DF9300D0CDB7DEB761E081E00E94A1
:10FE6000758D2091580F2A832B83822F8B5F898376
:10FE70008CE0782E721A88E0682E621A8BE0582E79
:10FE8000521A8AE0482E421A89E0382E321A87E048
:10FE9000282E221A2A812111ECC08091570F882325
:10FEA00009F4C3C080918202882361F06B8161955F
:10FEB00081E09091570F911180E024E043E958E0F0
:10FEC0000F94799E2CEA35EC47E25EE36091161DB3
:10FED0007091171D8091181D9091191D0F9450CA93
:10FEE00060933407709335078093360790933707F4
:10FEF0002CEA35EC47E25EE360911A1D70911B1D00
:10FF000080911C1D90911D1D0F94CAC260933007F3
:10FF10007093310780933207909333078A8185303D
:10FF200009F0C5C110926D0F8091570F853009F40B
:10FF3000A7C1809182028823D1F011E08091570FF0
:10FF4000853009F010E06091121D7091131D8091B1
:10FF5000141D9091151D0E94894F65E02B81621B35
:10FF600000E09C014CE857E0812F0E94FB9B2CEAAB
:10FF700035EC47E25EE36091B80F7091B90F809164
:10FF8000BA0F9091BB0F0F9450CA609334077093CF
:10FF9000350780933607909337072CEA35EC47E214
:10FFA0005EE36091BC0F7091BD0F8091BE0F909188
:10FFB000BF0F0F94CAC260933007709331078093CC
:10FFC0003207909333079A81993009F099C28FEFE5
:10FFD00080936D0F8091570F893009F47AC2809118
:10FFE00082028823C1F011E08091570F893009F017
:10FFF00010E06091B40F7091B50F8091B60F9091A1
:020000021000EC
:10000000B70F0E94894F00E09C014CE857E0632D38
:10001000812F0E94FB9B9A819F5F9A832981921373
:1000200039CF8DE08093510F0EC08091500F109208
:10003000500F882309F436CF0E94BB8E8091520F57
:10004000882309F42FCF0F900F900F90DF91CF915D
:100050001F910F91FF90EF90DF90CF90BF90AF90E6
:100060009F908F907F906F905F904F903F902F90D8
:1000700008958A81813091F59091570F9130D1F098
:1000800080918202882309F41DCF61E08B81681B77
:1000900081E0913009F080E09091DC0C2EEA37E0AD
:1000A000911102C02AEA37E001E041EB57E00E94DB
:1000B000FB9B08CF8091500F1092500F882301F3C3
:1000C0008091DC0C2A8182278093DC0C83E0809372
:1000D00082028091520F882399F2B5CF9A81923093
:1000E00009F0CEC28091570F823009F468C0809128
:1000F00082028823B1F011E08091570F823009F01D
:1001000010E080913702909138020F94881D62E0D0
:100110002B81621B00E09C0143EA57E0812F0E9483
:10012000FB9B2CEA35EC47E25EE36091161D709173
:10013000171D8091181D9091191D0F9450CA60933E
:1001400034077093350780933607909337072CEA6E
:1001500035EC47E25EE360911A1D70911B1D8091A2
:100160001C1D90911D1D0F94CAC26093300770939F
:10017000310780933207909333079A81983009F0C2
:10018000F6CE10926D0F8091570F883009F486C11A
:1001900080918202882309F4B3C011E08091570F47
:1001A000883009F010E080910202909103020F94D0
:1001B000881D00E09C014DE657E0662DD5CE80916C
:1001C000500F1092500F882309F491CF10E000E0F7
:1001D0002CE231E050E040E067E372E083EA97E030
:1001E0000F944CA18091520F882309F480CF2BCF1C
:1001F0008091570F8330D1F080918202882309F4D7
:1002000090CF11E08091570F833009F010E080917A
:100210003502909136020F94881D63E02B81621B9A
:1002200000E09C014CE957E0812F41CF8091500FB5
:100230001092500F882301F310E000E02CE231E02F
:1002400050E040E065E372E08CE997E00F944CA148
:100250008091520F882381F2F6CE8091500F109238
:10026000500F882309F418C261E372E084E997E033
:100270000F9445A28091520F882309F40DC2E3CE5A
:100280008091500F1092500F882309F452CE0F9492
:10029000D49F50E040E062E17DE18CE897E00F946C
:1002A000F9A18091520F882309F443CECCCE8A81E4
:1002B000863009F0B9C010926D0F8091570F8630CB
:1002C00009F46DC0809182028823D1F011E0809101
:1002D000570F863009F010E06091340770913507B0
:1002E00080913607909137070E94933866E02B8102
:1002F000621B00E09C0144E857E0812F0E94FB9BB9
:100300002CEA35EC47E25EE36091B80F7091B90FCB
:100310008091BA0F9091BB0F0F9450CA609334072D
:100320007093350780933607909337072CEA35ECA6
:1003300047E25EE36091BC0F7091BD0F8091BE0FEC
:100340009091BF0F0F94CAC260933007709331072A
:1003500080933207909333072A812C3009F05BCECB
:100360008FEF80936D0F8091570F8C3009F46DC122
:1003700080918202882309F44ECE11E08091570FBC
:100380008C3009F010E080910002909101020F94EE
:10039000881D00E09C014DE657E0672D39CE809125
:1003A000500F1092500F882309F48CCF0F94D49FD4
:1003B00020E030E048EC52E460913407709135075A
:1003C00080913607909137070F94CAC220E030E041
:1003D000A9010F9456C920E030E040E85FE30F9494
:1003E00055C90F94C9CA1F9232ED832E35E8932E5A
:1003F00044EAA42E40E4B42E6B0117E5E12E1EE37F
:10040000F12E0FE010E021E030E040E050E064E346
:1004100077E084E897E00E94F98E0F908091520F68
:10042000882309F44FCF0FCE8A81873009F0A5CEFB
:1004300010926D0F8091570F8730D9F08091820212
:10044000882309F45DCF11E08091570F873009F0C0
:1004500010E06091300770913107809132079091E0
:1004600033070E94894F00E09C014CE757E0622D62
:100470007BCD8091500F1092500F8823F9F20F948A
:10048000D49F4BEB55E860E377E08CE797E00F945F
:10049000F9A18091520F882389F2D5CD8091500F18
:1004A0001092500F882309F473CE0F94D49F04E860
:1004B0001FE52CE231E046E950E062E072E08DE6B3
:1004C00097E00F944CA18091520F882309F460CEDD
:1004D000BACD8091500F1092500F882309F47FCD30
:1004E0000F94D49F50E040E064EB7FE08CE897E00D
:1004F0000F94F9A18091520F882309F470CDA3CDF8
:100500002A812A3009F066C08FEF80936D0F8091A9
:10051000570F8A30D9F080918202882309F47BCD6D
:1005200011E08091570F8A3009F010E06091340794
:100530007091350780913607909137070E94933864
:1005400000E09C0144E857E0642D62CD8091500F9B
:100550001092500F8823F9F20F94D49F20E030E0DE
:1005600048EC52E46091340770913507809136076A
:10057000909137070F94CAC220E030E0A9010F9490
:1005800056C920E030E040E85FE30F9455C90F946E
:10059000C9CA1F928CEE882E8BE3982E94EAA92E5E
:1005A00090E4B92E6B0117E5E12E1EE3F12E0FE06A
:1005B00010E021E030E040E050E064E377E084E8E0
:1005C00097E00E94F98E0F908091520F882309F4D2
:1005D000A2CF39CD8A818B3009F0BECE8FEF8093C8
:1005E0006D0F8091570F8B30D9F080918202882354
:1005F00009F411CD11E08091570F8B3009F010E014
:1006000060913007709131078091320790913307E4
:100610000E94894F00E09C014CE757E0652DF8CC23
:100620008091500F1092500F8823F9F20F94D49FAD
:1006300045ED5BE360E377E08CE797E00F94F9A189
:100640008091520F882389F2FECC8091500F109236
:10065000500F882309F48CCE0F94D49F01E81FE536
:100660002CE830E046E450E060E072E08DE697E090
:100670000F944CA18091520F882309F479CEE3CCDA
:100680008A81833009F4B4CD843009F01BCC809189
:10069000570F843009F4E1CD80918202882309F458
:1006A00040CD11E08091570F843009F010E0609147
:1006B00031027091320280913302909134020E9493
:1006C000147C64E02B81621B00E09C0144E957E04C
:1006D000ABCD61116093050240933F078C3008F069
:1006E0003AC0E82F880FFF0B8827E658FC478F4F4A
:1006F0000D944DC9AD8386839183B0839483978392
:100700009A83A6839D83AB83A083A38381EC96E524
:1007100021E02093450720E040E070E060E00C9489
:10072000D38D89EC96E5F4CF8DEC96E5F1CF81ED94
:1007300096E5EECF85ED96E5EBCF89ED96E5E8CF32
:100740008DED96E5E5CF81EE96E5E2CF1092970F1D
:1007500087E79FE3DDCF0C94568E8DEB96E5D8CFDF
:1007600085EC96E5D5CFCF92DF92EF92FF926B01A9
:100770007C0120E030E0A9010F9464C287FD26C00F
:100780006DEB77E386E095E3A70196010F9456C9D8
:100790006B017C0120E030E0A9010F9464C220E0ED
:1007A00030E040E05FE387FF04C020E030E040E05D
:1007B0005FEBC701B6010F9456C90F94C2CACB01B3
:1007C000FF90EF90DF90CF900D94DE1C6DEB77E300
:1007D00086E095EBD9CF0F946BC220E030E0A90101
:1007E0000F9456C90C94B383CF92DF92EF92FF928D
:1007F000CF93DF9300D01F92CDB7DEB76B017C01A2
:1008000020E030E0A9010F9464C287FD1BC06DEBAE
:1008100077E386E095E3A70196010F9456C96983B3
:100820007A838B839C83CE0101960F94BA9E0F909E
:100830000F900F900F90DF91CF91FF90EF90DF908E
:10084000CF9008956DEB77E386E095EBE4CF0F94BE
:100850006BC220E030E04AE754E40F9450CA20E035
:1008600030E0A9010F9456C90C94F4834F925F9223
:100870006F927F928F929F92AF92BF92CF92DF92B0
:10088000EF92FF920F931F93CF93DF9361E081E08C
:100890000E94758DC091580F65E0562E5C0ED3E016
:1008A000DC1B82E0782E7C1A81E0682E6C1A4C2EBC
:1008B0004194C11137C08091570F8823B1F08091C6
:1008C0008202882359F081E09091570F911180E0C6
:1008D00024E043E958E0642D0F94799ECF5FC51161
:1008E000E8CF84E08093510F0CC08091500F10929C
:1008F000500F882321F30E94BB8E8091520F8823D2
:10090000F1F2DF91CF911F910F91FF90EF90DF9067
:10091000CF90BF90AF909F908F907F906F905F909F
:100920004F900895C13009F061C08091570F813018
:10093000E9F080918202882389F211E08091570FBB
:10094000813009F010E060919C1D70919D1D809197
:100950009E1D90919F1D0E94493900E09C0148E531
:1009600058E0662D812F0E94FB9BB8CF8091500FDD
:100970001092500F8823E9F220E030E040E251E489
:1009800060919C1D70919D1D80919E1D90919F1D59
:100990000F94CAC220E030E0A9010F9456C920E0AC
:1009A00030E44CE955E40F9456C90F94C9CA1F921C
:1009B000912C812C4CE8A42E40E4B42E6B0110E164
:1009C000E12E17E2F12E00E010E028E73CEE4FEFB9
:1009D0005FEF6CE97DE188E598E00E94F98E0F9069
:1009E0008091520F882309F4A4CF8BCFC23009F035
:1009F0009FC08091570F8230D9F080918202882366
:100A000009F46CCF11E08091570F823009F010E0AB
:100A10006091A01D7091A11D8091A21D9091A31DB8
:100A20000E94493900E09C0149E458E0672D9ACFC3
:100A30008091500F1092500F8823F9F220E030E09F
:100A400040E251E46091A01D7091A11D8091A21D12
:100A50009091A31D0F94CAC220E030E0A9010F9429
:100A600056C920E030E44CE955E40F9456C90F9480
:100A7000C9CA1F92912C812C2CE8A22E20E4B22E00
:100A80006B0110E1E12E17E2F12E00E010E028E703
:100A90003CEE4FEF5FEF60EA7DE189E498E00E9471
:100AA000F98E0F908091520F882309F4A6CF29CF99
:100AB0008091500F1092500F882309F441C020E01C
:100AC00030E04AE754E46091A41D7091A51D809127
:100AD000A61D9091A71D0F94CAC220E030E0A90185
:100AE0000F9456C920E030EA4CE056E40F9456C902
:100AF0000F94C9CA1F92912C812C8CEBA82E80E4F4
:100B0000B82E6B0110E5E12E16E4F12E00E010E0A6
:100B100028ED3CED4FEF5FEF64EA7DE18AE398E07A
:100B20000E94F98E0F908091520F882349F0E9CEF0
:100B3000C33009F0D3CE8091570F833009F4B8CF7A
:100B400080918202882309F4C9CE11E08091570F69
:100B5000833009F010E06091A41D7091A51D809173
:100B6000A61D9091A71D0E94F48300E09C014AE31A
:100B700058E06D2FF7CE2CEA35EC47E25EE360914A
:100B800030077091310780913207909133070F94AD
:100B900050CA60931A1D70931B1D80931C1D909367
:100BA0001D1D08952CEA35EC47E25EE360913407A1
:100BB0007091350780913607909137070F94CAC21C
:100BC0006093161D7093171D8093181D9093191D27
:100BD000089580915B0F90915C0FA0915D0FB09193
:100BE0005E0F8093550290935602A0935702B093E4
:100BF00058020895FC0184910895FC0180810895B4
:100C0000FC01A081B1811C92A281B3818C918F5F84
:100C10008C930280F381E02D90818CE0989F800D71
:100C20001124E5EEFDE113AE84AF089511980000A4
:100C300000009091020187FD9095917090930001C2
:100C4000119A000000000000000011980000000050
:100C50009091020186FD9095917090930001119AF8
:100C600000000000000000001198000000009091BA
:100C7000020185FD9095917090930001119A0000FA
:100C80000000000000001198000000009091020197
:100C900084FD9095917090930001119A00000000DE
:100CA000000000001198000000009091020183FDF7
:100CB0009095917090930001119A0000000000003F
:100CC00000001198000000009091020182FD9095B3
:100CD000917090930001119A000000000000000044
:100CE0001198000000009091020181FD9095917093
:100CF00090930001119A000000000000000011987C
:100D00000000000080910201817080930001119A1F
:100D10000000000000000000089590E080E00895C9
:100D200090E080E00895282F9091A50F833021F462
:100D300095FD0FC094FD0FC0892F90E0B0E0A0E0BA
:100D400004C0B695A795979587952A95D2F7817097
:100D5000089581E0089580E008950F931F93CF9345
:100D60008C01C62F87EE9CE10F94D54AC8010F94E1
:100D7000D54A8AE30F94484A80E38C0F0F94484A7F
:100D80008AE0CF911F910F910D94484A8AE69EE127
:100D90000F94D54A60E08AE59EE10E94AD8660E04E
:100DA00085E49EE10E94AD8661E08EE39EE10E94B3
:100DB000AD8661E083E39EE10E94AD8661E083E25F
:100DC0009EE10E94AD8660E08AE19EE10E94AD86D0
:100DD00061E080E19EE10E94AD8661E086E09EE1F7
:100DE0000E94AD8661E08FEF9DE10E94AD8661E0DB
:100DF00087EF9DE10E94AD8661E089EE9DE10E9452
:100E0000AD8661E08BED9DE10E94AD8660E08CECEB
:100E10009DE10E94AD8660E08EEB9DE10E94AD8673
:100E200060E088EA9DE10E94AD8661E087E99DE18E
:100E30000E94AD8661E088E89DE10E94AD8661E098
:100E400081E89DE10E94AD8660E08AE79DE10E9415
:100E5000AD8661E081E79DE10E94AD8661E08CE5B1
:100E60009DE10E94AD8661E08EE49DE10E94AD8629
:100E700061E08BE39DE10E94AD8660E08EE29DE142
:100E80000E94AD8661E089E29DE10E94AD8661E04D
:100E90008CE19DE10E94AD8660E088E09DE10E94CA
:100EA000AD8660E085EF9CE10E94AD8660E083E363
:100EB0009EE10E949086682F61708CEE9CE10C94FC
:100EC000AD86AF92BF92CF92DF92EF92FF920F93D7
:100ED0001F93CF93DF936B01E9014A3009F4C1C03E
:100EE000453109F073C0DB011296ED91FC91F2805F
:100EF000C681D78180910201809582708093000124
:100F000088E28A950000E9F7BF2CB29420EFB22264
:100F100030E1A32EAF0C48E2E42E88EF0E94168643
:100F20008E2D8A950000E9F7BFE1BF1508F485C052
:100F30008F2D807780680E9416868B2D0E941686E2
:100F40008E2D8A950000E9F780E80E94168680E0E1
:100F50000E9416868E2D8A950000E9F78AEF0E947E
:100F600016868E2D8A950000E9F78E01005F1F4FCF
:100F70008881807F0E94168689918295807F0E9459
:100F80001686C017D107A1F78E2D8A950000E9F7C4
:100F9000F394E0E1BE0EFA10C0CF8091020182709E
:100FA00080930001D6011296CD91DC91CE010F9471
:100FB00086AB811147C2DF91CF911F910F91FF90B6
:100FC000EF90DF90CF90BF90AF900895FB0102812A
:100FD0001381423309F4F1C108F4F5C1463409F430
:100FE000E2C1473409F4E5C14B3329F589812B81EE
:100FF000D80112966C91129713964C91213009F4F6
:1010000038C2233009F002C238EF380F582F91E070
:10101000431708F490E041E0531708F040E031E056
:10102000561708F430E0592F542B352309F016C217
:10103000942309F013C281E0BECF80EE8F0D80684B
:10104000807F0E9416868F2D8295807F0E94168653
:101050008E2D8A950000E9F780E80E94168680E8C8
:1010600077CF80910101826080930101809102011C
:101070008270809300018091010181608093010161
:1010800080910201817080930001099A119A8091E8
:101090000201809582708093000188E28A950000A9
:1010A000E9F788E790E0CEE9DFE0FE013197F1F75C
:1010B0000197D9F788EF0E94168618E2812F8A954A
:1010C0000000E9F780E20E94168680E00E94168602
:1010D000812F8A950000E9F780E00E94168680E85B
:1010E0000E941686812F8A950000E9F780E00E9411
:1010F000168680E10E941686812F8A950000E9F706
:10110000CE010197F1F7CE010197F1F7CE010197DA
:10111000F1F7CE010197F1F7CE010197F1F7CE017A
:101120000197F1F7CE010197F1F7CE010197F1F7A1
:10113000CE010197F1F7CE010197F1F7CE010197AA
:10114000F1F7CE010197F1F7CE010197F1F7CE014A
:101150000197F1F72197F1F780E20E94168680E46B
:101160000E941686812F8A950000E9F780E20E948E
:10117000168680E60E9416861A950000E9F710E0B0
:10118000D0E0C8E28D2F807780680E941686812F7C
:101190000E9416868C2F8A950000E9F780E80E944D
:1011A000168680E00E9416868C2F8A950000E9F74B
:1011B0008AEF0E9416868C2F8A950000E9F790E24C
:1011C000119800000000809102018170809300015D
:1011D000119A0000000000000000119800000000BB
:1011E00080910201817080930001119A000000003B
:1011F0000000000011980000000080910201817041
:1012000080930001119A0000000000000000119876
:101210000000000080910201817080930001119A0A
:101220000000000000000000119800000000809104
:101230000201817080930001119A000000000000FB
:1012400000001198000000008091020181708093DD
:101250000001119A00000000000000001198000039
:10126000000080910201817080930001119A0000BA
:1012700000000000000011980000000080910201B1
:10128000817080930001119A0000000000000000AE
:10129000119800000000809102018170809300018C
:1012A000119A0000000000000000119800000000EA
:1012B00080910201817080930001119A000000006A
:1012C0000000000011980000000080910201817070
:1012D00080930001119A00000000000000001198A6
:1012E0000000000080910201817080930001119A3A
:1012F0000000000000000000119800000000809134
:101300000201817080930001119A0000000000002A
:10131000000011980000000080910201817080930C
:101320000001119A00000000000000001198000068
:10133000000080910201817080930001119A0000E9
:1013400000000000000011980000000080910201E0
:10135000817080930001119A0000000000000000DD
:101360008C2F8A950000E9F7915009F029CF88EF7A
:101370000E9416868C2F8A950000E9F7DF5F105FC8
:10138000D03209F0FFCE80E00E94168680EC0E94E9
:101390001686CA950000E9F7809102018270809359
:1013A000000181E008CED80115968C91888381E0F8
:1013B00002CEF80181818883FACFB901C8010F9468
:1013C000A3AB81E0F8CD443171F0473109F033CE61
:1013D0001882F80182818983858181508A83838183
:1013E0008B8381E0E8CDD80115964C91159750E09C
:1013F000440F551F70E060E016968D919C910F94FC
:10140000D9CDC8010F949CAB81E0D5CD481708F425
:1014100012CE861708F40FCEFA80E12CD12C24309E
:1014200070F41DC0BE01C8010F94A3AB89819881DF
:101430009D0D98838E0D8983FF0C09F4FCCDF7FE7A
:10144000F6CFF0CF4D8150E0440F551F70E060E0C3
:101450008E819F810F94D9CD81E0ADCDFA8030E0AF
:10146000F901EA50FD4FD0802E503D4FF901E08048
:10147000E6CF58E0580F382FCACDEF92FF920F9366
:101480001F93CF93DF93EC018B017A018A859B85B3
:101490008617970731F0888199810F947CAD1B875F
:1014A0000A87B701888199810F94A09F2E813F817F
:1014B000820F932F911D9F838E8390E080E0DF91B8
:1014C000CF911F910F91FF90EF9008959F92AF924F
:1014D000BF92CF92DF92EF92FF920F931F93CF9321
:1014E000DF93EC018B01942EA52E8A859B858617B0
:1014F000970731F0888199810F947CAD1B870A870B
:1015000088859985019649F5BC800A818E81080FEE
:10151000C880D980D6015596ED91FC91C6011995E8
:10152000B80EE92CFA2C10E0F70121917F0121116E
:1015300027C08E819F81810F911D9F838E8390E0B4
:1015400080E0DF91CF911F910F91FF90EF90DF909E
:10155000CF90BF90AF909F9008950E811F81692D0D
:101560007A2D888199810F94A09F800F912F911DD2
:10157000288539852817390738F681E090E0E1CFD2
:101580004B2D602FC6010F94D4AD080F180FCCCF90
:10159000DF92EF92FF920F931F93CF93DF93EC01B3
:1015A000D62E1CAD0BAD7C0184E0E80EF11CE98D5C
:1015B000FA8DC7011995412F480F2D2D602FC701B6
:1015C0000F94D4AD9BAD890F8BAF81E090E0DF919C
:1015D000CF911F910F91FF90EF90DF900895CF92E0
:1015E000DF92EF92FF920F931F93CF93DF93CDB7CC
:1015F000DEB72C970FB6F894DEBF0FBECDBFF090CC
:10160000201EE090211E20918F0821111DC044EE64
:1016100051E26E2D8F2D0F9440AE90E080E0F80ED9
:10162000F092201EE092211E99272C960FB6F89476
:10163000DEBF0FBECDBFDF91CF911F910F91FF9005
:10164000EF90DF90CF900895C090ED1DD090EE1DEB
:1016500029EE3DE13A8329832F2D30E03C832B8313
:101660002E2D30E03E832D8318861F827A8769876E
:101670001C861B8606E61AE89E012F5F3F4F4AEF45
:1016800055E8BC01C6010F949F86B60189EE9DE125
:101690000F947CAD8F819885C2CFCF93C62F0F94C6
:1016A000983D882319F0CF910D94F23C8C2FCF9167
:1016B0000895CF93DF93EB010F94983D882319F0A1
:1016C0000F94E23CEB01CE01DF91CF9108950F938F
:1016D0001F93CF93DF9300D01F92CDB7DEB79C014D
:1016E0000FE71FE090E1EBE9F0E1D80101900D92E6
:1016F0009A95E1F7F9012081318142815381F80106
:1017000060857185828593850F9456C9F80160873D
:1017100071878287938780E090E0A0EAB0E48983B4
:101720009A83AB83BC83CE0101960F94340C0F9047
:101730000F900F900F90DF91CF911F910F9108950F
:10174000CF9384E50F94983DC0E08823D9F00F949F
:10175000F23CC82F1816B4F40F941A5E8DE40F945F
:10176000484A80918808909189080F947BAF6C2F2C
:10177000CC0F770B86E799E10F94CA4D8AE00F945E
:10178000484ACFEF8C2FCF91089583E50F94983D71
:101790008823E9F00F94D5A560938F0F7093900F75
:1017A0008093910F9093920F0F941A3D20E030E0B8
:1017B0004AE754E40F94CAC20F94C9CA60931D0249
:1017C00070931E0280931F029093200208958091CF
:1017D0007D0784FD13C080917F0787FD0FC0809136
:1017E0008007837059F40E9470EE8091440788232B
:1017F00021F0109244071092450708950E945FEE71
:1018000088E50F944A3D882331F05F9A8091F70E66
:101810008E7F8093F70E89E50F944A3D882331F03F
:101820008A9A8091F70E8D7F8093F70E8AE50F9448
:101830004A3D882359F080910801809581708093FA
:1018400006018091F70E8B7F8093F70E85E40F944D
:101850004A3D882351F20F94AF47C7CF809152077A
:1018600090915307009731F04AE050E070E060E05B
:101870000D9442C060E070E0CB01089580917D0737
:10188000827149F480917F078C7829F480918007D8
:10189000837009F475C082E40F944A3D882351F0A7
:1018A0000E942E8C6093AD177093AE178093AF1784
:1018B0009093B01783E50F944A3D882351F00F941D
:1018C0001A3D6093DD177093DE178093DF179093B6
:1018D000E01784E50F944A3D882351F00F941A3D98
:1018E0006093E1177093E2178093E3179093E417E6
:1018F00088E50F944A3D882351F00F941A3D609378
:10190000C0107093C1108093C2109093C31089E5EA
:101910000F944A3D882351F00F941A3D6093C410F0
:101920007093C5108093C6109093C7108AE50F94EA
:101930004A3D8823B1F00F941A3D6093C81070930C
:10194000C9108093CA109093CB102DEC3CEC4CEC5A
:101950005DE30F9464C2181624F08CE798E10F94AD
:10196000D54A85E40F944A3D882351F00F941A3DDF
:101970006093CC107093CD108093CE109093CF10C5
:101980000895AF92BF92CF92DF92EF920F931F9381
:10199000CF93DF935B01EA016901882309F463C0F7
:1019A00085E798E10F94D54AF501608171818281C4
:1019B000938146E00F94D825E1100BC08CE698E1A6
:1019C0000F94D54A688179818A819B8146E00F9482
:1019D000D82585E698E10F94D54AF601608171819A
:1019E0008281938143E00F94D8258EE598E10F948E
:1019F000D54AF801608171818281938143E00F941F
:101A0000D82585E598E10F94D54AF60120813181EA
:101A100042815381F80160817181828193810F94A9
:101A200055C943E00F94D825EE20F9F08AE00F94D1
:101A3000484A80E498E10F94D54A688179818A8187
:101A40009B8146E00F94D8258AE00F94484A8AE0AB
:101A5000DF91CF911F910F91EF90DF90CF90BF90CA
:101A6000AF900D94484AE110E4CFDF91CF911F91E0
:101A70000F91EF90DF90CF90BF90AF900895CF93EC
:101A8000DF93CDB7DEB720E2488559856F818E811F
:101A90000F94799EDF91CF9108954FE350E0BC0100
:101AA0008CEF9EE00D941ECE63E972E084E690E038
:101AB0000E94EA5F6AEB72E084E690E00C94EA5FD1
:101AC00081110C94548D68EB71E084E190E00C94EA
:101AD000EA5F0E9424EA0C94608D0F947C310C9490
:101AE000608D0F9494140C94548D282F1092630FD2
:101AF0008091530F9091540FA091550FB091560FB4
:101B0000B7FF08C01092530F1092540F1092550F48
:101B10001092560F80914307882331F08091530F24
:101B20008093570F1092520F8091510F1816FCF4AA
:101B3000082E000C990B821B91092091570F022E41
:101B4000000C330B2817390794F097FF02C090E080
:101B500080E08093570F092E000CAA0BBB0B8093DB
:101B6000530F9093540FA093550FB093560F80913D
:101B7000570F6623A9F09091580F891714F480939A
:101B8000580F2091580F022E000C330B2C5F3F4F43
:101B9000482F082E000C550B241735071CF48450D1
:101BA0008093580F08958F929F92AF92BF92EF92B9
:101BB000FF920F931F93CF93DF93EC018B01E42EE1
:101BC000F22E8091E31D9091E41D8C179D0709F47E
:101BD00040C020911E0927FD10921E0921E7C9313E
:101BE000D20709F041C082559F4971F40F94D5A5E1
:101BF0006E517B4F8F4F9F4F609320097093210947
:101C00008093220990932309D093E41DC093E31D90
